:020000040800F2
:1000000000000220512F0108D9920008DB9200085D
:10001000DD920008DF920008E19200080000000075
:10002000000000000000000000000000E392000853
:10003000E592000800000000E7920008E99200083D
:10004000952F0108952F0108952F0108952F01087C
:10005000952F0108952F0108952F0108952F01086C
:10006000952F0108952F0108952F01087976000832
:10007000952F0108952F0108952F0108952F01084C
:10008000952F0108952F0108952F0108952F01083C
:10009000952F0108952F0108952F01080995000853
:1000A000952F0108952F0108952F0108952F01081C
:1000B000E5940008952F0108952F0108952F010858
:1000C000952F0108952F0108952F0108952F0108FC
:1000D000952F0108952F01081D960008952F0108FE
:1000E000952F0108952F0108ED920008952F010822
:1000F000952F0108952F0108952F0108952F0108CC
:10010000952F0108952F0108952F0108952F0108BB
:10011000952F0108952F0108952F0108952F0108AB
:10012000952F0108952F0108952F0108952F01089B
:10013000952F0108952F0108952F0108952F01088B
:10014000952F0108952F0108952F01081D93000890
:10015000952F0108952F0108952F0108952F01086B
:10016000952F0108952F0108952F0108952F01085B
:10017000952F0108952F0108952F0108952F01084B
:08018000952F0108952F0108DD
:10018800D4B2050800000020080C0020080C00204C
:10019800A43C002008B5074B186809F03BF80DF09F
:1001A8002BFE054B054806221A70BDE8084001F0F1
:1001B800C4BB00BF10260020A4250020800F00200B
:1001C80008B5034801F0B9FB024B00221A7008BDBC
:1001D800D4170020A425002008B5054B01220020D3
:1001E8001A7005F041FD0348BDE8084001F0A5BBC1
:1001F800282C0020441500202DE9F041144C2046FD
:1002080003F091FE00201349134A03F043FC1349FD
:10021800134A0746002003F03DFC1249124A0646DD
:10022800002003F037FCD22105463A4623460A202F
:1002380003F048FDD22132462346FA2003F042FD5E
:100248005A20D2212A462346BDE8F04103F03ABDA0
:1002580058130020469F0508C90100084F9F05084C
:10026800E1010008579F05089D01000808B5054BE6
:10027800012200201A7005F0F7FC0348BDE8084089
:1002880001F05BBB282C00204415002008B503486A
:1002980001F053FB024B00221A7008BDD41700204E
:1002A800A425002008B5054B07221A700DF0A4FDFF
:1002B8000348BDE8084001F040BB00BFA42500206A
:1002C800581300202DE9F041144C204603F02BFE72
:1002D80000201349134A03F0DDFB1349134A07466C
:1002E800002003F0D7FB1249124A0646002003F00B
:1002F800D1FBD22105463A4623460A2003F0E2FC08
:10030800D221324623465A2003F0DCFCAA20D2210F
:100318002A462346BDE8F04103F0D4BC800F0020F4
:10032800469F050895020008609F0508AD02000871
:10033800699F050875020008014801F0FEBA00BF70
:100348006C11002010B5094C204603F0ECFD00208C
:100358000749084A03F09EFBD221024623464FF480
:100368008270BDE8104003F0ADBC00BF8C160020C1
:10037800729F05084103000870B50C4C0C4D2068AD
:100388004FF6E076314602F0C9FE2068294602F0B1
:1003980073FE6068314602F0C1FE6068294602F0CB
:1003A8006BFEBDE8704003F0F7BF00BF080C0020EB
:1003B80061A5050838B52B4CFFF7DEFF002005F0D6
:1003C80053FC237A23B90A203221274A05F05AFD23
:1003D800637A23B90A206421244A05F053FD214C8D
:1003E800A37A23B90A209621214A05F04BFDA37A66
:1003F8001C4DFBB16B7AEBB12B7ADBB100232B726E
:100408006B72AB721B4B286801221A704FF6E071B1
:1004180002F084FE2868184902F02EFE6868174921
:1004280002F02AFE0BF0E5F903F0B6FF144803F0DA
:10043800F7FF0DE00B4C4FF47841206802F06EFE98
:100448002068104902F018FE60680F4902F014FE97
:10045800FFF792FF00200BF08FF90C48BDE83840F9
:1004680001F06BBA080C0020799F0508879F0508E2
:10047800969F0508A4250020A49F050862A50508E5
:1004880080969800B89F050864A50508D417002031
:1004980008B500200BF070F90248BDE8084001F0EB
:1004A8004CBA00BFD417002038B5FFF765FF0DF030
:1004B800BBFC3C213F220023DF2005F0C5FC4FF4A4
:1004C80080600EF035FA124C3E223C21DF200023DA
:1004D80005F0BAFC012323720E4B4FF6E07518683D
:1004E80008F098FE2068294602F018FE20680A499C
:1004F80002F0C2FD6068294602F010FE60680749F4
:1005080002F0BAFD03F048FF054B00221A7038BD0F
:10051800080C002010260020CA9F0508DD9F05084A
:10052800A425002038B5FFF727FF0DF07DFC6E21CC
:100538003F220023DF2005F087FC4FF486400EF0B1
:10054800F7F9124C3E226E21DF20002305F07CFCD7
:10055800012363720E4B4FF6E075186808F05AFED7
:100568002068294602F0DAFD20680A4902F084FD75
:100578006068294602F0D2FD6068074902F07CFDF8
:1005880003F00AFF054B00221A7038BD080C002042
:1005980010260020F09F050801A00508A4250020CA
:1005A80010B5FFF7E9FE0DF03FFCA0213F22002324
:1005B800DF2005F049FC4FF402400EF0B9F9114C68
:1005C8003E22A021DF20002305F03EFC0123A37278
:1005D8000D4B186808F01EFE20684FF6E07102F017
:1005E8009DFD2068094902F047FD6068084902F04E
:1005F80043FD03F0D1FE64200AF098FF054B00226A
:100608001A7010BD080C00201026002012A0050842
:1006180062A50508A42500202DE9F74F3A4D3B4E69
:100628000024284603F07FFC224623464FF6FF713C
:1006380037480094019402F035FD4FF6E07804271E
:10064800F06041462246234632480097019402F062
:1006580029FD23463060414622462F4800970194E1
:1006680002F020FD2D4970602D4A204603F012FA51
:100678002C492D4A0746204603F00CFA2B492C4AF0
:100688008046204603F006FA2A492B4A814620462E
:1006980003F000FA29492A4A8346204603F0FAF96A
:1006A80021468246F2682B46204603F00BFB5A216E
:1006B80032682B460A2003F005FB6E2172682B4630
:1006C8000A2003F0FFFA9B213A462B46FA2003F052
:1006D800F9FA692142462B46FA2003F0F3FA37214A
:1006E8004A462B46FA2003F0EDFAC82152462B461B
:1006F800AA2003F0E7FAF020C8215A462B4603B097
:10070800BDE8F04F03F0DEBAFC130020080C00200F
:1007180026A005082EA0050841A0050850A0050838
:10072800A905000858A005082D05000848A00508D7
:10073800B104000860A005089904000867A005082E
:10074800BD03000838B50C4C4FF6E0752068294603
:1007580002F0E4FC2068094902F08EFC6068294632
:1007680002F0DCFC6068064902F086FC03F014FE27
:10077800BDE8384003F010BE080C00202EA0050884
:100788006EA0050870B52DED028B9FED248A88B008
:100798000A26F0EE488A03E0B0EE608AF0EE418A5D
:1007A8000CF07BFA8DED000ACDED010A9DE80300FF
:1007B80004AB83E80300F0EE680AB0EE480A9DED4A
:1007C800041ADDED051A8DED028ACDED038A0CF0D1
:1007D80007F8CDED010A8DED000A9DE8030002AD92
:1007E80085E80300013E6C46DDED020A9DED031A23
:1007F800D2D19FED0B0A0CF047FA8DED000ACDED32
:10080800010A9DE8030085E80300DDED030A9DED7C
:10081800020A08B0BDEC028B70BD00BF00000000EA
:10082800CDCCCC3D2DE9F74F564D574CDFF86491B0
:10083800DFF864814FF6E07005F0EAF9286811F0F6
:100848008BFA064668680F4611F086FA3246CDE9FB
:1008580000013B464946204616F0F4F8224600239C
:100868000520372105F00EFB2869484F484E11F046
:1008780073FA824668698B4611F06EFA5246CDE9E2
:1008880000015B463946204616F0DCF82246002374
:100898000520692105F0F6FA286B11F05DFA824609
:1008A800686B8B4611F058FA5246CDE900015B4659
:1008B8004146204616F0C6F8002305209B21224613
:1008C80005F0E0FA31462A6C204616F0BBF82246BD
:1008D80000239B21A22005F0D5FA4FF4FC6005F017
:1008E80097F9A86811F038FA8246E8688B4611F043
:1008F80033FA5246CDE900015B464946204616F0D8
:10090800A1F8224605205021002305F0BBFAA8696A
:1009180011F022FA8246E8698B4611F01DFA524618
:10092800CDE900015B463946204616F08BF8224691
:1009380000230520822105F0A5FAA86B11F00CFA16
:100948008246E86B8B4611F007FA5246CDE9000162
:100958005B464146204616F075F800230520B42171
:10096800224605F08FFA31466A6C204616F06AF87E
:10097800A220B4212246002303B0BDE8F04F05F0C1
:1009880081BA00BF303A0020180C002093A0050857
:10099800B6A0050881A00508A5A0050808B500208F
:1009A80005F062F90A4B1B780B2B0BD8DFE803F034
:1009B8000A0A0A0A0A0A08060A0A0A0A054802E08E
:1009C800054800E00548BDE8084000F0B6BF00BF94
:1009D800A425002058130020800F0020D4170020E1
:1009E8002DE9F14F2D4C204603F09DFA00202C49AB
:1009F8002C4A03F04FF82C492C4A8146002003F07A
:100A080049F82B492B4A0746002003F043F82A49A6
:100A18002A4A0646002003F03DF82949294A054696
:100A2800002003F037F82849284A8046002003F0C0
:100A380031F82749274A8246002003F02BF8D221B3
:100A480083464A462346E62003F03CF928203A46E6
:100A58002346014603F036F946213246234628202C
:100A680003F030F964212A462346282003F02AF9A6
:100A7800822142462346282003F024F95246234681
:100A88002820A02103F01EF928205A46BE2123461B
:100A980001B0BDE8F04F03F015B900BF44150020C0
:100AA800BBA00508A5090008C4A005087512000820
:100AB800CFA0050851120008D9A005082D1200087A
:100AC800E4A0050809120008EFA00508E5110008D0
:100AD800F9A00508C1110008023810B50A2800F26B
:100AE8003C83DFE810F00B000F006400D2008A019D
:100AF8002001170231023A03A102F502BDE81040B5
:100B08000AF0E4BE00204FF6E0710BF03FF86320D6
:100B18004FF6E0710BF03AF8B3204FF4F0610BF0A8
:100B280035F8C7204FF6E0710BF030F84FF6FF703C
:100B380005F06EF8DC2100237D20D34A05F0A2F9E8
:100B48004EF29C7005F064F8052001210023CF4A7D
:100B580005F098F9052052210023CD4A05F092F9B5
:100B6800B62100230520CB4A05F08CF94FF4F0603C
:100B780005F04EF80121002340F21310C34A05F096
:100B880081F9002340F213105221C24A05F07AF984
:100B9800B621C14A40F21310002305F073F94EF252
:100BA8009C7005F035F80520A221BC4A68E00020B9
:100BB8004FF6E0710AF0EAFF31204FF6E0710AF0D3
:100BC800E5FF63204FF6E0710AF0E0FF95204FF64D
:100BD800E0710AF0DBFFC7204FF6E0710AF0D6FF9C
:100BE8004EF29C7005F014F8052001210023AC4A50
:100BF80005F048F9052020210023AA4A05F042F90A
:100C0800052052210023A84A05F03CF9052084213B
:100C18000023A64A05F036F9B62105209D4A00238F
:100C280005F030F94FF4F06004F0F2FF012140F2D2
:100C3800131000239A4A05F025F940F213102021D9
:100C48009B4A002305F01EF940F213105221914AE5
:100C5800002305F017F940F213108421954A002368
:100C680005F010F9B621944A40F21310002305F05C
:100C780009F94FF6FF7004F0CBFF904A7D20DC2184
:100C88000023BDE8104005F0FDB800204FF6E071E4
:100C98000AF07CFF27204FF6E0710AF077FF4F201B
:100CA8004FF6E0710AF072FF77204FF6E0710AF014
:100CB8006DFF9F204FF6E0710AF068FFC7204FF6DE
:100CC800E0710AF063FF4EF29C7004F0A1FF05206A
:100CD800012100236F4A05F0D5F8052016210023CD
:100CE800774A05F0CFF805203E210023754A05F024
:100CF800C9F8052066210023734A05F0C3F88E2140
:100D080000230520714A05F0BDF80520704AB62178
:100D1800002305F0B7F84FF6FF7004F079FF7D2047
:100D2800DC216C4AACE700204FF6E0710AF02EFF98
:100D380031204FF6E0710AF029FF63204FF6E07189
:100D48000AF024FF95204FF6E0710AF01FFFC72034
:100D58004FF6E0710AF01AFF4EF29C7004F058FF4B
:100D68000520012100235C4A05F08CF8052020218C
:100D780000235A4A05F086F8052052210023584AD4
:100D880005F080F8052084210023564A05F07AF8FA
:100D9800B62105203F4A002305F074F84FF4F060AF
:100DA80004F036FF012140F2131000234E4A05F0EB
:100DB80069F840F2131020214C4A002305F062F82C
:100DC80040F213105221334A002305F05BF840F239
:100DD80013108421464A002305F054F8B621454AE9
:100DE80040F21310002305F04DF84FF6FF7004F0A1
:100DF8000FFF7D20DC21404A42E700204FF6E071DA
:100E08000AF0C4FE31204FF6E0710AF0BFFE6320FD
:100E18004FF6E0710AF0BAFE95204FF6E0710AF03D
:100E2800B5FEC7204FF4FC610AF0B0FE4EF29C708C
:100E380004F0EEFE052001210023304A05F022F8D7
:100E48000520202100232E4A05F01CF805205221F8
:100E580000232C4A05F016F88421002305202A4A8D
:100E680005F010F84FF4F06004F0D2FEB62105202A
:100E7800264A002305F006F84FF6FF7004F0C8FE76
:100E88008720234ADC21FBE6CFA0050803A105083B
:100E9800FEA00508B1A6050802A1050830A10508AD
:100EA8001CA1050807A1050817A105080CA105083C
:100EB80011A1050816A105081BA10508D9A0050858
:100EC8001FA1050823A1050827A105082BA10508CE
:100ED8002FA1050833A105083FA1050843A105086E
:100EE80047A105084AA1050853A105084FA105080F
:100EF8004EA1050852A1050857A1050862A10508D9
:100F080028A1050820A1050872A10508C8A7050899
:100F1800F9A0050800204FF6E0710AF037FE6320BB
:100F28004FF4FC610AF032FE4FF6E071C7200AF078
:100F38002DFE4FF6FF7004F06BFE002004F06AFFF0
:100F4800A520D721854A9BE6042004F063FF0020F2
:100F58004FF6E0710AF01AFE31204FF6E0710AF000
:100F680015FE63204FF6E0710AF010FE95204FF64B
:100F7800E0710AF00BFEC7204FF6E0710AF006FE9A
:100F88004EF29C7004F044FE052001210023744AAF
:100F980004F078FF052020210023724A04F072FF34
:100FA800052052210023704A04F06CFF052084219B
:100FB80000236E4A04F066FF0520B6216C4A002320
:100FC80004F060FF4FF6E07004F022FE40F20B10D0
:100FD8000121684A002304F055FF40F22B1020211C
:100FE800654A002304F04EFF40F223105221634A61
:100FF800002304F047FF40F21B108421604A0023BD
:1010080004F040FFB6215F4A002340F2131004F0B9
:1010180039FF4FF6FF7004F0FBFD002004F0FAFEE4
:101028006E20D221584A90E0042004F0F3FE0020FC
:101038004FF6E0710AF0AAFD27204FF6E0710AF09A
:10104800A5FD4F204FF6E0710AF0A0FD77204FF67E
:10105800E0710AF09BFD9F204FF6E0710AF096FDC3
:10106800C7204FF6E0710AF091FD4EF29C7004F033
:10107800CFFD052001210023444A04F003FF052089
:1010880016210023424A04F0FDFE05203E210023DC
:10109800404A04F0F7FE052066213F4A002304F089
:1010A800F1FE05208E213D4A002304F0EBFEB62117
:1010B8003B4A0023052004F0E5FE4FF6FF7004F0DC
:1010C800A7FD002004F0A6FE6420D221354A3CE0AA
:1010D800042004F09FFE00204FF6E0710AF056FD50
:1010E80043204FF6E0710AF051FD85204FF6E0717C
:1010F8000AF04CFD4FF6E071C7200AF047FD4EF2AA
:101108009C7004F085FD05200121274A002304F086
:10111800B9FE05204521254A002304F0B3FE052029
:1011280087211F4A002304F0ADFEB621204A002380
:10113800052004F0A7FE4FF6FF7004F069FD0020BB
:1011480004F068FE1B4A7D20D221002304F09AFE99
:101158000420BDE8104004F05DBE10BD7AA5050866
:1011680066A1050872A1050871A1050874A1050802
:1011780078A105087DA105081CA1050884A105081A
:1011880088A105088DA1050893A1050899A105085E
:101198004FA1050854A105089EA10508A1A10508AD
:1011A80030A10508A4A10508ADA1050862A105089C
:1011B800B1A6050825A6050810B5064C064806235D
:1011C800237000F0BAFB2078FFF786FCBDE81040DA
:1011D8000DF07CBB282C00203017002010B5064CE1
:1011E80006480723237000F0A8FB2078FFF774FC5B
:1011F800BDE810400DF06ABB282C002030170020F5
:1012080010B5064C06480523237000F096FB20789D
:10121800FFF762FCBDE810400DF058BB282C0020F9
:101228003017002010B5064C06480423237000F040
:1012380084FB2078FFF750FCBDE810400DF046BB5A
:10124800282C00203017002010B5064C0648032330
:10125800237000F072FB2078FFF73EFCBDE81040D9
:101268000DF034BB282C00203017002010B5064C98
:1012780006480223237000F060FB2078FFF72CFC5F
:10128800BDE810400DF022BB282C002030170020AC
:1012980038B5094C05464FF6E071206801F03EFF6D
:1012A80020680DB1054900E0054901F0E5FEBDE8FB
:1012B800384003F071B800BF340C0020B1A1050814
:1012C800C4A105081A4B10B51C78012C14BF1024B2
:1012D8000024002C14BFD820C82006F01FFA154996
:1012E8000246154815F0AEFB002C14BFDC20CC20BC
:1012F80006F014FA0F490246104815F0A3FB002C1B
:1013080014BFE020D02006F009FA0A4902460C482A
:1013180015F098FB002C14BFE420D42006F0FEF949
:10132800044902460748BDE8104015F08BBB00BFD2
:10133800F40D0020B6A00508E025002004260020B2
:101348001A2C0020CC25002010B5E82006F0E6F97C
:101358000F4C024621460F4815F074FBEC2006F0AE
:10136800DDF9214602460C4815F06CFBF02006F02A
:10137800D5F921460246094815F064FBF42006F029
:10138800CDF9024606482146BDE8104015F05ABB83
:10139800B6A00508E0250020042600201A2C00200D
:1013A800CC2500200E4A012310B513700D4A0024E5
:1013B80014700D4A204613700AF0DEF9204604F036
:1013C80053FC0A4B03221A700AF01AFD0BF001FABB
:1013D800074B08481C70BDE8104000F0AEBA00BFCB
:1013E800282C00204F0D00204D0D0020A4250020A2
:1013F800043800201012002038B50D4B0D4D002484
:101408001C700D4B28681C700C4B4FF6E0711C705B
:1014180001F084FE28680A4901F02EFE02F0BCFFA4
:10142800204604F021FC0748BDE8384000F085BAA2
:10143800AC0D0020340C00204F0D0020A425002006
:1014480066A50508D417002007B50E4B0E481A7874
:10145800D2F1010238BF00221A700C4B05221A7013
:1014680000F06BFA022201238DE80C00B020602105
:10147800102232230DF0CEFB03B05DF804EB02F02E
:101488008BBF00BFAC0D0020C8100020A425002091
:101498002E4A002310B513702D4A13700DF00EF864
:1014A8000446002842D02B4C4FF6E071206801F02A
:1014B80035FE2068284901F0DFFD60684FF6E071CD
:1014C80001F02CFE6068254901F0D6FDA0684FF6B2
:1014D800E07101F023FEA068214901F0CDFD02F082
:1014E8005BFF4FF47A600AF021F820684FF6E0714C
:1014F80001F014FE20681B4901F0BEFD60684FF63C
:10150800E07101F00BFE6068164901F0B5FDA068B6
:101518004FF6E07101F002FEA068124901F0ACFD3F
:1015280002F03AFFBDE8104002F036BF0CF064FC50
:10153800204604F099FB0C4B0C4804221A7000F06A
:10154800FCF9BDE81040FFF7FDB800BFAC0D002066
:101558004F0D0020340C0020D7A10508EBA1050889
:10156800FBA1050865A50508A4250020FC1300209B
:101578002DE9F04F6A4DDFF8F4916A4E85B00024EA
:101588004FF6FF78284602F0CEFC41462246234615
:1015980065480094019401F085FD042703904146B5
:1015A8002246234648460097019401F07BFD4146B8
:1015B80030602246234648460097019401F072FDA8
:1015C800414670602246234648460097019401F040
:1015D80069FDA8F50048B0604146224623465348B5
:1015E8000097019401F05EFD4146F06022462346D3
:1015F8004F480097019401F055FD4146306122465D
:1016080023464C480097019401F04CFD2346706135
:101618004146224648480097019401F043FD474956
:10162800B061474A204602F035FA4649464A8046A4
:10163800204602F02FFA4549454A8246204602F0E4
:1016480029FA4449444A0746204602F023FA434906
:10165800434A8146204602F01DFA4249424A8346DF
:10166800204602F017FA21468446039ACDF808C0AE
:101678002B46204602F026FB052132682B46A02087
:1016880002F020FB692172682B46782002F01AFBD1
:101698007D21B2682B46782002F014FB2821F268DD
:1016A8002B46052002F00EFB4B2132692B46052004
:1016B80002F008FB052072696E212B4602F002FB3E
:1016C8009121B2692B46052002F0FCFAD2213A4654
:1016D8002B46052002F0F6FAD22142462B4660201E
:1016E80002F0F0FAD2214A462B46B02002F0EAFA7C
:1016F800D22152462B464FF4807002F0E3FAB4210F
:101708005A462B46052002F0DDFADDF808C06020B5
:10171800B42162462B4605B0BDE8F04F02F0D2BABC
:10172800A0140020340C00200BA2050815A20508FF
:101738001CA2050822A2050828A205082EA2050851
:101748009914000836A20508011400083EA20508ED
:101758005114000847A20508AD1300084FA2050858
:101768005113000858A20508CD12000862A5050803
:10177800544A00232DE9F0471370534ADFF860916B
:101788001370524B1D780127BD4214BF1025002548
:10179800B842044689F8007003D0022840F08C80D3
:1017A8000BE021464FF4747005F09FFF0AF04EFAE3
:1017B800204605F0A7F920467CE0002D14BFD8206C
:1017C800C82005F0ABFF0446002D14BFDC20CC2058
:1017D80005F0A4FF8046002D14BFE020D02005F0BE
:1017E8009DFF0646002D14BFE420D42005F096FF87
:1017F80005460AF02BFA364B36491A68A2421846B3
:1018080002DB0B68434513DD334B04601E60334B2A
:10181800C1F800801D6009F06FFF314B01221A707A
:10182800304A0520B4210023BDE8F04704F02ABB64
:10183800944218D1984516D1274B1B689E4212D165
:10184800264B1B689D420ED14FF47470394689F8B7
:10185800007005F04AFF244B00221A60234B4FF01A
:101868007E521A6028E01E4B02251D7029464FF44F
:10187800747005F03AFF164B1B6806EE906A1C1B45
:10188800F8EEE67A06EE904AB8EEE67A164B87EE60
:10189800277A284683ED007A0F4B1B6806EE903AAC
:1018A800B8EEE67A114BC7EE277AC3ED007A05F059
:1018B80029F90020FFF7ECFC0AF087F9BDE8F047AA
:1018C80002F06ABDAC0D00204F0D0020F40D002081
:1018D80018260020342C00200C2C0020C8250020BD
:1018E800B501002061A20508A0250020D825002008
:1018F80008B500F0A5FEFEF77FFC00F04FF800F0F9
:101908006FF8FEF789FEFEF7DDFCFFF769F801F0D6
:1019180095FAFFF72DFE01F067F8FEF713FD01F0C9
:1019280089F900F06DFB00F081FD00F013FE00F076
:101938005FFABDE8084000F02DBB10B5044628B991
:101948000F48104A104B532102F04EFF0F4B1868F6
:10195800844213D010B1C36900219847002004F0D5
:1019680083F9002004F06AF94FF6FF7004F050F98B
:10197800E369204601219847044B1C6010BD00BF55
:1019880075A205083420040891A20508500C00200F
:101998000048D2E7D41700200CF054BD10B5084C0D
:1019A800204602F0C0FA00200649074A02F072F801
:1019B800D22102462346FA20BDE8104002F082B93F
:1019C800380E0020AFA20508A1190008024B0348F1
:1019D80001221A70FFF7B1BFA4250020A01400202F
:1019E8002DE9F743374D384F384E0024284602F08A
:1019F8009AFA2246234647F6FF7135480094019427
:101A080001F050FB4FF6FF788146414622462346B7
:101A180038460094019401F045FB41463060224667
:101A2800234638460094019401F03CFB414670601F
:101A38002246234638460094019401F033FB23469E
:101A4800B0604146224638460094019401F02AFBD2
:101A58002049F060204A204602F01CF81F49204A1D
:101A68000746204602F016F8214680464A462B468D
:101A7800204602F027F93C2132682B46192002F053
:101A880021F95A2172682B46192002F01BF9782196
:101A9800B2682B46192002F015F99621F2682B46F8
:101AA800192002F00FF9D2213A462B46EC2002F019
:101AB80009F99C20D22142462B4603B0BDE8F043E9
:101AC80002F000B91012002062A50508540C00208D
:101AD800A1A20508AEA20508D5190008B7A20508F5
:101AE800A51C000870B5474E474C327847492DED84
:101AF800028B142592B005FB02420C320FA814F099
:101B0800A1FF33780D2B05FB03F504EB050332D851
:101B1800D3ED016A9B6807EE103A6359B8EEE68A7E
:101B280006EE903ADFED3A7AF8EEC78AB8EEE67A32
:101B380088EE278AC8EEA78AC7EE277A17EE900A9A
:101B480010F00AF902460B466846324914F07AFF4B
:101B580018EE100A10F000F902460B4605A82E49A7
:101B680014F070FF18EE900A10F0F6F802460B46D3
:101B78000AA82A4929E093ED017A9B6807EE903A72
:101B8800635906EE903AF8EEE78AF8EEE67AB8EE90
:101B9800C78A17EE900A10F0DFF802460B4668462F
:101BA8001F4914F04FFF18EE100A10F0D5F802463E
:101BB8000B4605A81B4914F045FF18EE900A10F0D3
:101BC800CBF80B46184902460AA8184C14F03AFFFD
:101BD8002068174901F050FA20680FA901F04CFA63
:101BE8006068694601F048FAA06805A901F044FA5E
:101BF800E0680AA901F040FA02F0CEFB12B0BDEC91
:101C0800028B70BD1626002000000020C0A2050827
:101C180000007A44CBA20508DCA20508EDA205085D
:101C2800FEA205080FA3050820A30508540C0020F0
:101C38006BA5050808B5114B114A1B780D2B8CBFF5
:101C480000210121117014225A430E4988588B181B
:101C58004FF47A720C495043086059684A430B495B
:101C68000A609A680A4B1A6009F046FD094B0A484F
:101C780001221A70BDE80840FFF75FBE1626002053
:101C8800F40D00200000002018260020342C00202D
:101C98000C2C0020A4250020A0140020CAE700BFB7
:101CA8004FF6FF7070474FF6FF7070471FB5002959
:101CB80047D04FF2DE7003F0D7FF002004F0AAF8F7
:101CC8000F2003F0A5FF1F4C1F4A412101230A20C2
:101CD80004F0D8F8042004F09DF823682820962101
:101CE800042B24DC0123194A04F0CCF803A90DF1D4
:101CF8000E02206804F04CFB0F2003F089FFBDF8AA
:101D08000C00BDF80E1014380F242822002380B2CE
:101D1800009403F0ADFFBDF80E10BDF80C00009460
:101D2800143989B22822012303F0A2FF09E0084AE6
:101D3800012304F0A7F81E20A521064A012304F078
:101D4800A1F81FBD640C002031A3050844A30508B1
:101D580060A3050876A3050837B51E4C2368042B35
:101D680005462BDC01A80DF1060104F00FFBBDF8B8
:101D78000630BDF80420184904200DF0A1F82368A6
:101D8800002B04DA1548164A164B592105E0042B96
:101D980005DD1248124A144B5A2102F025FD04EBC6
:101DA8008302BDF8041001339180BDF8061023604A
:101DB800052BD18008D1201D04F06AFB00230B48B5
:101DC8002360FFF7BAFD03E028460121FFF76EFF05
:101DD8003EBD00BF640C00208DA30508D2A30508F2
:101DE80046200408F4A305080BA40508E8150020FC
:101DF80037B50B4C204602F096F80A4B0A49009377
:101E080000250120094A0A4B019501F034FF2946B3
:101E180002462346284603B0BDE8304001F052BFD1
:101E2800B4120020B51C0008A91C0008AF1C00084B
:101E3800611D00084FF6FF7070474FF6FF7070473E
:101E480030B54FF6E07087B003F00EFF002003F0C6
:101E5800E1FF0F2003F0DCFE00212C4A2C4C01236B
:101E68000A2004F00FF8002003F0D2FE042003F04B
:101E7800D1FF0A201921274A012304F003F825215C
:101E8800254A01230A2003F0FDFF1F2003F0C0FEAE
:101E980001230A203721214A03F0F4FF2378002B7D
:101EA80031D001231E2096211D4A03F0EBFF6288E2
:101EB8001C4902A814F0C6FD01231E20A22102AA73
:101EC80003F0E0FFA288184902A814F0BBFDAE2178
:101ED80002AA01231E2003F0D5FF0F2003F098FE6D
:101EE8006088A188143880B20F2528220023009525
:101EF80003F0BEFEA18860880095143989B22822B3
:101F0800012303F0B5FE07B030BD00BF39A40508B2
:101F18007C0C00204BA405086BA405088BA40508BD
:101F2800AEA40508C0A40508CDA4050801B187E73B
:101F3800704713B50DF1060101A804F0DBF9144B45
:101F480001221A705988BDF80420891A0E311C29FB
:101F580019460AD89C88BDF80600201A0E301C289D
:101F680003D899680131996001E000238B60084B20
:101F78009968012905DD00229A601A70FFF708FDAB
:101F880005E05A80BDF806209A80FFF759FF1CBD6E
:101F98007C0C002037B50B4C204601F0C4FF0A4BDF
:101FA8000A49009300250120094A0A4B019501F0CE
:101FB80062FE294602462346284603B0BDE8304063
:101FC80001F080BEE8150020351F00083D1E0008FE
:101FD800431E00083B1F000808B5064B00221A7074
:101FE800054B186814F0C4F90448BDE80840FFF729
:101FF800A4BC00BFA4250020F0350020D417002081
:102008002DE9F04F514D524E85B00024284601F07D
:102018008AFF2246234647F6FF714E4800940194F2
:1020280001F040F84FF6FF770390394622462346E1
:1020380049480094019401F035F839463060224649
:10204800234646480094019401F02CF84FF001080B
:102058007060224623464FF6E0714148CDF8008073
:10206800019401F01FF82346B060394622463D48E6
:10207800CDF80080019401F015F83B49F0603B4A27
:10208800204601F007FD3A493A4A0746204601F042
:1020980001FD3949394A8046204601F0FBFC3849A0
:1020A800384A8146204601F0F5FC3749374A8246CE
:1020B800204601F0EFFC3649364A8346204601F0B7
:1020C800E9FC21468446039ACDF808C02B462046F1
:1020D80001F0F8FD3C2132682B46142001F0F2FD96
:1020E8003C2172682B46EC2001F0ECFDB421B2686B
:1020F8002B460F2001F0E6FDD2213A462B46E6207A
:1021080001F0E0FD642142462B46052001F0DAFD8E
:102118004A462B460520872101F0D4FD52462B461E
:102128000520D22101F0CEFDD2215A462B4650205F
:1021380001F0C8FDDDF808C09B20D22162462B467D
:1021480005B0BDE8F04F01F0BDBD00BFDC0E0020BA
:10215800880C0020DAA40508E4A405085EA2050896
:1021680060A5050862A50508AEA20508E11F0008DC
:1021780048A00508C921000858A00508C922000878
:10218800EDA40508D1230008F5A405088D2300084F
:10219800FDA405084923000808B50BF045FE4FF4D7
:1021A80041400CF0C5FB044B186807F033F8034BAB
:1021B80009221A7008BD00BF10260020A42500209F
:1021C80010B50C4CFFF7E8FF0B4A0023B42005219B
:1021D80003F058FEA0684FF6E07100F09FFFA0687A
:1021E800064900F049FF0BF01FFEBDE8104002F061
:1021F800D3B800BF880C002068A5050805A5050808
:10220800264B2DE9F7431888C00014F0A9F80546B5
:1022180028B90520B421224A2B4603F033FE214B6E
:10222800DFF878801D6000240BF0FEFD26461E4F67
:10223800DFF8889023E009F0B7F83B68D9F8000088
:1022480045F8083C7B6845F8043C184B1B68C018E7
:1022580006F0E0FF164B186809F068F9B8F80000B6
:1022680094FBF0F080B24FF4FC63009328210246FF
:10227800322303F059FC04F59E7401360334B8F890
:1022880000300835B342D6DA0A4B186806F0C2FFA8
:10229800094B09221A70BDE8FE8300BFFC390020F3
:1022A8001EA50508F0350020BC3700209C2500201D
:1022B800C825002010260020A4250020F83500207D
:1022C80010B5094CFFF79CFFA0684FF6E07100F0CD
:1022D80025FFA068054900F0CFFE0BF0A5FDBDE87D
:1022E800104002F059B800BF880C00202CA5050842
:1022F80010B5074C4FF6E071A06800F00FFFA0681A
:10230800044900F0B9FEBDE8104002F045B800BF2E
:10231800880C002046A5050810B5074C4FF6E0715B
:10232800A06800F0FBFEA068044900F0A5FEBDE827
:10233800104002F031B800BF880C00205CA50508E9
:1023480010B50C4C0B2323700B4B01221A70002084
:1023580002F058FF0948FFF7F0FA2078FEF7BCFBB7
:10236800074B032093ED000A0BF06DFDBDE810400C
:10237800D2E700BF282C0020500D00203017002085
:102388000C03002038B50C4D0C232B700B4B01248B
:102398001C70002002F036FF0948FFF7CEFA2878B3
:1023A800FEF79AFB074B204693ED000A0BF04BFD16
:1023B800BDE83840B0E700BF282C0020500D0020B1
:1023C800301700200C03002010B50C4C0923237093
:1023D8000B4B01221A70002002F014FF0948FFF786
:1023E800ACFA2078FEF778FB074B022093ED000A41
:1023F8000BF029FDBDE810408EE700BF282C002017
:10240800500D0020301700200C0300200CF0DCB821
:10241800034A044800231370034A1370FFF78DBA68
:1024280004380020D4170020A42500202DE9F74304
:10243800384D394EDFF8FC800024284601F073FD42
:102448002246234647F6FF7134480094019400F071
:1024580029FE4FF6FF778146394622462346304803
:102468000094019400F01EFE39463060224623464F
:1024780040460094019400F015FE394670602246EB
:10248800234640460094019400F00CFE2346B060B9
:102498003946224640460094019400F003FE214943
:1024A800F060214A204601F0F5FA2049204A074603
:1024B800204601F0EFFA214680464A462B46204640
:1024C80001F000FC3C2132682B46282001F0FAFB81
:1024D8005A2172682B46192001F0F4FB7821B26862
:1024E8002B46192001F0EEFB9621F2682B461920A5
:1024F80001F0E8FBD2213A462B46EC2001F0E2FB42
:102508000520D22142462B4603B0BDE8F04301F036
:10251800D9BB00BF24100020980C002076A5050820
:102528007EA50508AEA205081924000889A5050896
:102538001524000862A50508034A044800231370FF
:10254800034A1370FFF7F9B904380020D4170020A4
:10255800A42500202DE9F743324E334DDFF8DC8007
:102568000024304601F0DFFC2246234647F6FF717F
:102578002E480094019400F095FD4FF6FF778146B0
:102588003946224623462A480094019400F08AFDE1
:10259800394628602246234640460094019400F0BC
:1025A80081FD3946686022462346404600940194DE
:1025B80000F078FD2346A86039462246404600943C
:1025C800019400F06FFD1B49E8601B4A204601F0AA
:1025D80061FA214607464A463346204601F072FB17
:1025E8003C212A683346192001F06CFB5A216A689D
:1025F8003346192001F066FB7821AA683346192072
:1026080001F060FB9621EA683346192001F05AFB75
:10261800EC20D2213A46334603B0BDE8F04301F03E
:1026280051BB00BF78180020A80C002091A5050810
:102638009FA50508AEA205084125000862A5050862
:1026480010B50B4C204601F06EFC002001462246D6
:1026580000F088FD00200749074A01F01BFAD22143
:10266800024623464FF48270BDE8104001F02ABBB1
:1026780030170020ACA50508A926000870B5C924A4
:102688000AE0A8B200223146013502F04BFCF02DD9
:10269800F7D10134EF2C02D00025A6B2F1E770BDC6
:1026A80010B51A4C2378092B08D1194A0023137046
:1026B800184A1370FFF7E2FF174823E00A2B0ED1E0
:1026C800164B186813F054FE154A00231370114A6C
:1026D8001370144A1370FFF7D1FF134812E000205B
:1026E80002F090FD114A00231360114A13800D4B2C
:1026F80002221A700F4B186806F08CFD22780E4BD8
:102708000E481A70BDE81040FFF717B9A42500203D
:10271800500D00204F0D0020DC0E0020F035002069
:10272800510D002004380020241000209C0D0020AA
:10273800AA0D002010260020C22500206C110020C0
:10274800034B01224FF4FC601A7003F061BA00BF1A
:102758004F0D0020044B054800221A70044B0C2230
:102768001A70FFF7EAB800BF4F0D00207818002054
:10277800A425002007B50A4A0023137004228DE817
:102788000C00C6201022232356210CF043FA054BD7
:1027980005480A221A7003B05DF804EBFFF7CDB8BC
:1027A8004F0D0020A42500202410002007B50A4A58
:1027B8000023137004228DE80C0097201022232395
:1027C80056210CF027FA054B054809221A7003B068
:1027D8005DF804EBFFF7B1B84F0D0020A4250020E9
:1027E800DC0E002007B50B4B00221A7008220323C9
:1027F8008DE80C004920102223233D210CF00AFA11
:10280800054B064801221A7003B05DF804EBFFF788
:1028180094B800BF4F0D0020A4250020A01400206C
:1028280008B50A4B00201870094B1870094B08228C
:102838001A70094B187003F017FA084B0848012260
:102848001A70BDE80840FFF778B800BFAC0D00204B
:102858004F0D0020A4250020282C00200836002039
:10286800380E002070B51F4C1F4E20684FF6E075DB
:10287800294600F053FC20681C4900F0FDFB606805
:10288800294600F04BFC6068194900F0F5FBA06888
:10289800294600F043FCA068164900F0EDFB01F062
:1028A8007BFD4FF47A6008F041FE2068294600F06D
:1028B80035FC2068314600F0DFFB6068294600F0EF
:1028C8002DFC6068314600F0D7FBA068294600F06F
:1028D80025FCA068314600F0CFFBBDE8704001F050
:1028E8005BBD00BFB80C002065A50508D7A1050889
:1028F800EBA10508FBA105080C4B10B500241C70C2
:102908000B4B01221A70204608F036FF204603F0D0
:10291800ABF9084B0B221A7009F072FA09F059FF4B
:102928000548BDE81040FFF708B800BF4F0D00206C
:10293800282C0020A4250020441500200F4A00233D
:1029480010B513700E4A13700BF0B8FD044628B189
:10295800FFF788FFBDE8104001F01EBD03F084F9C1
:1029680009F074F9074B1C70074B07221A7009F01D
:1029780067F90648BDE81040FEF7DFBFAC0D002040
:102988004F0D0020282C0020A425002058130020DB
:10299800104A002310B513700F4A13700BF08EFD08
:1029A800044628B1FFF75EFFBDE8104001F0F4BC13
:1029B80003F05AF909F04AF906F084FC074B1C7039
:1029C800074B06221A7009F03BF90648BDE810408B
:1029D800FEF7B3BFAC0D00204F0D0020282C0020BF
:1029E800A4250020800F00202DE9F04F6D4DDFF861
:1029F80010928BB000244FF6FF78284601F093FA26
:102A080041462246234668480094019400F04AFB58
:102A18004FF6E07604270490314622462346634861
:102A28000097019400F03EFB31460590224623466C
:102A38005F480097019400F035FB41460690224616
:102A4800234648460097019400F02CFB594E414616
:102A580030602246234648460097019400F022FB46
:102A6800234670604146224648460097019400F08C
:102A780019FB5149B060514A204601F00BF8504902
:102A8800504A0746204601F005F84F494F4A80460C
:102A9800204600F0FFFF4E494E4A8146204600F08E
:102AA800F9FF4D494D4A8246204600F0F3FF4C4954
:102AB8004C4A8346204600F0EDFF4B494B4A84467A
:102AC8002046CDF80CC000F0E5FF49490790494A77
:102AD800204600F0DFFF48490890484A204600F0A9
:102AE800D9FF21460990049A2B46204601F0EAF8BE
:102AF8002146059A2B46C82001F0E4F80A21069AD7
:102B08002B46C82001F0DEF8552132682B46782084
:102B180001F0D8F8692172682B46782001F0D2F8C4
:102B28007D21B2682B46782001F0CCF805203A4682
:102B380028212B4601F0C6F8D22142462B46052013
:102B480001F0C0F8D2214A462B46562001F0BAF8C7
:102B5800D22152462B46A62001F0B4F8B4215A4699
:102B68002B46052001F0AEF8DDF80CC0B421624612
:102B78002B46562001F0A6F8B421079A2B46A6202A
:102B880001F0A0F8B421089A2B46F62001F09AF833
:102B9800099AF620D2212B460BB0BDE8F04F01F080
:102BA80091B800BFD4170020B1A50508BAA505083B
:102BB800C7A50508B80C0020D2A50508ED27000810
:102BC800DAA5050801290008E3A5050899290008E0
:102BD800ECA5050845290008F5A5050829280008D9
:102BE800FEA50508B527000807A605087D270008E3
:102BF80010A605085D27000818A60508492700083B
:102C080062A5050807B5032308228DE80C004920B2
:102C1800102223233D210BF0FDFF044B0448012221
:102C28001A7003B05DF804EBFEF787BEA4250020F8
:102C3800A01400202DE9F743314E324F324D0024C5
:102C4800304601F070F92246234647F6FF712F48B7
:102C58000094019400F026FA4FF6FF788146414629
:102C68002246234638460094019400F01BFA414658
:102C780028602246234638460094019400F012FA50
:102C8800414668602246234638460094019400F085
:102C980009FA2346A8604146224638460094019422
:102CA80000F000FA1A49E8601A4A204600F0F2FEDD
:102CB800214607464A463346204601F003F83C21A0
:102CC8002A683346192000F0FDFF5A216A68334606
:102CD800192000F0F7FF7821AA683346192000F080
:102CE800F1FF9621EA683346192000F0EBFFEC204B
:102CF800D2213A46334603B0BDE8F04300F0E2BFC4
:102D0800C810002062A50508C40C002020A60508EC
:102D1800AEA205080D2C00081C4B1A781C4B10B5E8
:102D28001A7009F073F81B4B1B4A00241C60022020
:102D38002346CA2103F0A6F8204608F01DFD174BCC
:102D48001C80174B1C70174B1B78023B052B1CD89B
:102D5800DFE803F003070B13170FBDE81040FEF779
:102D680085BABDE81040FEF76FBABDE81040FEF71F
:102D780059BABDE81040FEF731BABDE81040FEF779
:102D88003FBABDE81040FEF717BA10BDC2250020B3
:102D9800A42500209C0D002061A50508043600200C
:102DA80004380020282C002008B5084B186806F0C5
:102DB80031FA002002F058FF09F022F8044B0548C8
:102DC8000B221A70BDE80840FEF7B7BD1026002098
:102DD800A425002044150020114B10B500241C70B8
:102DE800104B186806F016FA204602F03DFF0E4B0D
:102DF8001B780B2B0ED8DFE803F006060D0D0D0D22
:102E08000A080D0D0D06094802E0094800E00948C6
:102E1800FEF793FD084B1C70BDE8104008F0F0BFAA
:102E2800282C002010260020A4250020D4170020DC
:102E380058130020800F0020043800202DE9F041AD
:102E4800144C204601F06FF800201349134A00F093
:102E580021FE1349134A0746002000F01BFE1249C1
:102E6800124A0646002000F015FED22105463A46D1
:102E78002346E62000F026FF4B21324623466420F5
:102E880000F020FF642069212A462346BDE8F0416E
:102E980000F018BF6C110020BBA00508E12D000848
:102EA80028A60508B12D000834A60508212D00081C
:102EB80008B508B143682BB90348044A044B9B2161
:102EC80001F092FC586908BD41A60508582004087D
:102ED80063A6050808B5FFF7EBFF8068123080B2DB
:102EE80008BD08B5FFF7E4FF4068063080B208BDAA
:102EF8002DE9F84F04468846FFF7DAFF6689E58929
:102F0800074606F1030905F10F0AB8F1000F1FD0B3
:102F18001F2002F07DFE2046FFF7DCFF8346204697
:102F2800FFF7DFFF294603465FFA8BF2F0B202F0A3
:102F3800AFFE042002F06EFF0B364FF6FF7003352C
:102F480002F066FEB0B2A9B23A68012302F09AFF15
:102F58003D69204641464A465346A847BDE8F88F92
:102F680013B504460DF1060101A803F0C3F9204684
:102F7800FFF79EFF6389BDF80410BDF80620C91A43
:102F8800E389D21A0339C3680F3A204698471CBD13
:102F9800F7B5044614200D4616461F4613F0E0F90F
:102FA800089BC7600361064B0649074A80E8700022
:102FB80000930190054B002000F05DFEFEBD00BFB0
:102FC800F92E0008EB2E0008DD2E0008692F0008F6
:102FD800704708B508B143682BB90448044A054B43
:102FE800AD2101F001FC586908BD00BF82A60508A3
:102FF8007020040863A60508F8B505460E46FFF7D5
:10300800E8FF836B04461BB128463146984700E029
:1030180018466F8994F83C30ED890EB9034310D0F7
:10302800208E02F0F5FD608E02F008FE94F835005F
:1030380002F0F0FE94F8343038462946224602F071
:1030480021FF002384F83C30F8BD08B5FFF7C1FF25
:1030580090F83500BDE8084002F0F1BE38B5FFF73A
:10306800B8FF044613F074FD054694F8350002F0E5
:10307800E1FE684380B238BD38B50D46FFF7A9FFB9
:1030880029462E22044613F093FD50B120462946C6
:103098002E2213F0DFFD002384F82E30012384F85C
:1030A8003C3038BD2DE9F743074640200E4615460B
:1030B800984613F055F9044628B91148114A124B9D
:1030C8004E2101F091FB114B114A12498DE818006D
:1030D8000020114B00F0CFFD39468146FFF7CCFFA9
:1030E8009DF82830268684F835300B9B6586A363C7
:1030F800002384F8348084F83C304846BDE8FE83D9
:1031080082A6050888200408A0A605080130000842
:103118005330000865300008D92F000810B50C4658
:10312800FFF757FF0123048680F83C3010BD00BF2D
:103138004FF4A0707047C82070477047074B1B7842
:10314800022B07B508D1064B1B78022B04D001A827
:103158000DF1060103F0CEF80EBD00BF04380020C3
:10316800282C002073B50A4B06460D4614460093DA
:1031780000200849084A094B019000F07CFD2946C7
:1031880002462346304602B0BDE8704000F09ABDC2
:1031980043310008393100083F3100084531000843
:1031A80013B502AB03E90600436843B1027C01246E
:1031B800082A9C7004D11B692146984700E01C46E8
:1031C80020461CBD30B500282BD0058B002425E0F7
:1031D800036A1A7C012A05D15B681A888A421BD1C6
:1031E800187F30BD052A06D15B681A888A4213D138
:1031F80093F82C0030BD032A06D15B681A888A42EE
:103208000AD193F8250030BD062A05D15B681A88D3
:103218008A4201D1D87A30BD01340430AC42D7D3C8
:10322800002030BD08B1817501207047F8B504460B
:103238000D46D0B1E175D0F898309847012D0DD1E1
:103248002746002606E0F86900F10802436906CA25
:1032580098470136238B04379E42F4D3D4F898302C
:103268002046294698470120F8BDF8BDF8B505461F
:10327800084617460E4613F06BFC013FB84234BFB0
:1032880004463C463CB128463146224613F0E2FC4F
:1032980000232B55F8BD2C70F8BDF7B50446002067
:1032A8000090019000296CD00E8B68E000F10803B3
:1032B80051F823301D7C042D04D15D682D8895427A
:1032C80047D0013000F1080351F823301D7C012D4F
:1032D80004D15D682D8895423BD0013000F1080388
:1032E80051F823301D7C052D04D15D682D88954249
:1032F8002FD0013000F1080351F823301D7C032D35
:1033080004D15D682D88954223D0013000F108036F
:1033180051F823301D7C022D04D15D682D8895421B
:1033280017D0013000F1080351F823301D7C072D18
:1033380004D15D682D8A95420BD0013000F1080355
:1033480051F823301D7C062D08D15D682D889542E3
:1033580003D103F10801204615E0013000F108030C
:1033680051F823502B7C082B09D16F683F8897426E
:1033780004D105F1080120461A4605E00130B042A3
:1033880094D320466946082213F09AFA2046FEBDD7
:10339800F8B505460F461646002830D04388032B5B
:1033A8002FD0202012F0DCFF044600282BD040F854
:1033B8000C5B39460C22FFF759FF1820E66112F022
:1033C800CFFF0646B8B102230374012363760F4B7F
:1033D800446063600E4BA360002323766B8805EB83
:1033E800830201339BB2012B50606B800CD16A6859
:1033F8005268137608E0204612F0BAFF04E0064649
:1034080002E0002600E006463046F8BDD49F0408D6
:10341800729C040837B5456802AB03E906003DB362
:10342800037C0124042B85F8314022D1688E02F0F8
:10343800EFFB95F8300002F0EDFC95F8343043B915
:10344800BDF80200BDF80610AA1C234602F01AFDBA
:103458000FE0012B03D1084840F2395104E0022B58
:1034680007D1054840F24151044A054B01F0BCF927
:103478002C4620463EBD00BFB3A60508486B04088D
:10348800B1A60508F8B504460F46164610B3838A58
:103498000A2B20D0202012F063FF0546E8B14460D3
:1034A800102200F108003946FFF7E0FE4FF6FF73DF
:1034B800A08A2B801F236B8000232B76831D01306D
:1034C80080B20128EE6144F82350A08207D1A36995
:1034D8001876F8BDF8BD0020F8BD0120F8BD012020
:1034E800F8BD2DE9F3471D464B1C984282460C4611
:1034F8001746BDF828600DDD95420BDC01320AF154
:1035080001035B1A521BC8B2D2B29BB2294600967D
:1035180002F0B6FBAAF1020A3046C4EB0A0A02F02E
:1035280077FB4FF000084FF001091FFA8AFA0BE009
:10353800601C08EB050180B289B252460023009650
:1035480002F096FB09F101097B1B08F10108994576
:103558001FFA88F8ECD3BDE8FC87F8B5C7B2144663
:1035680038461E460D4602F095FB621E92B238465A
:10357800294602F08FFB304602F04AFB022606E09D
:10358800A21B92B23846294602F084FB0136A642B5
:10359800F6D3F8BD73B504460E4600F11E00154675
:1035A800009200233C2280B21E3E02F061FBB1B2C1
:1035B80020463C220123009502F05AFB7CBD73B5DE
:1035C80004460E460138154600920023032280B2B5
:1035D800013E02F04DFBB1B22046032201230095C3
:1035E80002F046FB7CBDF7B5089D2E7BEF7A1C46A2
:1035F8003604AB7A06EB0726F618431A687B06EB07
:1036080000602D1800200190121B084621460095E5
:1036180001F026FFFEBD30B5456885B004AB03E96F
:1036280006007DB101242C736D68BDF80800BDF853
:103638000A109DF80C209DF80E300095FFF7D3FF77
:10364800204600E0284605B030BD2DE9F04385B09E
:1036580004AB03E906004468BDF80860BDF80C70C7
:10366800002C41D0012384F8263094F825300BB97A
:10367800A26800E06268FFB2BDF80A109DF80E303B
:10368800009230463A46FFF7AEFF04F10C080220DC
:1036980002F0C0FB404613F05BFA054600B1451E38
:1036A8000F3F0024153E1FFA87F90DE002F0BCFB1E
:1036B80002F0C0FB04FB106189B2484620220023B7
:1036C80002F0FAFB0134E4B2AC42EFD3002002F07E
:1036D8009FFAB8B2B1B24246012302F0EDFB0020D6
:1036E80002F098FB012000E0204605B0BDE8F08319
:1036F8002DE9F04385B004AB03E906004568BDF841
:103708000860BDF80C70002D3CD001236B762B7E31
:10371800BDF80A10012B0CBF6A68AA689DF80E3024
:103728000092FFB23A463046FFF75DFF0C350220A3
:1037380002F070FB284613F00BFA0E3F8146002476
:10374800163E1FFA87F80DE002F06EFB02F072FBDE
:1037580004FB106189B240462022002302F0ACFB32
:103768000134E4B24C45EFD9002002F051FAB8B266
:10377800B1B22A46012302F09FFB002002F04AFB67
:10378800012000E0284605B0BDE8F0832DE9F04FA0
:1037980085B00546DDF8409002914846904603936F
:1037A80013F0D6F9DDF838A0DDF83CB00646294616
:1037B80000242F4611E024B1B4420CBF5B465346A7
:1037C80000E0039B01F10805ADB200932846029A78
:1037D8004346FFF708FF01342946B442EBDD0020D9
:1037E80002F016FA022002F015FB7D1D08F105080B
:1037F800A8B21FFA88F14A46012305B0BDE8F04F88
:1038080002F040BB70B5406886B006AB03E906001D
:1038180000282ED0012380F82D308668164BF21A26
:10382800534243EB020390F82C205AB1002B134D5E
:10383800134B144A08BF1D46134B00F11C0418BF54
:1038480013460AE0002B0D4D0D4B0E4A18BF1D46BE
:103858000D4B00F10C0408BF1346BDF81200BDF86B
:103868001410BDF81620009601950294FFF78EFFFC
:10387800012006B070BD00BFB8740408F4700408D5
:103888009A760408D67204087C78040870B54468EF
:1038980086B006AB03E9060004B301236377A66884
:1038A800104B227FF11A4B4243EB01030AB10BB9CB
:1038B80004E01BB966680C4D0C4B01E00C4D0D4B38
:1038C800BDF81200BDF81410BDF8162000960C348F
:1038D80001950294FFF75AFF012000E0204606B048
:1038E80070BD00BF04800408407C0408227E0408E0
:1038F800DA810408B08304082DE9F04385B004ABED
:1039080003E906004468BDF80860BDF80A90BDF8F0
:103918000C50BDF80E80002C00F08C800123A3749D
:103928000220676802F076FA4FF6FF7002F086F917
:10393800002002F06DF9EDB25FFA88F8A6F11601E1
:1039480089B230462A4643460097FFF74CFE277A4D
:10395800002F2ED1A28A234600E00137974204D2D5
:103968009969097E04330029F7D002F05DFA02F064
:1039780061FAA9F116091FFA89F90E2101FB1091C4
:103988004FF6FF7208F101085FFA88F389B20092D6
:1039980048462A46FFF7A5FD022002F03BFA1F2001
:1039A80002F036F9A38A002B38D0103DE8B2303E39
:1039B8002CE0E3685C68A28A2346013A002700E00D
:1039C8000137974204D29969097E04330029F7D058
:1039D80002F02AFA02F02EFA0E2101FB10914FF69E
:1039E800FF7208F101085FFA88F389B2009248462D
:1039F8002A46FFF776FD022002F00CFA1F2002F09B
:103A080007F9A38A53B1103DE8B21A3E0637B1B29E
:103A180054F827200123083202F04EFA002002F061
:103A2800F9F94FF6FF7002F009F91F2002F0F0F8DB
:103A3800012000E0204605B0BDE8F0832DE9F04103
:103A480005463620884614461F4612F089FC06466D
:103A5800E0B120F8025B41462E22FFF707FCBDF8D3
:103A6800183086F8344073861820012386F83070A1
:103A780086F8313012F074FC044618B1042346600D
:103A8800037404E0304612F073FC00E0044620465C
:103A9800BDE8F081F8B5064624200F46154612F019
:103AA8005FFC0446D8B10F4B068083600E4B394645
:103AB8004360102200F10C00FFF7D8FB0126002319
:103AC800182025622377667712F04AFC054610B164
:103AD8004460067404E0204612F04AFC00E0054603
:103AE8002846F8BD048004085E7A0408F8B506463E
:103AF8002C200F46154612F033FC0446E8B120F896
:103B08000C6B39461922FFF7B1FB0D4BA562A36078
:103B18000C4B6360002384F825301820012384F8B7
:103B2800263012F01DFC054618B1032344600374C7
:103B380004E0204612F01CFC00E005462846F8BDCB
:103B480010990408AE95040810B50446142012F024
:103B580007FC20B100234380014B0480036110BDA2
:103B68009933000838B50546442012F0F9FB04469D
:103B7800C0B10E4B058243600D4B03600123837473
:103B88000023037283820B4B0364182012F0E8FBB6
:103B9800054618B107234460037404E0204612F078
:103BA800E7FB00E00546284638BD00BFA49104089D
:103BB8009A8D04088D3400082DE9F041054634201B
:103BC800884614461F4612F0CBFB064620B3144B1A
:103BD80005808360134B41464360102200F10C00BE
:103BE800FFF744FB214606F11C001022FFF73EFBBD
:103BF800002386F82C3018200123376386F82D30EF
:103C080012F0AEFB044618B105234660037404E0C5
:103C1800304612F0ADFB00E004462046BDE8F081D6
:103C2800B8740408126F04082DE9F0410446142002
:103C38000D461646984612F093FB0746B8B1069B08
:103C4800048003610023C37201234560068180F864
:103C58000A800373182012F083FB044618B1062368
:103C68004760037404E0384612F082FB00E0044623
:103C78002046BDE8F0812DE9F041044618200D46A4
:103C88001646984612F06CFB0746B8B101238370BC
:103C9800069B04800361079B45608660C0F80C8022
:103CA8004361182012F05CFB044618B108234760F2
:103CB800037404E0384612F05BFB00E0044620463B
:103CC800BDE8F0812DE9F34198461B8B1D2B054675
:103CD8000C4617464FF0000000F2B480B5F5A07FFF
:103CE8000090019000F2AE80F02900F2AB80127CC7
:103CF800ADF80610511EADF80250072900F28A806F
:103D0800DFE801F045595E04456A14767B684E4A3F
:103D18007A611A8893F834303A80013BDBB2012B80
:103D28007FD8ADF80240ADF806507AE005F11602EA
:103D3800ADF8002004F11602ADF8042002AE434AA3
:103D480016E903007A6107F1080282E8030003F12B
:103D58000802013348F82270A8F818307B681A8ADC
:103D6800187A3A8000286CD1FFF7FCFE384943687E
:103D780059603849DF600126163D196002461E72F7
:103D8800A8B2E1B24346FFF79DFF30465AE0012A48
:103D98000CBF314B314B78687B6130F80C3B3B8072
:103DA80012F0D6FE431CDB001A34ED18ADF80440BF
:103DB800ADF8005035E07B68294A1B687A6102E05B
:103DC800284A7B687A611B8814353B80ADF800501F
:103DD8001434ADF8044024E07B68234A7A611A88D9
:103DE8003A801A899B7AAD18ADF80050E418F0E7CC
:103DF8007E681E4B7B61338838463B8073689847E2
:103E0800013D4519ADF80050B36838469847013C64
:103E18000419DEE71648174A174B40F21A3100F02A
:103E2800E3FC02AA12E9030007F1080383E8030090
:103E3800B8F8183003F10802013348F82270A8F8DE
:103E480018300120BDE8FC811D3400080139000844
:103E58009089040886850408953800080D380008FC
:103E6800F9360008533600081F360008A931000843
:103E7800B3A60508586B0408B1A60508F8B5164698
:103E8800002834D01378002B2ED0028B002327E093
:103E9800046A257C042D21D165682F888F421DD1A5
:103EA80095F8313053B16F8E01F0D8FE04F1080255
:103EB80068866369204606CA98476F86A81C3146FB
:103EC8002E22FFF7D3F995F831307BB104F10802BF
:103ED8006369204606CA98470120F8BD01330430BB
:103EE8009342D5D30020F8BD1846F8BD0120F8BD8F
:103EF80070B5B8B1068B0446002310E0256A287C0B
:103F080004280AD16D682888884206D11046A91C61
:103F18002E22FFF7ABF9012070BD01330434B34200
:103F2800ECD3002070BD38B5044620B3134BC361F1
:103F3800134BC0F89830134BC0F89C30124B002537
:103F48007822C0F8A0308575C5750583294600F12B
:103F5800200012F0F7FCD4F89830204629469847FC
:103F68000A4A1388312B07D8094941F823400133FD
:103F78001380012038BD38BD284638BD35320008C9
:103F88002D320008CD310008A3320008D40C0020DF
:103F98001C1900202DE9F0410446002800F0B380E8
:103FA800078B02460025A8E0136A1E7C042E00F049
:103FB8008780012E23D1586803888B4240F09B806C
:103FC80005F1080712F0D4F954F827004FF000085B
:103FD800C0F8048012F0CCF9228B531E9D4208D001
:103FE8000732238354F8221044F8271044F822801B
:103FF80002E044F8278025833046BDE8F081052E8D
:104008005ED0032E5CD0022E13D15B68186803883B
:104018008B4270D14388013B9BB243800BB912F0AD
:10402800A7F905F1080654F82630586812F0A0F9E7
:104038004EE0072E21D15E68338A8B425BD1002780
:1040480006E0BB1D013756F8230012F091F9FFB2C4
:10405800B38ABB42F5D80027B78205F1080654F8A1
:104068002630586812F084F954F8260033E044F8F2
:10407800267025830120BDE8F081062E1ED15868E0
:1040880003888B4237D105F1080612F071F954F80C
:1040980026000027476012F06BF9228B531E9D42C1
:1040A80009D00833013A54F82310228344F8261023
:1040B80044F82370DEE744F826701AE0082E1AD177
:1040C800586803888B4216D112F052F905F1080698
:1040D80054F826000027476012F04AF9228B531E35
:1040E8009D42C4D0073254F8221044F8261044F8F0
:1040F80022702383BEE701350432BD42FFF454AF7A
:104108000020BDE8F081BDE8F08170B504460028C4
:104118002AD0068B751E083600EB86061EE056F878
:10412800043D1A7C042A13D0012A11D0052A0FD085
:10413800032A0DD0022A02D15B681B6809E0072A0E
:1041480002D15B68198A05E0062A01D0082A04D141
:104158005B6819882046FFF71DFF013D681CDED10A
:1041680000232383012070BD70BDF0B528B3002360
:10417800068B1A461EE0046A257C072D18D1646850
:10418800258A8D4214D1A78A002504EB83040DE00B
:1041980004EB050C0435DCF818C09CF818C0BCF119
:1041A800010F03F1010301D1D8B2F0BDBB42EFD337
:1041B80001320430B242DED30020F0BD70B508B33E
:1041C800048B00231BE0026A157C072D15D1526869
:1041D800158A8D4211D10023958A11461C4601206B
:1041E80007E013B99669307601E08E6934760133B9
:1041F8000431AB42F5D3012070BD01330430A34232
:10420800E1D3002070BD2DE9F04128B30023078BCE
:104218001A461EE0046A257C072D18D16468258A91
:104228008D4214D1B4F814C0002504EB83040CE0CB
:1042380066190435B66996F81880B8F1010F03D1EC
:1042480006F10800BDE8F08101336345F0D301327F
:104258000430BA42DED30020BDE8F0812DE9F047F2
:1042680000282FD00023B0F818C01D4627E0046AA4
:10427800267C072E21D16468268A8E421DD1B4F887
:104288001480002604EB830915E009EB0604A769EE
:104298003C7E012C0DD192F800A0BAF1000F08D095
:1042A80007F1080011461022FEF7E0FF2046BDE89E
:1042B800F087013304364345E7D3013504306545BB
:1042C800D5D30020BDE8F087F0B5B0B1068B002546
:1042D80010E0046A277C062F0AD1646827888F4279
:1042E80006D123819DF814306260A3720120F0BDCD
:1042F80001350430B542ECD30020F0BD10B50021E3
:104308000446FEF793FF20460121BDE81040FEF762
:104318008DBF38B598B1048B024600230CE0106AB3
:10432800058804328D4206D100F10802436906CAA5
:104338009847012038BD0133A342F0D3002038BD8F
:1043480010B50C460021FEF771FF20460121BDE89B
:104358001040FEF76BBF13B502AC04E90C00BDF8C2
:104368000230834206D8BDF80030834234BF0020B3
:10437800012000E00020BDF806308B4206D8BDF8C9
:1043880004308B4234BF0021012100E000210028C5
:1043980018BF0846C0B21CBD38B5114B114A198860
:1043A800002319E052F8045FA87D012812D10024E7
:1043B8000CE004F1080355F82300037C082B03D113
:1043C800436800211B6998470134A4B22B8BA34290
:1043D800EFD838BD01339BB28B42E3D138BD00BF63
:1043E800D40C002018190020704770B5094CA57826
:1043F8007DB9094B1E78012E0BD1636801336360C8
:104408006268064B9A4204D9284601F0C5FCA6709A
:10441800656070BDD40C00208401002040420F006C
:10442800054A9060134602E09968013999609168DD
:104438000029F9D1704700BFD40C0020F0B585B031
:1044480001F056FF002800F04981002502A80DF16F
:104458000A01ADF80850ADF80A5001F04BFF03A867
:104468000DF10E01ADF80C50ADF80E5001F08EFFB5
:10447800BDF80C10BDF808200091BDF80E10BDF86D
:104488000A3001912C46964D964908200AF018FDED
:10449800A878012803D101F07FFCAC7019E1924B98
:1044A8005B78012B40F01581AB78002B40F011812F
:1044B8006B6029888D4A09E152F8046FB07D0128A4
:1044C80040F002810025FAE005F10803BDF8080074
:1044D80056F82340BDF80A1004F108030CCBFFF787
:1044E8003AFF002800F0E980237C013B062B00F20C
:1044F8009F80DFE803F00429159D1F9D4C00666826
:10450800012304F10805337795E80600636920461E
:104518009847002333772046636995E8060086E0CC
:10452800636893F8252012F1FF3218BF012283F83F
:10453800252077E0636893F82C2012F1FF3218BF2A
:10454800012283F82C206DE06268137E1568002B29
:104558006ED16E882F462946184606E051F804EFBA
:10456800DEF804E001338EF81800B342F6D30123D5
:104578001376002607E057F8040F00F10802436994
:1045880006CA984701366B889E42F4D350E06568A6
:1045980020892E68A37B227B0096A0F1160189B2A0
:1045A800FFF721F81420FFF73BFF2B7AC3B9AF8A36
:1045B80029461A461E4609E0886990F818E00676EA
:1045C800BEF1010F08BF134604310132BA42F3D3DA
:1045D80001220BB9AB6924E0053355F8233020E0FC
:1045E8006368DB685A680023908A154619461F4697
:1045F80009E0AE6996F818E03776BEF1010F08BFFA
:104608000B46043501318142F3D3411E8B4203D15D
:10461800053052F8203003E004D2073352F8233033
:1046280001221A7604F1080206CA636920469847EF
:10463800237C013B072B4CD8DFE803F00410074B21
:104648000A0D123A63681B6A34E063689B6A2DE0BE
:1046580063681B6B2AE063681B6927E0636824E0D2
:1046680063681A7A7AB9988A1946013800E00132E3
:10467800824204D28C69247E0431002CF7D00632A1
:1046880053F8223011E0DB685A68908A11460138E5
:10469800002300E00133834204D28C69247E043174
:1046A800002CF7D0063352F82330DB69984710E026
:1046B8006368DB68204698470BE00135ADB2338B61
:1046C800AB423FF601AF04E001339BB28B427FF46B
:1046D800F3AE01F053FE0F20FFF7A2FE05B0F0BDC8
:1046E800D40C0020D9A60508840100201819002040
:1046F800034B9A6812B19A68013A9A60704700BFF2
:10470800D40C00202DE9F3470120DFF8D080DFF832
:10471800D09001460BF06EFF012400254FF48076FF
:1047280002274046694600968DF804708DF80540CA
:104738008DF806508DF807400BF0B4FB4046082171
:1047480022460BF02FFC244BDFF898801A6844F2BD
:10475800A243B2FBF3FA0AF1FF3A204621461FFAB8
:104768008AFA0BF077FFC8F804A048464146A8F833
:104778000050A8F80250A8F8085088F80A500CF021
:1047880005FB7023A8F80C300423A8F810300AF1B0
:10479800FF3A6323642203FB0AF3B3FBF2F39BB2F1
:1047A800C8F8143008F10C014846A8F80E40A8F8DB
:1047B8001870A8F81A50A8F81C60A8F81E500CF039
:1047C80003FC484621460CF076FB484621460CF08F
:1047D8007CFEBDE8FC8700BFD0010020000002403D
:1047E80000000140E40C002083B50E460746154939
:1047F80010201C4615460AF063FB102012490AF0E7
:104808005FFB102011490AF05BFB10200E490AF0EB
:1048180057FB002310200E4901930AF051FB334641
:1048280010200C493A460AF04BFB10200A492A4648
:104838000AF046FB1020094922460AF041FB019B79
:104848000133E7E713A7050818A7050838A70508DF
:1048580048A7050858A705086DA705087EA70508F5
:1048680008B5164B1A6A01321A621A6A012A1A46E0
:1048780003D0134840F21D210FE05862194602E0A8
:104888004B6A013B4B62506A0C4B0028F8D11A6AFC
:10489800012A06D00A484FF40A710A4A0A4BFFF760
:1048A800A3FF1A6A013A1A621B6A2BB10448054A27
:1048B800064B40F22A21F2E708BD00BFE40C0020B5
:1048C8008FA7050836A30408B9A70508CAA70508CD
:1048D80010B5084C0221002220460BF058FB44F684
:1048E800FF70FFF7BDFF204602210122BDE81040FE
:1048F8000BF04DBB000402400C4B0D491A6844F202
:10490800A2436428B2FBF3F3D4BF20EAE07064202A
:10491800013B9BB24B60013B58436422B0FBF2F071
:1049280080B2486103480C310CF0D1BAD0010020A4
:10493800E40C00200000014010B5134B93F8282028
:104948002AB11248124A134B4FF442710EE0012269
:1049580083F8282066234FF0C042013BDBB2108069
:1049680033B90A480A4A0C4B40F21231FFF73CFFB0
:104978001488A4B28442F0D1084B1980024B00225B
:1049880083F8282010BD00BFE40C00208FA705087D
:1049980040A30408DBA70508B1A6050800000260CB
:1049A80010B5FFF7AFFE6420FFF7A6FF212107200F
:1049B800FFF7C2FF3220FFF753FF01210020FFF766
:1049C800BBFF3220FFF74CFF23210720FFF7B4FF7E
:1049D8003220FFF745FF00211020FFF7ADFF41F21D
:1049E8008830FFF73DFF33210720FFF7A5FF32206E
:1049F800FFF736FF112046F63001FFF79DFF322002
:104A0800FFF72EFF4FF4C0610220FFF795FF322019
:104A1800FFF726FF122046F6EB41FFF78DFF322005
:104A2800FFF71EFF03204AF6A401FFF785FF322097
:104A3800FFF716FF00210C20FFF77EFF3220FFF75B
:104A48000FFF0D2040F60C01FFF776FF3220FFF72D
:104A580007FF0E204FF42C51FFF76EFF3220FFF7AF
:104A6800FFFEB0211E20FFF767FF3220FFF7F8FE98
:104A7800012042F63F31FFF75FFF3220FFF7F0FEDB
:104A880005200021FFF758FF3220FFF7E9FE00213B
:104A98000620FFF751FF3220FFF7E2FE16204EF600
:104AA8001C71FFF749FF3220FFF7DAFE172040F2AA
:104AB8000311FFF741FF3220FFF7D2FE00210B2040
:104AC800FFF73AFF3220FFF7CBFE00210F20FFF758
:104AD80033FF3220FFF7C4FE41200021FFF72CFFEF
:104AE8003220FFF7BDFE42200021FFF725FF3220CC
:104AF800FFF7B6FE00214820FFF71EFF40F23F14E3
:104B08003220FFF7ADFE21464920FFF715FF32207E
:104B1800FFF7A6FE00214A20FFF70EFF3220FFF71D
:104B28009FFE00214B20FFF707FF3220FFF798FE7A
:104B380044204FF46F41FFF7FFFE3220FFF790FE4D
:104B480000214520FFF7F8FE3220FFF789FE2146B5
:104B58004620FFF7F1FE3220FFF782FE302040F2B8
:104B68000771FFF7E9FE3220FFF77AFE31204FF494
:104B78000171FFF7E1FE3220FFF772FE32204FF499
:104B88000171FFF7D9FE40F202543220FFF768FEA8
:104B980021463320FFF7D0FE3220FFF761FE342094
:104BA80040F20751FFF7C8FE3220FFF759FE3520C3
:104BB8004FF40171FFF7C0FE3220FFF751FE362097
:104BC8004FF40171FFF7B8FE3220FFF749FE214686
:104BD8003720FFF7B1FEA4F500743220FFF740FE3E
:104BE80021463A20FFF7A8FE3220FFF739FE2F2092
:104BF80041F2BE21FFF7A0FE3220FFF731FE214629
:104C08003B20FFF799FE3220FFF72AFE00212320E0
:104C1800FFF792FE3220FFF723FE00212420FFF742
:104C28008BFE3220FFF71CFE25204FF40041FFF7D2
:104C380083FE3220FFF714FE00214F20FFF77CFE91
:104C48003220FFF70DFE4E200021FFF775FE3220BF
:104C5800BDE8104004E608B5124B93F829202AB1A4
:104C68001148124A124B40F222310FE0012283F818
:104C78002920222166234FF0C042013BDBB211807C
:104C880033B90948094A0B4B40F23B31FFF7ACFDF9
:104C9800108880B22228F0D1024B002283F8292004
:104CA80008BD00BFE40C00208FA705084DA3040829
:104CB800DBA70508B1A6050810B51E4B032826D8A2
:104CC800DFE800F0021A080E1C8841F2280246F6B6
:104CD80028000AE01C8841F2080246F6080004E0B1
:104CE8001C8841F2300246F6300049F241318C42CC
:104CF80014BF014611460BE0188846F6200249F217
:104D08004131884214BF11464FF4815100E000211F
:104D18001B8848F68912934205D049F22032934203
:104D280004D1032000E01120FFF706FEBDE8104083
:104D380091E700BF86010020014B18800A208FE50B
:104D4800000002604FF0C043188003F500331A8852
:104D58001A88188880B270474FF0C04322221A8000
:104D680003F5003382B01A8892B2ADF806201B888A
:104D78009BB2ADF80630BDF8060080B202B07047AD
:104D8800072040F27311D7E507200021D4E582B04F
:104D9800044BADF80600BDF8062092B25A8502B061
:104DA800704700BFE40C002082B0044BADF8060049
:104DB800BDF8062092B25A8002B0704786010020E2
:104DC800014B80B218807047000002604FF0C0436A
:104DD80080B218807047024B80B21880704700BFBD
:104DE800000002604FF0C04380B218807047024B49
:104DF80080B21880704700BF0000026082B0044B88
:104E08000190019ADA62DA6A002AFCD102B070478E
:104E1800E40C002070B54FF0C0452A242C800A4CC1
:104E2800060AC0B226802080100AD2B220802280D2
:104E38002B222A800A0A2280C9B21A0ADBB22180F0
:104E48002280238070BD00BF0000026010B50B46B1
:104E580014460246FFF7DEFF4FF0C0432C22A0B2F3
:104E68001A80BDE8104067E7114B1B8848F6891285
:104E7800934210B504460BD049F22032934212D126
:104E8800C1F1EF01202089B2FFF756FD212006E08D
:104E9800C1F1EF014E2089B2FFF74EFD4F202146A8
:104EA800BDE8104048E502460B46BDE81040B1E7B2
:104EB8008601002008B5FFF7D7FF0F4B1B78012BA1
:104EC8004FF0C0420D4B0FD12E2111801A881A883D
:104ED8001B8892B202F0FC0002F4784242EAC00059
:104EE800C3F3C423184308BD222111801A881A88E5
:104EF800188880B208BD00BFEC19002000000260CD
:104F080070B5074D0646012421463046FFF7D2FF0B
:104F18000134A4B2C82C25F8020FF5D170BD00BF2A
:104F28000638002010B5084B1B78012B144602D117
:104F3800BDE810408AE7FFF797FFFFF78CFE204691
:104F4800BDE81040F8E600BFEC19002070B5074D29
:104F5800064601242146013435F8022F3046A4B212
:104F6800FFF7E0FFC82CF5D170BD00BF0638002060
:104F780070B505460E46FFF7C3FF012421460134EC
:104F880028463246A4B2FFF7CDFFC82CF6D170BD33
:104F98002DE9F04104460D461646BDF81880032B4E
:104FA80039D8DFE803F00B351927381980B22946BC
:104FB80042460137FFF7B6FFBFB200E00027B7420D
:104FC800F3D1BDE8F081E01B80B2294642460137A3
:104FD800FFF7A8FFBFB200E00027B742F3D1BDE852
:104FE800F081E91B89B2204642460137FFF79AFF54
:104FF800BFB200E00027B742F3D1BDE8F0817919CC
:1050080089B2204642460137FFF78CFFBFB200E065
:105018000027B742F3D1BDE8F08170B5194B1A4AA1
:10502800598E92F9004064180025A4B28AB0AC42A7
:1050380008BF0124C62C28BFC62415700F264FF6BA
:10504800FF721E865C865A8519202B4600922146DF
:105058000A22FFF79DFF21463046FFF72BFF224625
:1050680003460A4902A811F0EDFC02AA06A808495D
:1050780011F0E8FC3220D22106AA2B4600F002FFEC
:105088000AB070BDE40C0020591A0020F0A70508EA
:10509800F8A705082DE9F341BDF820500C469046C5
:1050A8001F461A46002306460095FFF771FF611E4A
:1050B800414430463A46002389B20095FFF768FF1D
:1050C80030462146424601230095013EFFF760FF26
:1050D800BF19B8B2214642460123089502B0BDE87F
:1050E800F04155E72DE9F0410D46C5F1F008411EA4
:1050F8005E18C2EB0802C5F1EF039BB292B2B6B2DA
:105108009A422CBF904698469A4234BF1146194697
:10511800864234BF3746074640F23F13864238BFBF
:1051280006469E4228BF1E46174B1B8848F6891222
:10513800B8F1EF0F28BF4FF0EF089342044610D0A4
:1051480049F2203293421AD15020FFF7F5FB512043
:105158004146FFF7F1FB52203946FFF7EDFB53209C
:105168000AE041EA082189B24420FFF7E5FB45201F
:105178003946FFF7E1FB46203146FFF7DDFB2046C5
:105188002946BDE8F0416FE686010020002001466F
:10519800F0224FF4A073A5E770B580B202FB03F4C8
:1051A80089B292B29BB2FFF79DFF0020FFF784FD02
:1051B8000025064E04E0708D80B2FFF7BDFD013575
:1051C800A542F8DBBDE87040E0E700BFE40C002032
:1051D80070B54FF0C0452A242C80094C060A268059
:1051E8002080080A208021802B212980110A218013
:1051F80022801A0A228023802C232B8070BD00BFB6
:105208000000026070B5114B1B78012B044607D1D2
:10521800002040F23F110246EF23FFF7D9FF04E0D8
:10522800FFF7B4FF0020FFF747FDF02509E0013E36
:105238002046B6B2FFF780FD002EF8D1013DADB291
:1052480015B14FF4A076F2E770BD00BFEC1900204D
:105258002DE9F04F1C463E4B87B01B7803918346DF
:105268009DF8441010980591012B039B04909246D9
:105278001FFA8BF09AB208D1411E531E09195344E4
:1052880089B29BB2FFF7A4FF09E01FFA8AF511461D
:10529800A3B22A46FFF726FF0020FFF70DFD0027DF
:1052A800DDF80C803E4640F23F1CA14639E0BBF1D8
:1052B800000F2EDB65452CDC0398002829DBB8F1AC
:1052C800EF0F26DC220702D1002CC8BF0136214986
:1052D8002140002903DA013961F00F010131059AF3
:1052E8000AB1C1F10F01049830F8162003FA01F150
:1052F8000A4012B26AB118494A8D029392B2A8B212
:105308001FFA88F1CDF804C0FFF70CFEDDF804C0E1
:10531800029B013401354C45C9DB0136013708F1E0
:105328000108574503DA5D4600240123F3E7084BDB
:105338001B78012B08D1002040F23F110246EF23D1
:1053480007B0BDE8F04F43E707B0BDE8F04F1DE7F1
:10535800EC1900200F000080E40C00202DE9F74F25
:105368001F463B4BDDF830801B7816469DF83420ED
:10537800012B044601920D4680B28AB208D1411E23
:10538800531EC9199B1989B29BB2FFF721FF09E087
:105398001FFA86FE1146BBB27246FFF7A3FE002035
:1053A800FFF78AFC4FF0000BDA463DE0002C30DBBB
:1053B80009EB040340F23F1293422ADC002D28DB5C
:1053C8000BEB0503EF2B24DC19F00F0F04D1B9F117
:1053D800000FC8BF0AF1010A1E4B09EA0303002B9C
:1053E80003DA013B63F00F030133019A0AB1C3F1F9
:1053F8000F03012202FA03F338F81A2013401BB2F4
:1054080013B1154B588D01E0144A508880B2FFF74C
:1054180093FC09F1010901E04FF00009B945C5DB2A
:105428000AF1010A0BF1010BB345F5DB084B1B78B8
:10543800012B08D1002040F23F110246EF2303B0B0
:10544800BDE8F04FC4E603B0BDE8F04F9EE600BFEC
:10545800EC1900200F000080E40C002086010020D9
:105468002DE9F0411C4F069C3F789DF81C60012FE8
:1054780002FB03F580B28FB209D1411ECB1899B255
:105488007B1E9A1893B23A46FFF7A2FE07E092B243
:105498009BB23946FFF726FE0020FFF70DFC0027D8
:1054A80009E034F8020B1EB1030A43EA002080B277
:1054B800FFF742FC0137AF42F3DB074B1B78012BA8
:1054C80007D1002040F23F110246EF23BDE8F0412A
:1054D8007EE6BDE8F04159E6EC1900202DE9F043DD
:1054E8001F2093B0FFF78EFE4FF47840FFF78AFE37
:1054F8004FF6E0754FF4FC60FFF784FE2846FFF78F
:1055080081FE0020514CFFF77DFE00204FF6FF7909
:10551800014664220346A4F82A90CDF80090FFF7CC
:1055280037FD00200A2164220346CDF80090FFF7DA
:105538002FFD00200146642201234FF4784765853A
:105548000095FFF725FD7720EF21C82200234FF4AF
:10555800FC6667850097FFF71BFDBD2132220123FA
:1055680040F23F1066850096FFF712FDA020322218
:105578000023782167850097FFF70AFDA02078218E
:10558800322201234FF01F0866850096FFF700FDC1
:10559800A020782132220223A4F82A80CDF80080A6
:1055A800FFF7F6FCA02078213222032365850095B9
:1055B800FFF7EEFC264B2749A3F8028002AD3C22F8
:1055C800284611F07DF9EB20C321052230230095F0
:1055D8000025A4F82A900195FFF7C0FE32210A2081
:1055E80096220B4667850097FFF754FD32213C2031
:1055F80096220B4666850096FFF74CFD32210B4636
:1056080096226E20A4F82A80CDF80080FFF742FD8C
:10561800FFF7BAFBFFF7B4FB3220FFF76DF9284616
:10562800FFF76AF96420FFF767F90B4B03F11002E3
:105638008DE8240028465A681B682946FFF710FFA2
:105648001195119B01331193FBE700BFE40C002077
:105658008601002062A3040820C801082DE9F14F43
:10566800FFF750F84FF0C0456420FFF745F90127D0
:10567800FFF72EF94FF028096D48FFF7F1F82F8052
:105688000520A5F8009003F0CFF9CF232B80694BB4
:10569800002683221E801A8030221A80ED222A805A
:1056A8004FF064080322A3F800801A8012221A809F
:1056B80081221A80E8222A8085221A8079221F8076
:1056C8001A80CB222A8039221A804FF0340C022407
:1056D8002C21F72219801E80A3F800C01C802A8084
:1056E80020221A80EA222A80C0221E80C1211E8020
:1056F8002A8026221A80298011211980C521298013
:10570800352119803E211980C7212980BE211980A1
:10571800362129803A205521A3F800902880198045
:10572800B12129804FF0100BF2211E80A3F800B0A0
:105738002980082119802A80E0221F804FF01F0944
:105748002A801A22A3F800904FF0180A1A800F2115
:105758000A22A3F800A01A80198006211980452181
:105768001980872119803221198007211A804FF06A
:10577800E10E19801C80052419801C801E80A5F864
:1057880000E04FF0250E1E80A3F800E04FF0270E32
:10579800A3F800E01C80A3F800B04FF0090BA3F8B1
:1057A80000B04FF0780B1880A3F800B04FF04D0B05
:1057B800A3F800B01C800D24A3F800A01C80382496
:1057C8001C8018802A20A3F80090EF2428802B2022
:1057D8001E801E801E801C8028803F201E801E8008
:1057E8001F801880B720A5F800C028801980B6212E
:1057F80029801A8082221A801122A3F800E04046EC
:105808001E8029272A8003F00FF940462F8003F0D5
:105818000BF90948FFF724F82C232F8030462B80FA
:1058280040F23F113246234601B0BDE8F04FCFE4C5
:10583800400D03000000026040420F002DE9F041D6
:10584800022098B0012100240AF0D4FE0125022686
:105858008048169616A98DF85D408DF85E408DF843
:105868005F408DF85C500AF01DFB182029460AF0AD
:10587800C1FE284629460AF0D5FE21460C22764864
:105888000AF090FB0C22744829460AF08BFB04218D
:105898000C2271480AF086FB05210C226E480AF09A
:1058A80081FB07210C226C480AF07CFB08210C22A2
:1058B80069480AF077FB09210C2267480AF072FB55
:1058C8000A2165480C220AF06DFB0B2162480C2264
:1058D8000AF068FB0E210C225F480AF063FB0F21D7
:1058E8000C225D480AF05EFB07210C225B480AF097
:1058F80059FB08210C2259480AF054FB09210C22B3
:1059080056480AF04FFB0A210C2254480AF04AFB79
:105918000B210C2251480AF045FB0C210A464F483E
:105928000AF040FB0D210C224C480AF03BFB0E21EB
:105938000C224A480AF036FB0C2248480F210AF08C
:1059480031FB4CF6B3734448169316A98DF85C6086
:105958008DF85E408DF85F408DF85D500AF0A2FA30
:1059680016A94FF680733D4816938DF85C608DF844
:105978005E408DF85F408DF85D500AF093FA40F66E
:10598800B830FEF76DFFFEF7A3FF40F6B830FEF71C
:1059980067FF0F2311934FF4805310270DF13C0834
:1059A800099368464FF400231094129414941594A4
:1059B800009401940294039704940694079408941D
:1059C8000A9405940B940C93CDF834800F95139595
:1059D80009F0E1FF0523684611930F96109412947D
:1059E80014941594CDF83880139509F0D4FF2946FE
:1059F80020460AF050F840F6B830FEF731FF20464E
:105A0800FFF7A0F904461649164E3846224609F013
:105A180057FA41F289239C4248F68918124F01D05F
:105A280044450ED1FEF7BCFF00233B70A6F800806A
:105A380010200E4948F6891241F2892309F040FAEC
:105A480005E0FFF70BFE49F241333D70338018B093
:105A5800BDE8F08100040240000C02400010024042
:105A6800FDA7050886010020EC19002014A80508E8
:105A78004FF0C04336221A8003F50033012814BFC3
:105A8800682048201880704770B5244B01228CB0DC
:105A98001A7000240AE0A9B21F2230460135FFF728
:105AA80041FA642DF7D10134642C02D00025A6B246
:105AB800F1E73220014602460346FFF7ABF94FF003
:105AC800C0432E221A8003F5003300201A881C8850
:105AD8001D88A4B200F09CF8ADB2002322460093C2
:105AE8000F492B4603A810F0ADFF00230A20C82158
:105AF80003AA00F0C7F904F0FC0204F4784444EA6D
:105B0800C20242EAD522074903A810F09BFF0A20E7
:105B1800DC2103AA002300F0B5F9FEE7EC19002008
:105B280053A805086BA805082DE9F04F40F23F1966
:105B3800484534BF04464C46EF2B34BF98464FF0D7
:105B4800EF084A4538BF9146EF2934BF0D46EF2587
:105B5800C4EB090AC5EB080785B0BAF1000FB8BF56
:105B6800CAF1000A002FB8BF7F424FF6FF734C45B9
:105B78002CBF1A4601221FFA8AFA454538BF01236D
:105B8800BFB202930FFA8AF63BB29E42BDF838B014
:105B9800019202DDC6F34F0607E0022693FBF6F6F4
:105BA8007642B6B201E01E4603E00FFA8AF35B4282
:105BB8000393144A1378022B204629465A4602D1E9
:105BC800FDF7FDFC01E0FFF7ADF94C4501D1454576
:105BD80014D0039A33B2934205DD019AF31BA4183B
:105BE8009BB2A4B200E0334636B23AB29642DADA51
:105BF800029A5344AD189BB2ADB2D4E705B0BDE8E4
:105C0800F08F00BF282C002000487047F4190020AE
:105C180082B0064BADF80600BDF8062092B21A8095
:105C2800188880B202B0FFF7B2B800BFF0190020A0
:105C3800014B188880B27047F019002082B0064BDB
:105C4800ADF80600BDF8062092B21A80188880B216
:105C580002B0FFF7A9B800BFF2190020014B18885D
:105C680080B27047F2190020FFF7CCBAFFF73ABAB2
:105C780010B5BDF808400294BDE81040FFF788B998
:105C880010B5BDF808400294BDE81040FFF702BA0D
:105C9800FFF782BA2DE9F04F4FEA420800253D4C44
:105CA80085B082468B46C8F1030817462E461FFA70
:105CB80087F909EB0B0C228805EB0A031FFA8CFC09
:105CC8009BB26146184692B2CDF804C00293FFF722
:105CD80029F9C9EB0B0292B20392029B228803991D
:105CE800184692B2FFF71EF9DDF804C02288C5EB0A
:105CF8000A039BB26146184692B20293FFF712F963
:105D0800029B22880399184692B2FFF70BF905EB1C
:105D18000B0292B2039209EB0A03228803999BB201
:105D2800184692B20293FFF7FDF8029B2288C5EB52
:105D38000B0C1FFA8CFC1846614692B2CDF804C0D1
:105D4800C9EB0A09FFF7EEF8228803991FFA89F9C7
:105D580092B24846FFF7E6F82288DDF804C092B20E
:105D680048466146FFF7DEF8B8F1000F04DA08EBA1
:105D7800860808F1060805E0F31B08F10A0808EB95
:105D88008308013F01360135BE42ADB28FD905B057
:105D9800BDE8F08FF019002008B9FEF7F5BF01281B
:105DA80001D1FEF7EDBF7047704700200146F02291
:105DB8004FF4A073FFF796B9704708B505280CD8BB
:105DC800DFE800F0121403050709094808BD09486F
:105DD80008BD094808BD094808BD0948094A0A4BD1
:105DE80040F24111FEF700FD084808BD084808BD0B
:105DF80074010020640100205C010020540100208F
:105E080076A805089EA30408B1A605087C01002011
:105E18006C01002010B50446FFF7CFFF014B186056
:105E28001C7110BD8C010020014B1879704700BF10
:105E38008C01002008B5FFF7C0FF808808BD08B5B1
:105E4800FFF7BBFFC08808BDF7B51F460B4B0C4ECC
:105E58001D681446EA882B68203C5443A4B2AE1B44
:105E680003EB440418BF0126AB888DE8500017B136
:105E7800FFF7EEF901E0FFF771FAFEBD8C01002093
:105E88007C0100202DE9F0410F469846154604464E
:105E9800084E08E0204643463946FFF7D5FF3368E9
:105EA8009B88E418A4B215F8012B002AF2D1BDE8AA
:105EB800F08100BF8C01002010B504460846214639
:105EC800BDE81040DEE7094B70B5044618790E4668
:105ED8001546FFF7B4FFC6F1F001091A89B220464A
:105EE8002A460023BDE87040CCE700BF8C010020A3
:105EF800704700BF044B1A680AB9044A1A601A6846
:105F08001018186010467047180D0020A43C002097
:105F18004FF0FF30704708B50248034A034B37215A
:105F2800FEF762FC95A80508B4A30408B1A6050805
:105F38000120704710B504460A4802210AF0E0FD26
:105F48000028F9D0074821460AF0A3FD0548012199
:105F58000AF0D6FD0028F9D00248BDE810400AF042
:105F680095BD00BF0038004010B5194802210AF05D
:105F7800C7FD0028F9D0164800210AF08AFD144808
:105F880001210AF0BDFD0028F9D011480AF07EFD74
:105F98000402A4B2002301E001339BB2002BFBD022
:105FA8000B4802210AF0ACFD0028F9D0084800216E
:105FB8000AF06FFD064801210AF0A2FD0028F9D079
:105FC80003480AF063FD2043C0F3CB0010BD00BFB7
:105FD800003800402DE9F0478AB00AAF0A200121B5
:105FE8000AF008FB4FF4604347F8143D474EDFF8CA
:105FF80024A1012400254FF00208304639468DF8C7
:106008001A508DF818808DF819808DF81B4009F00A
:1060180049FF30460D21052209F0C4FF30460E2104
:10602800052209F0BFFF052230460F2109F0BAFF0B
:1060380021464FF480400AF001FB50460AF0DCFB91
:106048004FF48273ADF802304FF40073ADF80A30A4
:106058003823ADF80C30504607236946ADF81030A8
:10606800ADF80050ADF80450ADF80650ADF8085042
:10607800ADF80E500AF0F2FB504621460AF089FCB2
:10608800A9468DF81A5030464FF480553946059583
:106098008DF818408DF819808DF81B4009F002FF23
:1060A8003046294609F06FFF4025394618488DF8D3
:1060B80018908DF819808DF81A908DF81B40059569
:1060C80009F0F0FE21464FF480400AF0C3FA062199
:1060D80003200AF04DFD0C2307A88DF82130079501
:1060E8008DF820908DF8224009F0D0FB17238DF809
:1060F800243009A80F238DF825308DF826308DF827
:10610800274002F0AFFE0AB0BDE8F0870004024065
:10611800000C024000380040014B1878704700BF5F
:106128001C0D0020024B5A889B8802800B80704708
:106138001C0D0020014B00221A7070471C0D002016
:10614800F0B593B068460021482210F0FBFB6D467D
:10615800002464484FF4805109F017FF002301E040
:1061680001339BB2002BFBD09020FFF7E3FE002306
:1061780001E001339BB2002BFBD0FFF7F5FE4FF493
:1061880080510746574809F0FEFE002301E001331D
:106198009BB2002BFBD053484FF4805109F0F5FE19
:1061A800002301E001339BB2002BFBD0D020FFF786
:1061B800C1FE002301E001339BB2002BFBD0FFF7A7
:1061C800D3FE4FF480510646464809F0DCFE45F8F8
:1061D800047B01342E6244484021E4B209F0C1FE38
:1061E80010B9092CB5D101E0092C78D19DE80C0033
:1061F800D218029B03980699D218049BC018059BD5
:10620800C018079BCB180899032490FBF4F092FB65
:10621800F4F25B1893FBF4F3151AC11A9C1A002DBB
:10622800B8BF6D420029B8BF4942002CB8BF6442CC
:10623800502D03DD502909DD502C50DC8D4205DA44
:10624800AC424FF0020405DB111806E08C424FF017
:10625800020401DAD11800E0C1180A9B099A0C98C7
:106268000F9DD2180B9BD2180D9BC0180E9BC018FF
:10627800109BEB18119D91FBF4F1032492FBF4F2AF
:1062880090FBF4F05B1993FBF4F3161AC41A9D1AE9
:10629800002EB8BF7642002CB8BF6442002DB8BFAC
:1062A8006D42502E89B203DD502C09DD502D16DCCD
:1062B800A64205DAB5424FF0020405DB131806E0E2
:1062C800A5424FF0020401DAD31800E0C318074AC8
:1062D80093FBF4F39BB2938001235180137013B0A6
:1062E800F0BD00BF00040240000C02401C0D00205D
:1062F800FFF712BFF7B505460C4601A80DF10601D8
:10630800FFF710FF1B4BBDF80660BDF8040093E8CB
:106318000600724301FB002299685218164992FB45
:10632800F1F207EE102AF8EEC77A40F23F17FCEEBA
:10633800E77A17EE902A92B2B2F5207F28BF3A4644
:106348002A801D69DA685B696E4302FB0060C01829
:1063580090FBF1F107EE101AF8EEC77AFCEEE77A37
:1063680017EE903A9BB2B3F5F07F28BFEF23238056
:10637800FEBD00BF240D002040420F00FFF7DABE2B
:10638800014B187E704700BF240D0020FFF7CABEDE
:10639800042808B505D90748074A084B7D21FEF7A8
:1063A80023FA054B03EB8000038B0B80438B138090
:1063B80008BD00BFB6A80508BAA30408D4A80508F4
:1063C80008B5082001F082F942F69643C31A5842EC
:1063D80040EB030008BD10B50A2001F09FF90C4CF2
:1063E80020600E2001F09AF96060122001F096F901
:1063F800A060162001F092F9E0601A2001F08EF9F1
:1064080020611E2001F08AF901236061237610BD06
:10641800240D002010B5FFF7DDFD01F035FA044624
:1064280001F03EFA074903462246202008F048FDBD
:10643800FFF7C6FF28B101F041FA10B9BDE81040D6
:10644800C9E710BD10A9050810B5104C0A2021682D
:1064580001F04BF961680E2001F047F9A16812209C
:1064680001F043F9E168162001F03FF921691A208B
:1064780001F03BF961691E2001F037F9082042F666
:106488009641BDE8104001F013B900BF240D00206B
:106498002DE9F04F0346A7B0B0F800C01C898688E4
:1064A800DF885D89CDF810C0B249B0F802C0B3F8F2
:1064B8000C90B3F80E80CDF824C00FFA84FB30B2EC
:1064C80001220FFA87FE0BEB000C0A7629B20FFAAD
:1064D80089FACDF888C001EB0E0C0FFA88F2CDF8D6
:1064E80090C00AEB0B0CCDF830C002EB010CCDF8D4
:1064F80058C0B3F810C05B8ACDF800C00FFA8CFC06
:1065080006910CEB00010A9102930CEB0A011BB2F5
:10651800239103EB0E010E9199182591049900FA25
:1065280081F0584450446044DDF824C006990EFABE
:106538008CFEDDF810C01FFA80FB1CFB0CF08E44AB
:1065480016FB0600964414FB0400009A19FB090088
:106558009E4412FB02001FFA8EFA0BF0DBFBDDF8FB
:1065680024C0029ACDE912011CFB0CF017FB0700AE
:1065780015FB050018FB080012FB02000BF0CAFB14
:10658800DDF824C0029ACDE9140104991CFB01F33B
:1065980017FB063615FB0466009B18FB096612FB01
:1065A80003600BF0B7FBDDE91423CDE90001DDE959
:1065B80012010BF025FC04460D46DDE900010246F8
:1065C8000B460BF01DFC02460B46204629460BF0F5
:1065D80063FACDE9180158460BF0ACFBCDE9100180
:1065E800DDE91023DDE900010BF00AFCCDE9060125
:1065F80050460BF09FFB804689464246DDE9120172
:106608004B460BF0FDFBDDE91023CDE91C01DDE96C
:1066180014010BF0F5FB002206460F46564BDDE948
:1066280018010BF0EDFB424604460D464B46DDE9EA
:1066380006010BF0E5FB02460B460BF02FFA02466B
:106648000B46204629460BF029FA424604460D46D9
:106658004B46DDE91C010BF0D3FB02460B462046F6
:1066680029460BF019FADDE9102304460D46304699
:1066780039460BF0C5FB02460B46204629460BF06F
:106688000BFADDF828C0CDE902014FEA8C10DDF8DD
:1066980030C000EB0C20DDF810C0A0241CFB040067
:1066A8000BF038FBDDF838C0CDE90A014FEA8C1051
:1066B800DDF858C000EB0C20DDF824C01CFB0400FA
:1066C8000BF028FBCDE90C0150460BF023FBDDE96C
:1066D8001023CDE91601DDE90C010BF091FB4246D0
:1066E800CDE91E014B46DDE90A010BF089FB424664
:1066F800CDE920014B46DDE900010BF081FB324674
:106708003B460BF0C9F9CDE90E0158460BF002FBE8
:10671800DDE91C23CDE91A01DDE906010BF0BCF91E
:10672800DDF88CC0C024CDE9060104FB0CF0DDF8CF
:1067380088C0302505FB0C00DDF810C078261CFB4E
:1067480006000BF0E7FADDF894C0824604FB0CF073
:10675800DDF890C005FB0C00DDF824C01CFB06002A
:106768008B460BF0D7FADDE9102306460F460BF0EF
:1067780047FB03E0240D0020000014404246CDE909
:1067880004014B46504659460BF03AFBDDE9142309
:1067980080468946DDE90A010BF032FBDDE900237A
:1067A80004460D46DDE90C010BF02AFB02460B46B8
:1067B800204629460BF070F90022A14B0BF020FB74
:1067C800DDE9202304460D46DDE91E010BF064F9DE
:1067D80002460B46DDE916010BF012FB02460B469A
:1067E800204629460BF05AF9002204460D46954BDF
:1067F800DDE90E010BF004FB02460B462046294654
:106808000BF04CF9DDE902230BF024FC88A3D3E953
:1068180000230BF0F5FA0BF08DFD8B490860DDE9DC
:106828001223DDE90C010BF0EBFADDE90023044645
:106838000D46DDE90A010BF0E3FA02460B46204655
:1068480029460BF029F900227D4B0BF0D9FADDE936
:106858001E2304460D46DDE920010BF01DF9024612
:106868000B46DDE91A010BF0CBFA02460B4620462F
:1068780029460BF013F9002204460D46714BDDE959
:1068880006010BF0BDFA02460B46204629460BF0DE
:1068980005F9DDE902230BF0DDFB65A3D3E900234D
:1068A8000BF0AEFA0BF046FD674A5060DDE90E23A7
:1068B800DDE90A010BF0A4FADDE9062304460D46DA
:1068C800DDE90C010BF09CFA02460B4620462946EE
:1068D8000BF0E4F8002204460D465A4BDDE9180196
:1068E8000BF08EFA02460B46204629460BF0D6F8E6
:1068F800DDE902230BF0AEFB4DA3D3E900230BF037
:106908007FFA0BF017FD504B59469860DDE91423C8
:1069180050460BF075FADDE9002304460D46304673
:1069280039460BF06DFA02460B46204629460BF015
:10693800B3F80022424B0BF063FA424604460D4678
:106948004B46DDE904010BF0A7F802460B46DDE9EA
:1069580016010BF055FA02460B46204629460BF065
:106968009DF835A3D3E9002304460D46DDE90E0161
:106978000BF046FA02460B46204629460BF08EF8E5
:10698800DDE902230BF066FB29A3D3E900230BF012
:1069980037FA0BF0CFFCDFF8B0C0DDE91223CCF8F2
:1069A8000C00394630460BF02BFADDE9002304468B
:1069B8000D46504659460BF023FA02460B46204630
:1069C80029460BF069F800221D4B0BF019FADDE996
:1069D800042304460D46404649460BF05DF802463E
:1069E8000B46DDE91A010BF00BFA02460B4620466E
:1069F80029460BF053F810A3D3E9002304460D46AB
:106A0800DDE906010BF0FCF902460B462046294653
:106A18000BF044F8DDE902230BF01CFB04A3D3E9D7
:106A280000230BF0EDF90BF085FC074908610DE038
:106A38000000000080842E410000000000C0824059
:106A48000000144000008940240D0020DDE90E23D9
:106A5800504659460BF0D4F9DDE9062304460D46A5
:106A6800304639460BF0CCF902460B4620462946FB
:106A78000BF014F811A3D3E9002304460D46DDE911
:106A880018010BF0BDF902460B46204629460BF0CB
:106A980005F8DDE902230BF0DDFA0AA3D3E90023A8
:106AA8000BF0AEF90BF046FC034A506127B0BDE885
:106AB800F04FC9E4AFF30080240D0020000000006F
:106AC80000C082400000000080842E41AFF30080A7
:106AD800064A074B1A60074A074B1A60074B42F2EF
:106AE80010721A60064B64221A60704740420F0009
:106AF8001826002080C3C901342C00200C2C00204B
:106B0800C8250020012810B502D002283AD123E078
:106B18001D4B1E4C1B78012B1D4B0ED11968C8202C
:106B280000F0E3FD2168CC2000F0DFFD194BD020F8
:106B3800196800F0DAFDD4201EE01968D82000F0AA
:106B4800D4FD2168DC2000F0D0FD124BE02019684C
:106B580000F0CBFDE4200FE00D4BE820196800F0B1
:106B6800C4FD0A4BEC20196800F0BFFD094BF0206A
:106B7800196800F0BAFDF420074B1968BDE8104009
:106B880000F0B3BD10BD00BFF40D0020342C002070
:106B9800182600200C2C0020C825002010B5224BF8
:106BA8001B78012B02D0022B3DD128E01F4B204C33
:106BB8001B78012B0FD1C82000F0B0FD2060CC203D
:106BC80000F0ACFD1B4B1860D02000F0A7FD1A4B5D
:106BD8001860D4200EE0D82000F0A0FD2060DC2052
:106BE80000F09CFD134B1860E02000F097FD124B5D
:106BF8001860E42000F092FD104B186010BDE820EA
:106C080000F08CFD0A4B1860EC2000F087FD094B62
:106C18001860F02000F082FD074B1860F42000F0A7
:106C28007DFD064B186010BDB5010020F40D002055
:106C380018260020342C00200C2C0020C825002009
:106C480008B504F0CBFD10B1BDE80840A6E7BDE8E3
:106C580008403DE7064B07495960C02100221972D8
:106C68001E211A70D9601A745A611A76DA6170474F
:106C7800201A002040787D0110B50321FF22C02092
:106C880001F0D8FB1F4C102180222060C02001F0A9
:106C9800D1FB112180222060C02001F0CBFB122102
:106CA80080222060C02001F0C5FB132180222060D3
:106CB800C02001F0BFFB142180222060C02001F019
:106CC800B9FB152180222060C02001F0B3FB80228F
:106CD80020601621C02001F0ADFB2060C0201721E4
:106CE800802201F0A7FB80222060B721C02001F09C
:106CF800A1FB054B00221A745A611A76DA61012247
:106D08001A7010BDF0250020201A002038B5C020C8
:106D18000321FF2201F08EFB0B4D00242B19615D2E
:106D28005A78C020023401F085FBC82CF6D1B12175
:106D3800AC22C02001F07EFBC0200321002201F01C
:106D480079FB002038BD00BFE6A304082DE9F3470E
:106D580006460F4692461D461AB90C1FE401914695
:106D680035E005EE902A06EE903AB8EE657AF8EE30
:106D7800667AFC01C7EE277AA4F500749FED5C7A69
:106D880067EE877A17EE900A0AF0E6FF41EC100BDF
:106D98000DF0F6F859EC108B494640460BF0F2FA24
:106DA80024184FEACA100AF0B5FFCDE900012846B9
:106DB8000AF0B0FF4B4642460BF022F802460B465B
:106DC800DDE900010AF068FE0BF0DCFA8146002ECE
:106DD80014BF4FF022084FF01A08C5F307224146A6
:106DE800C02001F027FB08F10101EAB2C02001F040
:106DF80021FBC4F3014208F10201C02001F01AFB93
:106E0800C4F3072208F10301C02001F013FBE2B22A
:106E180008F10401C02001F00DFBC9F3034305F498
:106E2800702243EA123208F10501C02001F002FB8A
:106E380008F10601C9F30722C02001F0FBFA08F1A6
:106E480007015FFA89F2C02001F0F4FAC020B121ED
:106E5800A02201F0EFFA07EE107A264CF8EEC77A76
:106E68000EBBD4ED015A06EE90AAB8EE657A05EE8F
:106E7800905AB8EE666AF8EE656A0123C6EE266A8D
:106E8800237477EEA67A67EE277A17EE900A0AF04F
:106E980063FF41EC100B0DF073F851EC100B0BF085
:106EA80071FA606120E005EE90AAD4ED016AB8EEAF
:106EB800656A05EE905AB8EE667AF8EE656A0123BF
:106EC800C6EE266A237677EEA67A67EE277A17EE5D
:106ED800900A0AF041FF41EC100B0DF051F851EC0B
:106EE800100B0BF04FFAE0610020BDE8FC8700BFF3
:106EF80000000043201A00200022012326E7012871
:106F080038B50D4604D002280CBF3C242C2400E0E0
:106F180034242146C02001F007FB05F0070200F0E9
:106F28000F0040EA02122146C020BDE8384001F0B7
:106F380081BA2DE9F3470A9C1D4607468A4616463C
:106F4800524B01E06D0864089C42FBD82DB906F14C
:106F58000076043EF601A94634E006EE905AB8EEF3
:106F6800667A06EE904AF8EE667AF601C7EE277A58
:106F7800A6F500769FED467A67EE877A17EE900AB7
:106F88000AF0EAFE41EC100B0CF0FAFF59EC108BFA
:106F9800494640460BF0F6F93618E8010AF0BAFE01
:106FA800CDE9000120460AF0B5FE4B4642460AF0FC
:106FB80027FF02460B46DDE900010AF06DFD0BF0E4
:106FC800E1F98146022F9BBF324BDB194FF00008D5
:106FD80093F8C880C4F307224146C02001F02AFA7A
:106FE80008F10101E2B2C9B2C02001F023FA08F1A8
:106FF8000201C9B2C6F30142C02001F01BFA08F130
:107008000301C9B2C6F30722C02001F013FA08F140
:107018000401C9B2F2B2C02001F00CFA04F47024E1
:10702800C9F3034308F1050143EA1432C9B2C02089
:1070380001F000FA08F10601C9B2C9F30722C0201D
:1070480008F1070801F0F6F95FFA89F25FFA88F1AA
:10705800C02001F0EFF9BAF1010F0CBF2F220F2267
:107068000DB942F04002012F06D002D3022F0AD1F7
:1070780005E0C020102104E0C020112101E0C0205B
:10708800122101F0D7F90020BDE8FC87FFFF0F00AF
:1070980000000043E6A3040807B50123009300237A
:1070A800FFF747FF0EBD00280CBFFF22002208B5DE
:1070B800C020032101F0BEF9002008BD08B5C0209A
:1070C800B121AC2201F0B6F9002008BD08B50420B2
:1070D800012109F08FFA4FF480700121BDE80840C2
:1070E80009F0B8BA07B50223009303238DF80430DA
:1070F8000348002369468DF8073008F0D3FE0EBD1B
:107108000008024030B5124D8BB0002406A8069442
:1071180007940894099408F093F800948DF80440B3
:107128008DF8054002940394049428460124694686
:107138008DF8144008F055F828460B2122460623FE
:1071480008F0CAF82846214608F094F80BB030BD7C
:107158000020014010B5002104460122302001F032
:1071680069F9C0B9012001F05FFC002CB8BF4034B8
:10717800E4B210212246302001F05CF9012001F030
:1071880053FC30201121224601F054F90120BDE8BA
:10719800104001F049BC10BD10B500210446012281
:1071A800302001F047F9C0B9012001F03DFC002C66
:1071B800B8BF4034E4B212212246302001F03AF937
:1071C800012001F031FC30201321224601F032F970
:1071D8000120BDE8104001F027BC10BD38B50122E0
:1071E80005460C463020002101F024F9F0B90120B1
:1071F80001F01AFC25EAE5725F2AA8BF5F223B214D
:10720800D2B2302001F016F9012001F00DFC24EA79
:10721800E4725F2AA8BF5F22D2B230203C2101F07D
:1072280009F90120BDE8384001F0FEBB38BD30281F
:1072380010B504460ADC10F17F0F02DB002802DBE0
:1072480005E06FF07E0404F5807400E0302400212E
:1072580030200A4601F0EEF8A8B90120E4B201F0A6
:10726800E3FB41212246302001F0E4F8012001F03F
:10727800DBFB30204221224601F0DCF80120BDE88A
:10728800104001F0D1BB10BD282810B5044609DC18
:1072980010F1180F02DB002802DB04E06FF017047E
:1072A8007F3400E02824002130200A4601F0C2F88B
:1072B800A8B90120E4B201F0B7FB532122463020DF
:1072C80001F0B8F8012001F0AFFB3020542122462C
:1072D80001F0B0F80120BDE8104001F0A5BB10BDD9
:1072E80008B530200021012201F0A4F860B901207E
:1072F80001F09AFB30203321402201F09BF8012055
:10730800BDE8084001F090BB08BD10B53020002151
:10731800012201F08FF8044660B9012001F084FBD6
:1073280030203321224601F085F80120BDE81040C5
:1073380001F07ABB10BD10B530200021012201F008
:1073480079F80446A0B9012001F06EFB34212246E9
:10735800302001F06FF8012001F066FB3020372162
:10736800224601F067F80120BDE8104001F05CBB3F
:1073780010BD4020EEE640200EE708B500210122AE
:10738800302001F057F8012001F04EFB3020342165
:10739800024601F04FF8012001F046FB302037216A
:1073A800024601F047F80120BDE8084001F03CBB67
:1073B80008B500210122302001F03CF8012001F03D
:1073C80033FB302034210C2201F034F80120BDE8D1
:1073D800084001F029BB00002DE9F04F984B994A6D
:1073E8001968994B002914BF91469946974B2DED82
:1073F800048BC3F80090964B0025002287B01A80B2
:10740800AA46AB46A8465AE0A2004046CDF804C0BA
:1074180002920AF0A1FC0746584601F100460AF01C
:107428009BFC02460B46384631460AF035FB39F9D3
:10743800243007EE103AF8EEC77A064617EE900A9F
:107448000F460AF089FC02460B46304639460AF0D8
:1074580025FB0AF0B7FF074650460AF07DFC0446B4
:10746800284601F100460AF077FCCDE90401DDE980
:107478000423204631460AF00FFB029A09EB020367
:107488000446B3F9023007EE103AF8EEC77A0D4613
:1074980017EE900A0AF060FC02460B462046294681
:1074A8000AF0FCFA0AF08EFFDDF804C0684A0CF115
:1074B800010CC3465546A2F800C08246B846644B44
:1074C800B3F800C00FFA8CF4B32C9DDD58460AF0CF
:1074D80043FCCDE9020140460AF03EFC0022064684
:1074E8000F465C4BDDE902010AF08AFC02460B46B6
:1074F800304639460AF0D2FA0022574B0AF0AAFD64
:107508000AF060FF4CA3D3E9002309EE900ADDE9F5
:1075180002010AF075FC00224F4B0AF09BFD0AF0AD
:1075280051FF09EE100A28460AF016FC0446504698
:107538000D460AF011FC002206460F462046294651
:10754800444B0AF05DFC02460B46304639460AF0C9
:10755800A5FA0022404B0AF07DFD0AF033FF36A35E
:10756800D3E9002308EE900A294620460AF048FC91
:107578000022394B0AF06EFD0AF024FF08EE100ACB
:1075880069EE287A58EE297A17EE900A0AF0E4FB99
:1075980068EE097A48EEA97A044617EE900A0D4675
:1075A8000AF0DAFB45EC104B41EC110B0CF0ECFD4A
:1075B80051EC100B0AF006FF28EE088A08EEA88A9C
:1075C80007EE100A254B264CF1EE477AC3ED007AF8
:1075D80018EE100A0AF0C0FB41EC100B0CF0E2FEAA
:1075E80029EE099A51EC100B09EEA99A0AF0EAFE65
:1075F800206019EE100A0AF0AFFB41EC100B0CF0FA
:10760800D1FE51EC100B0AF0DDFED4ED007A07EE46
:10761800100A87EE877A134B1860134BFDEEE77A52
:1076280083ED007A114BC3ED007A07B0BDEC048BF3
:10763800BDE8F08FAFF30080912B50E67AB6EB3FB0
:10764800481A0020CA2200202A1D0020441A0020BF
:10765800501A00200000E03F00005940382C00205C
:10766800502C0020442C0020402C00204C1A0020D4
:1076780010B5084C204608F062F8074B1860FFF771
:10768800ABFE064B0649012220461A80BDE8104091
:1076980008F0D6B810600240481A0020400D0020BB
:1076A80020800010014B1868704700BF4C1A00205A
:1076B80038B505460C460135C1F3072101F0C2F97A
:1076C800A8B2E1B201F0BEF900B238BD38B504463F
:1076D80000F0F2FF01340546A0B200F0EDFFEDB274
:1076E800C0B240EA052000B238BD37B50B0E8DF8A0
:1076F80004300B0C8DF805300B0A8DF806308DF828
:107708000710002400E0284601AB451CE15C013469
:1077180001F098F9042CADB2F5D13EBD37B500247F
:1077280000E02846451C00F0C7FF01ABADB2E054AD
:107738000134042CF5D19DF805009DF804300004AF
:1077480040EA03609DF8073018439DF8063040EA88
:1077580003203EBD37B500230193002400E02846EE
:10776800451C00F0A9FF01ABADB2E0540134042C74
:10777800F5D19DED010A3EBD7047000038B50446BD
:10778800642001F051F925786068AD00EDB22570EC
:1077980008F0EDFB237A40FA03F000F003000543FC
:1077A800104B257005F00F055A5D6378D218D2B2D8
:1077B800D3B20132D2B2022A637001D80022A27079
:1077C8005BB2012B03DD0123A3700023637094F9DE
:1077D8000130013303DAFF23A3700023637094F9A7
:1077E800020038BDB2A40408F7B504200121234FD4
:1077F80008F000FF02AD01214FF48040012408F099
:1078080029FF00264FF4B0733846694645F8083D0D
:107818008DF804608DF8074008F044FB10202146DD
:1078280008F0E8FE78236946154800938DF804604F
:107838008DF8074008F036FB0420214608F0DAFEF0
:1078480021464FF4804008F005FF1C23384669465E
:1078580000938DF804608DF8074008F023FB0220A0
:10786800214608F0C7FEB02306488DF80460694633
:107878008DF80740009308F015FBFEBD0008024094
:107888000010024000040240802108B5034808F0B7
:1078980068FBD0F1010038BF002008BD0004024099
:1078A80008B54FF48071044808F05BFBD0F1010083
:1078B80038BF002008BD00BF0008024008B5FFF728
:1078C800E3FF08B1FFF7ECFFC0B208BD70B50028B0
:1078D8003AD01E4B1A7880181D4AC0B292F900207F
:1078E800187040B282421B4A02DD117801391970C2
:1078F80093F9001092F9002091FBF2F402FB1414A2
:107908001549E4B21C700A88144B1A80144B154AA6
:1079180018881080144A92F9000064B2013094FB70
:10792800F0F200FB1240114C2688114C258800FB10
:10793800065008800F4908880F49098802FB001281
:107948001A800E4B01221A7070BD00BFDE3900206C
:1079580009360020E5350020143A00202A36002098
:10796800DC390020DC370020163A002038370020A8
:10797800783A0020A43A0020BA370020E4350020E5
:10798800F0B5264A264C00231370264A2568167837
:10799800254A12680FE0D45C2F197F7817F0040F7E
:1079A80007D0302C02D12023135431E01B4A137026
:1079B80003E00133DBB29E42EDDA184B1B788342B9
:1079C800194B16D9A9B11A68164C31211154302116
:1079D8000BE01A681518125C2E2A19D0303AD2B268
:1079E800092A88BF29700130C0B222788242F0DAB1
:1079F8000EE01B681A5C79B12E2A0DD05118C9B255
:107A0800392903D82F2998BF302100E0392119548A
:107A1800BDE8F040FCF7C0BCF0BD00BF440D00203D
:107A280024030020983B0020003A002010B5642071
:107A380000F0FAFF8F48FFF7A1FE8F4B1B78044632
:107A48000C2B00F2ED80DFE813F00D000D00EB00C9
:107A58007400740037008A00EB008A009300AD00C0
:107A6800EB00D400FFF71CFF18B10120F9F780FEE6
:107A7800D6E0824B1888824B1B88C01A814B1B8822
:107A880090FBF3F0804B1A88804B1B88D31A804AEE
:107A9800128893FBF2F3DBB2C0B2032B00F2A5808D
:107AA800DFE803F0020406087A4A3FE07A4A3DE03C
:107AB8007A4A3BE07A4A39E0FFF7F2FED8B1002172
:107AC8000A22784810F00EF9774B002118600A2234
:107AD800764810F007F9764B18600420FEF79AF9FB
:107AE80096200521734A0023FEF7CCF90020FEF703
:107AF80091F906F055FF614B1888614B1B88C01A35
:107B0800604B1B8890FBF3F05F4B1A885F4B1B8818
:107B1800D31A5F4A128893FBF2F3DBB2C0B213B1F7
:107B2800012B62D101E05F4A00E0604A624B1A60B3
:107B38005BE0002874D0614B1A7806DD0132D2B2BE
:107B48000F2A1A7008D9102205E0013AD2B2102A79
:107B58001A7001D900221A70F9F7C4FF60E00028F2
:107B68005ED0574B93F90020002A59D1187057E07E
:107B7800FFF796FEA0B1002152480FF0FFFF524BCD
:107B8800042083ED000AFEF745F9B42005214F4A89
:107B98000023FEF777F9FAF7ABFB0020FEF73AF976
:107BA800484A16E0FFF77CFE90B1002148480FF0E4
:107BB800E5FF484B042083ED000AFEF72BF99620D9
:107BC8000521424A0023FEF75DF90020FEF722F95D
:107BD8003F4A394B1A60294B1888294B1B88C01A11
:107BE800284B1B8890FBF3F0C0B22146FFF7C8FE74
:107BF80016E0FFF755FE08B107F0AAF8364B1A68E9
:107C0800A41814F5967FB8BF344A1C60B8BF1A6030
:107C18001B68B3F5967F03DD2F4B4FF496721A60FD
:107C28002F48FFF7ABFD144B1B78013B0A2B60D89C
:107C3800DFE803F0065F5F5F5C15155F1111150043
:107C4800FFF744FEFFF720FE002852D00220BDE8CF
:107C58001040F9F78DBD234B1B78022B46D1002825
:107C6800214B01D1187010BD01DD012200E0FF2277
:107C78001A7010BD94010020A4250020143A002099
:107C8800783A002038370020DC390020BA37002045
:107C9800A43A0020E0250020042600201A2C002009
:107CA800CC250020803A0020B0010020F0390020C7
:107CB800AC0100204BA90508003A00201626002038
:107CC8000C3A0020FC3500200C0300205BA90508B5
:107CD8002036002008030020103A0020D4FEFFFFC1
:107CE800A001002004380020591A0020BDE81040E7
:107CF800ECE510BD10B58CB01E490F2268460EF099
:107D0800DFFD1D490F2204A80EF0DAFD1B490F22E2
:107D180008A80EF0D5FD00210822302000F08AFBCB
:107D2800012000F081FE002404AB1DF80420E15C72
:107D3800302000F07FFB0134012000F075FE0F2C8D
:107D4800F2D100210922302000F074FB012000F05C
:107D58006BFE002408AB1DF80420E15C302000F025
:107D680069FB0134012000F05FFE0F2CF2D10CB04A
:107D780010BD00BFC4A40408D3A40408E2A40408E6
:107D880010B58CB01E490F2268460EF099FD1D49AA
:107D98000F2204A80EF094FD1B490F2208A80EF02C
:107DA8008FFD00210822302000F044FB012000F064
:107DB8003BFE002404AB1DF80420E15C302000F0F9
:107DC80039FB0134012000F02FFE0F2CF2D10021E5
:107DD8000922302000F02EFB012000F025FE0024AF
:107DE80008AB1DF80420E15C302000F023FB0134CF
:107DF800012000F019FE0F2CF2D10CB010BD00BF0D
:107E0800F1A4040800A504080FA5040810B58CB057
:107E18001E490F2268460EF053FD1D490F2204A883
:107E28000EF04EFD1B490F2208A80EF049FD002157
:107E38000822302000F0FEFA012000F0F5FD0024B1
:107E480004AB1DF80420E15C302000F0F3FA0134A3
:107E5800012000F0E9FD0F2CF2D100210922302089
:107E680000F0E8FA012000F0DFFD002408AB1DF85F
:107E78000420E15C302000F0DDFA0134012000F03C
:107E8800D3FD0F2CF2D10CB010BD00BF1EA5040805
:107E98002DA504083CA5040807B50220012108F017
:107EA800A9FB012300938DF8043002238DF80530D7
:107EB8000448002369468DF806308DF8073007F02E
:107EC800F1FF0EBD0004024010B5084C012100224C
:107ED800204608F05CF840F2FF4000F0A5FD0121C3
:107EE80020460A46BDE8104008F051B80004024098
:107EF80008B5FFF7E9FF00210A46302000F09AFA9A
:107F0800012000F091FD01210A46302000F092FA8C
:107F1800012000F089FD00210122302000F08AFABA
:107F2800012000F081FD01210822302000F082FAB2
:107F3800012000F079FD02210122302000F07AFAB8
:107F4800012000F071FD00210A46302000F072FA8D
:107F5800012000F069FD1B21CD22302000F06AFAD3
:107F6800012000F061FD04210322302000F062FAB4
:107F7800012000F059FD06210922302000F05AFAAC
:107F8800012000F051FD07210822302000F052FAAC
:107F9800012000F049FD08217022302000F04AFA43
:107FA800012000F041FD1E213020B02200F042FAED
:107FB800012000F039FD05219122302000F03AFA25
:107FC800012000F031FD0D210322302000F032FAAB
:107FD800012000F029FD0E210022302000F02AFAAD
:107FE800012000F021FD14218022302000F022FA27
:107FF800012000F019FD0B218822302000F01AFA28
:10800800012000F011FD0C218222302000F012FA2C
:10801800012000F009FD12218822302000F00AFA20
:10802800012000F001FD13218C22302000F002FA1B
:10803800012000F0F9FC00210A46302000F0FAF98E
:10804800012000F0F1FC3D210222302000F0F2F97D
:10805800012000F0E9FCFFF74DFEFFF791FEFFF766
:10806800D5FE30200021012200F0E4F9012000F0C3
:10807800DBFC3D216422302000F0DCF9012000F017
:10808800D3FC03210022302000F0D4F9012000F0B5
:10809800CBFC04210022302000F0CCF9012000F0B4
:1080A800C3FC00210122302000F0C4F9012000F0B7
:1080B800BBFC0C210822302000F0BCF9012000F0A4
:1080C800B3FC0D210822302000F0B4F9012000F0A3
:1080D800ABFC0E210822302000F0ACF9012000F0A2
:1080E800A3FC0F210822302000F0A4F9012000F0A1
:1080F8009BFC00210A46302000F09CF9012000F08A
:1081080093FC02224021302000F094F9012000F075
:108118008BFC30204121002200F08CF9012000F076
:1081280083FC3F21D422302000F084F9012000F0A4
:108138007BFC00210122302000F07CF9012000F0B6
:1081480073FC10210F22302000F074F9012000F098
:108158006BFC11210F22302000F06CF9012000F097
:1081680063FC12210022302000F064F9012000F0A5
:108178005BFC13210022302000F05CF9012000F0A4
:1081880053FC09213C22302000F054F9012000F072
:108198004BFC00210122302000F04CF9012000F0B6
:1081A80043FC30203421024600F044F9012000F05D
:1081B8003BFC30203721024600F03CF9012000F05A
:1081C80033FC36210322302000F034F9012000F07E
:1081D8002BFC39210322302000F02CF9012000F07B
:1081E80023FC3B213C22302000F024F9012000F040
:1081F8001BFC3C210A46302000F01CF9012000F04D
:1082080013FC00210A46302000F014F9012000F088
:108218000BFC5121C022302000F00CF9012000F0A5
:1082280003FC52213020002200F004F90120BDE8AF
:10823800084000F0F9BB00BF2DE9F04F454E464D10
:1082480093B001214FF4001008F0D4F9304607F03C
:1082580077F94FF0C0630293404B0393404B0024DF
:1082680004934FF4B4794FF400334FF480684FF41B
:1082780000674FF4005A4FF4807B304602A90C93F4
:1082880001930997CDF8189005940794CDF82080AC
:10829800CDF828A0CDF82CB00D9407F0DDF92246D2
:1082A8003046304907F033FA3046012107F039FAF1
:1082B80001210A464FF0402008F00AFC284607F042
:1082C8003FF9294A019B0392284A0C9304922846B5
:1082D800402202A9059209970294CDF818900794B4
:1082E800CDF82080CDF828A0CDF82CB00D9407F05B
:1082F800B3F9224628461E4907F009FA2846012103
:1083080007F00FFA42F2107701220221194808F00B
:10831800DFFB384600F088FB3046012107F0D7F92B
:108328000121284607F0D3F9384600F07DFB0B23DE
:108338008DF8443011A801238DF845408DF846404A
:108348008DF8473000F08EFD384600F06DFB13B015
:10835800BDE8F08F10600240886002400C40004089
:10836800CA2200202A1D00200C3C0040FA1F0020D1
:108378005A1A0020003C004002481021012207F050
:108388001DBA00BF1060024013B50220012108F099
:1083980031F94FF410730E4C009302238DF804301A
:1083A8008DF8053001238DF80630204600236946F4
:1083B8008DF8073007F076FD20460621042207F0E5
:1083C800F1FD20460921042207F0ECFD1CBD00BF89
:1083D8000004024030B5154D85B001214FF400105E
:1083E80008F02CF9284607F0F3FD0023ADF8043017
:1083F8004BF6FF73ADF806303323ADF808304FF471
:108408008063ADF80A304FF48043ADF80C3004AC0B
:10841800074B2846012144F8103D07F07BFE28460B
:10842800694607F003FE05B030BD00BF00540040A8
:10843800801A060073B54FF4961306460D46144687
:10844800019304E0019B5A1E0192002B57D031483A
:108458004FF4003107F076FF0028F3D12D480121B1
:1084680007F064FE4FF48053019304E0019B5A1E09
:108478000192002B45D02748274907F04EFF0028D6
:10848800F4D024483146002207F068FE4FF48053A8
:10849800019304E0019B5A1E0192002B33D01D4822
:1084A8001E4907F03AFF0028F4D01A48294607F079
:1084B800D8FE4FF48053019303E0019B5A1E0192AA
:1084C8001BB31448164907F028FF0028F5D01148B7
:1084D800214607F0C6FE4FF49613019303E0019B73
:1084E8005A1E01929BB10B480E4907F02BFF00283A
:1084F800F5D00848012107F025FE002008E00120FA
:1085080006E0022004E0032002E0042000E0052049
:108518007CBD00BF0054004001000300820007003A
:10852800800007000400001037B54FF49613044686
:108538000D46019305E0019B5A1E0192002B00F0A5
:108548009B8056484FF4003107F0FCFE0028F2D11A
:108558005248012107F0EAFD4FF48053019305E0EA
:10856800019B5A1E0192002B00F088804B484C4911
:1085780007F0D3FE0028F3D048482146002207F030
:10858800EDFD4FF48053019304E0019B5A1E0192C4
:10859800002B75D04148434907F0BFFE0028F4D0AE
:1085A8003E48294607F05DFE4FF48053019304E0EE
:1085B800019B5A1E0192002B64D038483A4907F0B3
:1085C800C1FE0028F4D03548012107F0AFFD4FF473
:1085D8008053019304E0019B5A1E0192002B53D053
:1085E8002E482F4907F099FE0028F4D02B48214641
:1085F800012207F0B3FD4FF48053019304E0019B7F
:108608005A1E0192002B41D0244C2849204607F0DD
:1086180099FE0028F3D02046002107F0A7FD204648
:108628000121238B07F08EFD4FF48053019304E062
:10863800019B5A1E0192002B2AD018481C4907F0AA
:1086480081FE0028F4D0154807F00DFE4FF4805342
:108658000193124A03E0019B591E0191D3B113887B
:108668009B05F8D4012104460C4807F07FFD0B4810
:10867800104907F081FE0EE001240CE002240AE014
:10868800032408E0042406E0052404E0062402E0AC
:10869800072400E0082420463EBD00BF00540040E7
:1086A800010003008200070004000010020000100F
:1086B800400000100004001013B54FF49613044650
:1086C800019305E0019B5A1E0192002B00F0AF8038
:1086D80060484FF4003107F035FE0028F2D15D48BC
:1086E800012107F023FD4FF48053019305E0019B1E
:1086F8005A1E0192002B00F09C805648564907F0FC
:108708000CFE0028F3D05348A021002207F026FDD4
:108718004FF48053019305E0019B5A1E0192002BF0
:1087280000F089804B484D4907F0F7FD0028F3D049
:10873800210A484807F095FD4FF48053019304E05F
:10874800019B5A1E0192002B77D04248444907F0FA
:10875800F9FD0028F4D0E1B23E4807F082FD4FF45D
:108768008053019304E0019B5A1E0192002B66D0AE
:1087780038483B4907F0E6FD0028F4D03548012188
:1087880007F0D4FC4FF48053019304E0019B5A1E78
:108798000192002B55D02F482F4907F0BEFD002825
:1087A800F4D02C48A121012207F0D8FC4FF48053C3
:1087B800019304E0019B5A1E0192002B43D0254CE3
:1087C8002849204607F0BEFD0028F3D020460021A6
:1087D80007F0CCFC20460121238B07F0B3FC4FF4B3
:1087E8008053019304E0019B5A1E0192002B2CD068
:1087F80018481D4907F0A6FD0028F4D0154807F0D1
:1088080032FD4FF480530193124A03E0019B591E35
:108818000191E3B113889905F8D4012104460D4864
:1088280007F0A4FC0B48114907F0A6FD10E001244D
:108838000EE002240CE003240AE0042408E00524E6
:1088480006E0062404E0072402E0082400E00924E6
:1088580020461CBD005400400100030082000700B0
:108868000400001002000010400000100004001076
:1088780013B54FF496130446019305E0019B5A1E65
:108888000192002B00F0AF8060484FF4003107F0F0
:1088980059FD0028F2D15D48012107F047FC4FF44B
:1088A8008053019305E0019B5A1E0192002B00F0B2
:1088B8009C805648564907F030FD0028F3D05348AD
:1088C800A021002207F04AFC4FF48053019305E0F1
:1088D800019B5A1E0192002B00F089804B484D499C
:1088E80007F01BFD0028F3D0210A484807F0B9FC1F
:1088F8004FF48053019304E0019B5A1E0192002B10
:1089080077D04248444907F01DFD0028F4D0E1B271
:108918003E4807F0A6FC4FF48053019304E0019B06
:108928005A1E0192002B66D038483B4907F00AFDD1
:108938000028F4D03548012107F0F8FB4FF48053A4
:10894800019304E0019B5A1E0192002B55D02F4839
:108958002F4907F0E2FC0028F4D02C48A12101227D
:1089680007F0FCFB4FF48053019304E0019B5A1E6F
:108978000192002B43D0254C2849204607F0E2FC01
:108988000028F3D02046002107F0F0FB2046012103
:10899800238B07F0D7FB4FF48053019304E0019B2E
:1089A8005A1E0192002B2CD018481D4907F0CAFC0A
:1089B8000028F4D0154807F056FC4FF48053019373
:1089C800124A03E0019B591E0191E3B113889C05EB
:1089D800F8D4012104460D4807F0C8FB0B4811499B
:1089E80007F0CAFC10E001240EE002240CE0032486
:1089F8000AE0042408E0052406E0062404E007242D
:108A080002E0082400E0092420461CBD0054004070
:108A1800010003008200070004000010020000109B
:108A2800400000100004001082B0002304E0019B05
:108A380001330193009B01330093009B8342F6D3DB
:108A480002B0704737B54FF4805304460D46019382
:108A580004E0019B5A1E0192002B6DD03C484FF454
:108A6800003107F06FFC0028F3D13948012107F0E5
:108A78005DFB4FF48053019304E0019B5A1E019261
:108A8800002B5BD03248334907F047FC0028F4D06C
:108A98002F48A021002207F061FB4FF48053019377
:108AA80004E0019B5A1E0192002B49D028482A490C
:108AB80007F033FC0028F4D0210A254807F0D1FB41
:108AC8004FF48053019304E0019B5A1E0192002B3E
:108AD80038D01F48214907F020FC0028F4D0E1B223
:108AE8001B4807F0BEFB4FF48053019303E0019B42
:108AF8005A1E019243B31648184907F00EFC002885
:108B0800F5D01348294607F0ACFB4FF496130193B0
:108B180003E0019B5A1E0192C3B10D48104907F0AA
:108B280011FC0028F5D00A48012107F00BFB0D487D
:108B3800FFF77AFF00200AE0012008E0022006E0A3
:108B4800032004E0042002E0052000E006203EBDEA
:108B58000054004001000300820007008000070065
:108B680004000010A0860100F7B54FF480530446B6
:108B78000D461646019304E0019B5A1E0192002BF4
:108B880074D040484FF4003107F0DCFB0028F3D1E3
:108B98003C48012107F0CAFA4FF48053019304E0DE
:108BA800019B5A1E0192002B62D03648364907F0C5
:108BB800B4FB0028F4D03348A021002207F0CEFAF5
:108BC8004FF48053019304E0019B5A1E0192002B3D
:108BD80050D02C482D4907F0A0FB0028F4D0210ADA
:108BE800284807F03EFB4FF48053019304E0019BB3
:108BF8005A1E0192002B3FD02248254907F08DFBD1
:108C08000028F4D0E1B21F4807F02BFB4FF4805343
:108C1800019304E0019B5A1E0192002B2ED01948A3
:108C28001B4907F07AFB0028F4D000244FF496176C
:108C380010E0295D134807F014FB019703E0019B3E
:108C48005A1E0192E3B10F48124907F07BFB002836
:108C5800F5D00134E3B2B342EBD30A48012107F05F
:108C680071FA0D48FFF7E0FE00200AE0012008E055
:108C7800022006E0032004E0042002E0052000E0D2
:108C88000620FEBD005400400100030082000700DA
:108C98008000070004000010A086010013B505201D
:108CA800012107F0A7FC184C4FF4E053009302236E
:108CB8008DF804308DF805302046002369468DF87C
:108CC80006308DF8073007F0EDF820460A21062215
:108CD80007F068F920460C21062207F063F90622FE
:108CE80020460B21A4F5006407F05CF94FF400431B
:108CF80020466946009307F0D5F820460F21062242
:108D080007F050F91CBD00BF000802401FB504461B
:108D1800FFF7C2F8FFF75EFBFFF7EAF8FFF7BEFFC1
:108D280001214FF4004007F089FC02940F4C1023F6
:108D3800ADF80230204600236946ADF80430ADF89E
:108D48000C30ADF80030ADF8063007F0A6FD6946E6
:108D58004FF0402007F075FE2046012107F025FE60
:108D68004FF04020012107F020FE1FBD003C0040CD
:108D780082B0002304E0019B01330193009B01337F
:108D88000093009B8342F6D302B0704707B50420D6
:108D9800012107F02FFC01214FF4804007F05AFC15
:108DA8004FF40073009300238DF804300348012327
:108DB80069468DF8073007F075F80EBD00080240C7
:108DC8000D4B07B51A680D484FF47A73B2FBF3F2EE
:108DD8000B4B013A5A600B4AF02182F8231000220B
:108DE8009A6007221A60084B084A00930121084B31
:108DF80001F0E2FF0EBD00BFD00100201C260020BC
:108E080010E000E000ED00E0EC020020D0020020BD
:108E180038020020054B1A6812B11A68013A1A6024
:108E2800034B1A6801321A60704700BFDC25002026
:108E3800F425002082B0044B0190019A1A601A6848
:108E4800002AFCD102B07047DC250020704700BF23
:108E580040F0BE60024B40F42020D860704700BF4D
:108E680000ED00E0C37810B503B3164B4278DB6819
:108E78008478DB43C3F30223C3F10401C9B202FAC5
:108E880001F10F2242FA03F2C9B222400A430E4B03
:108E980001781201CB18D2B283F80023037801229B
:108EA800590903F01F0302FA03F307E003780122CC
:108EB800590903F01F0302FA03F32031024A42F86A
:108EC800213010BD00ED00E000E100E021F060413C
:108ED80021F07F01014B08439860704700ED00E0E6
:108EE800044B1A6909B1104301E022EA0000186135
:108EF800704700BF00ED00E0044B1A6804280CBF5F
:108F080042F0040222F004021A60704710E000E008
:108F1800014B93ED000A7047402C0020014B93ED64
:108F2800000A7047382C0020014B93ED000A704767
:108F38004C2C0020014B93ED000A70473C2C00207C
:108F4800014B93ED000A7047502C0020014B93ED24
:108F5800000A7047442C002010B5FDF78DFE002054
:108F6800012324210246FDF7F1FE114B1C78002055
:108F7800012C05D10146FDF7C2FF2046002104E07F
:108F88000721FDF7BCFF01200721FDF7B8FF632289
:108F98001221C020FFF74EFA02200121FDF7AFFF92
:108FA800FEF78CF80120BDE81040FEF77CB800BF42
:108FB800F40D00200D4B1B78062B05D10C4B0D4AE8
:108FC800196812688A181A600B4B1B78012B084B1A
:108FD800196805D1094A914207DD01321A607047C4
:108FE800074A914201DD01321A607047A42500202A
:108FF800142C00209C250020F40D00207FD1F008BF
:10900800FF27ED080E4B1B78062B05D10D4B0E4A9A
:10901800196812688A1A1A600C4B1B78012B094BC5
:1090280005D10B4A1968914208DC1A6070471A6822
:10903800B2F57A2FDCBF4FF47A221A60704700BF6E
:10904800A4250020142C00209C250020F40D0020CD
:1090580020A107002DE9F04F694B6A4C1B688DB0C1
:1090680019220A9068485343B0FBF1F01C190D46C9
:1090780008F050FE41EC100B0AF082FF51EC100B87
:1090880009F080F910F0010F804618BF00F1FF3891
:1090980005FB08F008F03EFE064620460F4608F09D
:1090A80039FE02460B463046394608F0D3FF0446DF
:1090B8000D4645EC104B0AF063FF57EC106B204649
:1090C80032463B46294608F0E7FCCDE9020139461D
:1090D800304609F057F946A3D3E900230B90DDE9A0
:1090E800020109F009F9002858D1012000264FF0A3
:1090F8001509314607464FF0000A4FF0000B03E010
:1091080030463946069E049FA7FB0A23541807FBDE
:109118000B333E4A43F100050023A242AB41CDE99F
:1091280004453ED3A6FB0A23141806FB0B33374825
:1091380043F100050021A042A941CDE9064530D3FD
:10914800DDE902012CA3D3E90023049C069D09F064
:10915800D3F840BBDDE9022300202D4908F07AFF4F
:1091680082468B464BEC10AB0AF00AFF5046594634
:1091780053EC102B8DED080B08F08EFCCDE90201A5
:10918800DDE9080109F0CCFB09F1FF395FFA89F93B
:1091980082468B46B9F1000FB2D104E001250024C4
:1091A80001E035463C460B9A0A9BD1B25BB918469A
:1091B80022462B46FDF7CAFD0A9801230093014673
:1091C8004246034609E022462B460120FDF7BEFD34
:1091D80001200090014642460023FDF7AAFEFDF754
:1091E8006DFF01200DB0BDE8F04FFDF75CBF00BF7B
:1091F800956479E17FFDA53DBBBDD7D9DF7CDB3D1B
:10920800103A002040787D0100E9A435FFFF0F00E7
:109218000000F03F224A234B1278012A10B518604B
:1092280009D1214A904201DD01321A601F4A1B68A8
:1092380093420DDC0AE01E4A904201DD01321A60B9
:109248001B68B3F57A2F03DC4FF47A22154B1A60AA
:10925800144B184A1968184B184C1B68CB189342C2
:10926800236018DC0020FFF7F5FE01202168FFF7D6
:10927800F1FE0B4B1C780020012C05D10146FDF7AF
:109288003EFE2046002104E00721FDF738FE0120BC
:109298000721FDF734FE034B1A68094B1A6010BD0D
:1092A800F40D0020142C00207FD1F00820A1070025
:1092B800FF27ED0880D1F0082C2C0020302C00204E
:1092C800F8350020014B1868A4E700BF10260020DD
:1092D8007047FEE7FEE7FEE7FEE770477047704716
:1092E80002F01AB910B5094CA37A4BB1084B1A68A9
:1092F80022F006021A6000F013F8204600F039FE4A
:109308004FF48020BDE8104006F028BB1C26002042
:1093180010ED00E0014800F0FBBF00BF1C26002054
:10932800364BD3F8882042F47002C3F88820344BB7
:109338001A6842F001021A6000229A60196821F046
:10934800847121F4803119602E495960196882B0FE
:1093580021F480211960DA60009201921A6842F4BF
:1093680080321A601A6802F400320192009A0132BF
:109378000092019A1AB9009AB2F5A06FF2D1204B67
:109388001B6813F4003318BF01230193019B012BC1
:109398002ED11B4B1A6C42F080521A641A4A11687B
:1093A80041F4804111609A689A609A6842F40042D8
:1093B8009A609A6842F4A0529A60144A5A601A68ED
:1093C80042F080721A6019680D4A8901FBD5104B6A
:1093D80040F205611960936823F003039360936872
:1093E80043F002039360936803F00C03082BFAD14F
:1093F800024B4FF000629A6002B0704700ED00E047
:109408000038024010300024007000400854400723
:10941800003C0240184B194A996801F00C010429D4
:1094280003D0082903D0164B19E0164B17E05968EA
:109438005A6811F4800F596814BF124B104B02F090
:109448003F02B3FBF2F30C4A5268C2F30142C1F384
:109458008811013252004B43B3FBF2F3074A136001
:10946800054B9A68054BC2F303129A1819681279CA
:1094780021FA02F21A60704700380240D001002039
:109488000024F40000127A0037B51C2301240025BB
:1094980001A88DF804308DF805508DF806408DF838
:1094A8000740FFF7DFFC2046214607F0C7F80A49C6
:1094B80041F287334B6040F24F130B800D814D8092
:1094C8004FF0804007F062FC4FF080402146224672
:1094D80008F021F83EBD00BF542C002008B54FF01D
:1094E8008040012108F02CF840B14FF08040012164
:1094F80008F031F8BDE80840FEF798BA08BD00BF8B
:1095080008B5402006F01CFA30B1FCF719FE4020DF
:10951800BDE8084006F022BA08BD0000014608B5BB
:10952800044808F0D7F90348402108F080FA0028D9
:10953800F9D008BD00440040F0B589B04FF4E133DC
:109548000120019300232B4CADF808301E4601463C
:10955800ADF80A30ADF80C30ADF810300C23ADF88A
:109568000E3007F047F84FF40030012107F066F895
:1095780020680221072206F015FD072260680321F2
:1095880006F010FD0125022704232068059305A98C
:109598008DF81A608DF81B508DF818708DF81970B9
:1095A80006F080FC08236068059305A98DF81870FB
:1095B80006F078FCA06801A908F0E2F82A4640F213
:1095C80025510D4808F01AFA262307A88DF81C30F3
:1095D8008DF81D608DF81E608DF81F50FFF742FC56
:1095E800A068294608F049F9044A054B1A6009B0F1
:1095F800F0BD00BFE40100200044004025950008AC
:109608009C3B0020024B9868002108F036B900BF47
:10961800E401002010B5094C40F22551204608F01D
:1096280010FA50B1A288D2B2112A02D1044B0121FA
:109638001970044B19884A401A8010BD0044004034
:10964800550D0020600D00207047704773B501204C
:10965800014606F0CFFF264C4FF4D853009302235F
:1096680003268DF804302046002369468DF806301D
:109678008DF807308DF8056006F014FC20460821A7
:109688000A2206F08FFC204609210A2206F08AFCED
:1096980020460B210A2206F085FC0A2220460C21CE
:1096A80006F080FC01254FF480632046694600934C
:1096B8008DF806508DF807508DF8056006F0F2FB1E
:1096C8000A210A46204606F06DFC29464FF48040E0
:1096D80006F0C0FF8020294606F098FF4FF0805022
:1096E800294606F0E7FF284606F038F97CBD00BF9A
:1096F8000000024007B54FF4C060FFF7A9FB432301
:109708008DF804300322012301A88DF805308DF867
:1097180006208DF80730FFF7A5FB0EBD78235843C8
:109728000723B0FBF3F0002301338342FCD97047D1
:109738004FF47A735843F1E737B50023104C01937F
:1097480005460320FFF7EAFFEB681A69013C01921E
:1097580013D0019A002AF4DA019A42F00102019228
:10976800019A1A61064A1969013A019102D00199D0
:10977800C907F8D40320FFF7D1FF00203EBD00BF82
:10978800410D030010B5C47874B900EB82000333AF
:109798009B10D0F8D000224603E051F8044C013267
:1097A800046004319A42F8D1002010BD033230B56C
:1097B8009210D0F8D0400B46002003E02568013015
:1097C80043F8045C04339042F8D101EB800030BDCB
:1097D8000122F0B50023827040220129C3708280E3
:1097E8000CD108230370042343704FF4A073C38083
:1097F80002230372C1724FF0A04309E041B90C2360
:109808000370062343704FF4A063C3801F4BC172DB
:1098180003F500620261C3604678044601461A46B1
:10982800002508E002F5106C02F530620A65C1F8FF
:1098380014C001353A460431B54202F12007F1D38C
:1098480003F58062426103F58862C0F8CC2006788F
:1098580003F5A0650146002203E0C1F88C500132EF
:1098680020350431B242F8D31946002202E0C4F888
:10987800CC1001320434B24201F58051F7D303F51C
:109888006063C0F80C310020F0BD00BF0000044048
:1098980038B5037AC2680025012B044625D1936B9D
:1098A800417A65F3104309B143F480139363D36895
:1098B80023F4800323F0500343F010036FF3C30332
:1098C8006FF3C7136FF351436FF3D343D36020464D
:1098D800FFF732FFE378012B3ED1052363F34405FC
:1098E800E36845F020059D6036E0D36843F0400307
:1098F800D360FFF721FF237A627A032B14BF4FF45A
:1099080034134FF43C130AB143F48013E268142073
:109918009363FFF70DFFE268217AD368032908BF34
:1099280043F48033D360237A032B15D1156B0123BD
:1099380063F39B656FF3D7552D2345F0805563F38B
:1099480016451563C820FFF7F3FEE36845F40005E4
:109958001D63C820FFF7ECFEE378012B07D1E3680D
:109968009D68052262F3440545F020059D600020AE
:1099780038BDC3689A6842F001029A6000207047B7
:10998800C3689A6822F001029A600020704707B500
:1099980000230193019B43F020030193019B61F392
:1099A8008A130193019BC2681361064B1169013B3D
:1099B800019102D001998806F8D40320FFF7AEFE82
:1099C80000200EBD410D030007B500230193019B44
:1099D80043F010030193019BC2681361064B1169A0
:1099E800013B019102D00199C906F8D40320FFF781
:1099F80095FE00200EBD00BF410D030008B5C268EA
:109A0800D36801296FF35D736FF39E7302D143F03E
:109A1800005302E009B943F080433220D360FFF7D6
:109A280087FE002008BDC368586900F00100704730
:109A3800C3685B6913F0010F14BF00200120704751
:109A4800C368586900F001007047C3685A6998698B
:109A580010407047C3685868704703691A6861F313
:109A680001021A607047C268002393614FF0FF3308
:109A78005361536053610B4B9361C3789169002B19
:109A880014BF4FF400634FF4016343F4701343F4BD
:109A9800405343F0080321EA03010B43936100207C
:109AA800704700BF00080080F8B5D0F80C310022DC
:109AB8001A60036915461A6865F3CC221A60C37ADE
:109AC800012B04461BD10321FFF7C7FFE368802160
:109AD8004FF4800261F30F0259629A62C02262F366
:109AE8000F0561F31F454FF4A072C3F8045162F3E8
:109AF8000F056FF31F45C3F80851C3F80C51102127
:109B08002046FFF744FF2046FFF75EFF2269002347
:109B18004FF0FF311361204653611E469161FF25C6
:109B2800D361214610E082691768C7F3076707F019
:109B38008007FFB2002F14BF4FF09047002717602F
:109B4800013316610430956062789342EBD30023A9
:109B58001D46FF2010E04A6D1668C6F3076606F03A
:109B68008006F6B2002E14BF4FF09046002616600D
:109B7800013315610431906062789342EBD3236915
:109B88001A6942F480721A61E278012A04D1054AFE
:109B9800402161F359421A632046FFF764FF002011
:109BA800F8BD00BF0301010003699B68C3F34103CB
:109BB800013B022B9ABF024AD05C0320704700BFCA
:109BC80080A5040810B5036981699C680A68C4F314
:109BD8004100022802D06FF30A0202E0032060F37A
:109BE8000A020A605A6842F480725A60002010BD66
:109BF80030B54D780B780022012D00EB830405D198
:109C080005FA03F3A46963F30F0205E0012505FAD9
:109C180003F3646D63F31F422368C3F3072505F05C
:109C28008005EDB26DB98D6865F30A03CD78C988F2
:109C380065F3934361F3995343F0805343F400432E
:109C480023600369D9690A43DA61002030BD30B561
:109C58004D780B780024012D224600EB830105D1B5
:109C680005FA03F3896963F30F0205E0012505FA94
:109C780003F3496D63F31F4203696FF3CF340C603C
:109C8800D96921EA0202DA61002030BDF8B54F78BF
:109C98000B78012F00EB830349D19E694C69356825
:109CA80033692A4664F3120314B967F3DC430BE003
:109CB8008F68E419013CB4FBF7F7CC7867F3DC4311
:109CC800012C08BF64F35E733361C378012B06D19E
:109CD8000B780C6900EB83039B695C610CE0CB7823
:109CE800012B09D04B693BB103690C785E6B0127E6
:109CF80007FA04F434435C63CB78012B07D103697A
:109D08009B68DB0554BF45F0005245F080520B7844
:109D180000EB830342F004429B691A60CB78012B65
:109D280038D10A788B8AC968FFF72CFD32E05E6D5E
:109D38004F6935688C6833692A462FB964F3120372
:109D4800012464F3DC430AE03F19013FB7FBF4F751
:109D5800BF05BF0D67F3DC437C4364F31203336133
:109D6800C378012B05D10B780C6900EB83035B6D7D
:109D78005C61CB78012B06D14B7913B145F00052C9
:109D880001E045F080520B7800EB830042F004427A
:109D9800436D1A600020F8BD73B54D78012D3DD193
:109DA80083694A691E681C690094E4B242B962F387
:109DB80006048DF800409DF8024065F3C4040EE0E7
:109DC8008D68AA4286BF4D6165F3060462F30604F6
:109DD8008DF800409DF80240012262F3C4048DF81A
:109DE8000240009A1A61C278012A05D10A780C69E2
:109DF80000EB82029269546146F004421A60C3780B
:109E0800002B34D14B69002B31D003690A78586B89
:109E1800012101FA02F202435A6328E00B784E69E5
:109E28008C6800EB83035B6D1A681D690095EDB2C1
:109E380006B14C6164F306059DF802408DF80050A8
:109E4800012565F3C4048DF80240009C1C61C378A9
:109E5800012B05D10B780C6900EB83035B6D5C610A
:109E68000B7800EB830042F00442436D1A60002037
:109E78007CBD4B78012B0B7800EB83000AD18269FB
:109E88001368C3F3076101F08001C9B221B143F03F
:109E9800804301E0426D136843F40013136000200F
:109EA80070474B78012B0B78C97800EB83000CBF07
:109EB8008269426D02391368C9B26FF3555301299B
:109EC80098BF43F0805313600020704703699A6974
:109ED800D8691040000C704700EB810102694B6D96
:109EE8009B6850691840704703699869DB69184096
:109EF80080B2704782B000230093C0238DF80330EE
:109F08000122002362F3C4038DF8023018238DF870
:109F18000030009A436D1A61C278012A06D100F513
:109F2800B96058611A684FF080221A6002B0704711
:109F3800D0F8143110B50446D3B103699A68D20732
:109F480016D5827A42B1D0F80C21D0F80C116FF3F3
:109F580041026FF300020A605A6842F001025A6037
:109F68000520FFF7E5FB23695A6822F001025A60D1
:109F780010BD837A63B103699B68D90708D5D0F807
:109F88000C31D0F80C216FF341036FF30003136019
:109F98007047012310B5002280F8123104460346A9
:109FA800FF2104E058698160186D01328160607892
:109FB80004338242F6D3236900221A615A61DA61B6
:109FC8004FF0FF329A612046FFF7FEFC2046102131
:109FD800BDE81040DBE44B78012B0B7800EB8300E5
:109FE8000FD183691868C0F3074000F02003DBB283
:109FF800CBB900F00200C0B200280CBF30202020EE
:10A008007047436D1868C0F3074000F02003DBB2C7
:10A018005BB900F00200C0B200280CBF4FF44050FA
:10A028004FF400507047102070474FF4805070472D
:10A038004B78012B0B7810B500EB83030AD19C6990
:10A04800102A236802D1BDE8104012E7202A0CD05C
:10A05800302A0FE05C6DB2F5805F236802D143F4CB
:10A0680000131BE0B2F5005F02D143F0006315E076
:10A07800B2F5405F0FD1C3F3074202F02002D2B21B
:10A0880022B100234B71BDE810400AE743F080631A
:10A0980043F0802302E00AB962F3CF33236010BD96
:10A0A800F8B50446FFF794FB0122002384F8122137
:10A0B80084F8133128271646194640250CE007FB7B
:10A0C80003F000F58C7022182354D3805670D17099
:10A0D8009560D1605161013362789342EFD30023D8
:10A0E8002826194640250CE006FB03F000F55C70B5
:10A0F80022182354D3805170D1709560D16051617A
:10A10800013362789342EFD32046FFF739FC2046AB
:10A11800FFF7BEFB00212046FFF770FC2046FFF743
:10A12800C3FC2046BDE8F840FFF723BC70B5CDB2AC
:10A138000C464FF0280601F07F0106FB010115F0DF
:10A14800800F14BF01F58C7101F55C7104F07F0478
:10A15800ED090C704D708A60CB7005B1CC80022B74
:10A1680001D100230B71FFF743FD002070BD10B52E
:10A17800CAB201F07F034FF0280404FB030312F076
:10A18800800F14BF03F58C7303F55C7301F07F0136
:10A19800D20919705A701946FFF759FD002010BDF1
:10A1A80038B501F07F0528246C4304F55C74011967
:10A1B8004B6100238B614B70EBB20355CA60C478C6
:10A1C800012C08BF0A6113B9FFF7E6FD01E0FFF7AC
:10A1D8005DFD002038BD70B501F07F04282565437A
:10A1E80005F58C7541190126E4B2CA600A6100229E
:10A1F8004E7044558A614B6114B9FFF7CDFD01E0FB
:10A20800FFF744FD002070BDCAB212F0800F10B5F0
:10A218004FF0280306D001F07F0403FB040303F585
:10A228008C7303E003FB010303F55C73D20901247B
:10A2380001F07F0119709C705A701946FFF719FEDA
:10A24800002010BDCAB212F0800F10B54FF02803DD
:10A2580006D001F07F0403FB040303F58C7303E0CD
:10A2680003FB010303F55C730024D20901F07F01AD
:10A2780019709C705A701946FFF713FE204610BDDE
:10A2880008B50B0604D501F07F01FFF780FB01E05C
:10A29800FFF79AFB002008BD0369002261F30A1248
:10A2A80019680A431A60704703695A6803206FF3F4
:10A2B80041025A60FFF73CBA03695A68032042F02A
:10A2C80002025A60FFF734BA11F0800F4FF02803EA
:10A2D80006D001F07F0103FB010101F58C7103E059
:10A2E80003FB010101F55C71FFF775BE11F0800FEA
:10A2F8004FF0280306D001F07F0103FB010101F5AF
:10A308008C7103E003FB010101F55C71FFF790BE5E
:10A318002DE9F74F0446FFF78BFB002800F03F823A
:10A328002046FFF792FB0546002800F03882C0F36C
:10A33800074000F00800C0B2002861D02046FFF7AF
:10A34800C5FDA146824627464FF00008DFF86CB3EA
:10A358002E4650E01AF0010F46D05FFA88F21146F7
:10A3680020460092FFF7B8FD10F0010F0546009A4D
:10A3780020D07B6D01259D60E178A94207D11B693A
:10A38800D9F87813C3F31203CB1AC9F88833DBF86A
:10A39800003020461B6811469847E378012B09D105
:10A3A800B8F1000F06D194F81131052B02D12046DF
:10A3B800FFF7A0FD05F00203DBB213B17B6D0225A8
:10A3C8009D6005F00403DBB213B17B6D04259D602D
:10A3D80005F00805EDB23DB1DBF8003020469B687A
:10A3E80098477B6D0820986008F101084FEA5A0ADF
:10A3F800043709F12809BAF1000FABD1354601201D
:10A40800C5F3074303F00403DBB2002B00F0AF8071
:10A418002046FFF769FD264683464FF00008019560
:10A428009FE01BF0010F00F0978023695FFA88F91D
:10A4380019695D6B04EB890225FA09F59269ED014A
:10A448009268EDB20D431540EA071CD55A6B0120FE
:10A4580000FA08F122EA01025A63B369974A986040
:10A46800136805465B68204649469847E378AB423F
:10A4780009D1B8F1000F06D194F81131042B02D19B
:10A488002046FFF737FD05F00403DBB213B1B369CB
:10A4980004259D6005F00803DBB213B1B3690825F4
:10A4A8009D6005F01003DBB213B1B36910259D6000
:10A4B80005F02003DBB213B1B36920259D6005F0D8
:10A4C8004003DBB213B1B36940259D6005F0020378
:10A4D800DBB213B1B36902259D6025F07F0515F045
:10A4E800FF0F39D0282505FB084505F58C75C246B0
:10A4F800AB696A69C3EB020CAB689C4528BF9C46F4
:10A508000CF1030CB3694FEA9C0C9B696746A046A3
:10A5180014E0AA68E9681C1B944228BF1446A3B239
:10A5280040464A46FFF72EF9EB681B19EB60AB690A
:10A53800E71C1C19AC61B3699B69BF089BB2BB429D
:10A5480005D9AC696B699C4201D2002BE1D1B36992
:10A55800802544469D60D04608F101084FEA5B0B10
:10A568000436BBF1000F7FF45CAF019D012005F0BC
:10A578000203DBB213B1E36802225A61C5F3076331
:10A5880003F08003DBB2CBB1A37A43B1D4F80C312A
:10A59800D4F80C216FF341036FF3000313602369B0
:10A5A8005A6822F001025A60444B1B6820469B6996
:10A5B8009847E3684FF000425A610120C5F307232A
:10A5C80003F00803DBB2F3B13C4B1B6820465B6920
:10A5D80098472369E2689B684FF400615161A27A49
:10A5E80082B1DB070ED5D4F80C311A6842F00102AB
:10A5F8001A601A6842F003021A60314B1A6942F075
:10A6080006021A61012005F00803DBB243B12B4BA7
:10A618001B682046DB689847E36808225A610120D6
:10A6280005F01003DBB2002B33D0E3689A6922F0FF
:10A6380010029A611F6A282607F00F0306FB0346DB
:10A64800C7F34343022B06F55C7602D0062B1AD1DA
:10A658000EE047F6F0733B40ABB1C7F30A1720464C
:10A66800F1683A46FFF7A2F8F368DB19F36007E0F0
:10A6780004F5B96120460822FFF798F8C7F30A17CE
:10A68800B369DF19B761E3689A6942F010029A6109
:10A698000120C5F3072303F01003DBB2002B39D0E8
:10A6A80023695A68002622F001025A603146204682
:10A6B800FFF76DF923463246FF2108E080020020AB
:10A6C80000ED00E058698160186D013281606078A2
:10A6D80004338242F6D3236901274FF0FF3267F330
:10A6E8000F069A6167F31F460F22DE615A612F2217
:10A6F8001A611A686FF30A121A602046FFF7FAFB0C
:10A70800E3684FF480525A61264B1B6820461B6948
:10A7180098473846C5F3072303F02003DBB2EBB1B3
:10A728002046FFF74FFAE3682046DE68FFF73CFA59
:10A73800032806D10023A3704FF40073A3800923D4
:10A7480004E00123A3704023A380052363F38D262F
:10A75800E3684FF40052DE6001205A61C5F30743F5
:10A7680003F01003DBB24BB10E4B1B682046DB69CC
:10A778009847E3684FF480125A610120C5F30745F2
:10A7880005F02005EDB255B1064B1B6820461B6A43
:10A798009847E3684FF400125A610120FFE7BDE8CB
:10A7A800FE8F00BF8002002043230B8000487047C3
:10A7B800F001002038B51F4B1A68511C052A196092
:10A7C80035D11979002201291A6030D09968B1F57C
:10A7D800006F08BF9A60174B9968DC68A1421A4657
:10A7E80002D100221A7122E086BFC1F5006313610D
:10A7F800C1EB0404D0F8EC3598BF14611569B3F8BF
:10A8080039300C4C9D428AB204D95918ED1AA1600E
:10A81800256104E06918A1600021ABB221610549F6
:10A8280001240C7104498A188121FFF7D4FC002007
:10A8380038BD00BF640D0020F32C002038B5282354
:10A848000A4D03FB01010A4BB1F888131B69044642
:10A8580028469847D4F8EC352046B3F84030012113
:10A868002A46FFF79DFC002038BD00BFAB2C002016
:10A878006C02002070B50B7813F0600506460C4694
:10A8880025D0202D1FD1CD88B5B113F0800F487881
:10A8980008D0214B21499B682A469847E2881F49DE
:10A8A800304625E01E4B1D4958641E4B30465D61FD
:10A8B8002A4600F022FB1DE0174B48789B68294682
:10A8C8002A46984725E000F077FB022521E04B78DF
:10A8D8000A2B11D00B2B14D0062B1AD14B881B0A2C
:10A8E800212B03D1CA883A2A28BF3A220E4930467A
:10A8F80000F0EAFA00250CE00C49012200F0E4FA25
:10A9080007E08B781BB9074A1D46936101E000F008
:10A9180053FB284670BD00BF6C020020EB2C0020C2
:10A92800F0010020640D0020020200207C0D0020B0
:10A9380010B581210446FFF71AFC01212046FFF7D4
:10A9480016FC82212046FFF712FC024B5B689847F1
:10A95800002010BD6C02002038B5D0F8EC35044654
:10A96800B3F8392081210223FFF7E0FBD4F8EC3556
:10A978000121B3F8402020460223FFF7D7FB8221AC
:10A98800082203232046FFF7D1FB094B02220025AA
:10A998001A715D71074B1B689847D4F8EC35064A65
:10A9A800B3F8403020460121FFF7FAFB284638BDAE
:10A9B800B00200206C020020AB2C002010B5074C20
:10A9C800606CFF2807D0064B064A9B680649526907
:10A9D8009847FF236364002010BD00BFF0010020EA
:10A9E8006C020020640D0020EB2C002038B51049C3
:10A9F8000B79012B19D10C690CB90C7115E0D0F841
:10AA0800EC358D68B3F839309C42AAB203D95D1988
:10AA18008D60E41A03E0A3B22C198C6000240C6149
:10AA2800044952188121FFF7D6FB002038BD00BF2A
:10AA3800640D0020F32C0020002070470020704790
:10AA48000023F0B5084A094E1D4609E01468C75CA2
:10AA5800375501340133B4F5006F146008BF156031
:10AA68008B42F3D10020F0BD700D0020F32C0020A4
:10AA7800104B114AD3F800C000232DE9F0410F4FC5
:10AA880016461D460DE0146810F8038007F8048088
:10AA98000134802C08BF2C4614603468644505D006
:10AAA80001338B42EFD10020BDE8F0810220BDE8E0
:10AAB800F08100BF7435002088350020F434002070
:10AAC80021280FD1084B1A680A701A68120A4A70AE
:10AAD8005A888A70DA78CA701A790A715A794A716A
:10AAE8009B798B71002070476402002007B502AB88
:10AAF800012103F8010D1846FFF7A2FF0EBD002142
:10AB080000E00131435C002BFBD199E798E70B4B40
:10AB18000B491A68096891420BD00A498A5C02708D
:10AB28001A680132802A1A6005D100221A600120B1
:10AB38007047002070470120704700BF743500201F
:10AB480088350020F4340020204B1A68204B1B68FD
:10AB58009A42F0B509D135E00133802B08BF0023B4
:10AB68009A4203D11A4B1A602CE01A4CE15C002976
:10AB7800F2D00A29F0D00D29EED0154C1549134D05
:10AB880023600E460023CF182268BA5CC25422689C
:10AB980001339F18802F08BF53422F689A18974295
:10ABA80010D0B25C1AB10A2A01D00D2AEBD10022CA
:10ABB800C254074A116859187F29116003D980398E
:10ABC800116000E000231846F0BD00BF8835002062
:10ABD80074350020F4340020704700BFD0F8E43505
:10ABE80010B51B6904469847032384F812310020E6
:10ABF80010BD08B5042380F81231D0F8E435DB68BD
:10AC08009847002008BD08B5D0F8E035DB6903B1E6
:10AC18009847002008BD08B5D0F8E0351B6A98476A
:10AC2800002008BD08B5D0F8E0355B6A98470020D9
:10AC380008BD002110B5402204460B46FFF776FAFE
:10AC48008021402200232046FFF770FA012384F870
:10AC58001231D4F8E435A0785B689847002010BD1D
:10AC680013B56946044600F085F99DF8001001F017
:10AC78001F03012B07D0022B0AD073B9204669465F
:10AC880000F026FA0FE02046694600F007FA0AE0CD
:10AC98002046694600F0A2F905E021F07F01C9B21B
:10ACA8002046FFF7B1FA00201CBD38B5044600293C
:10ACB8003DD190F81131022B42D1D0F83421D0F88F
:10ACC80020319A4211D9C178D21A0129C0F8342109
:10ACD80004D1D0F82411CB18C0F8243192B2204600
:10ACE800D4F8241100F000F92AE0D0F83821B2FB9A
:10ACF800F3F503FB152565B99A420AD3D0F83C3120
:10AD08009A4206D229462A4600F0EEF8C4F83C5189
:10AD180016E0D4F8E035DB682BB194F81221032A49
:10AD280001D120469847204600F00FF908E0D0F8F6
:10AD3800E0355B6923B190F81221032A00D19847C6
:10AD4800002038BD10B5044659BB90F81131032BCB
:10AD580030D1D0F88C23D0F878339A4214D9C178FE
:10AD6800D21A0129C0F88C2304D1D0F87C13C91851
:10AD7800C0F87C139A4228BF1A4692B22046D4F8EB
:10AD88007C1300F0CAF815E0D0F8E0351B6923B150
:10AD980090F81221032A00D19847204600F0C6F8FF
:10ADA80008E0D0F8E0359B6923B190F81221032A16
:10ADB80000D19847002010BD2DE9F041069F0446B8
:10ADC800164698460D46FEF741FC20462946C4F82B
:10ADD800E085C4F8E475C4F8E865FFF761F9D4F8CC
:10ADE800E4351B6898472046BDE8F041FEF782BC71
:10ADF80000207047D0F8E03510B504461B68984726
:10AE0800D4F8E4359B689847002010BD08B5D0F801
:10AE1800E0355B689847002008BD000012230B80CE
:10AE280000487047B002002004230B800048704798
:10AE3800C202002010B5044C04480A46214600F01E
:10AE480075FA204610BD00BF8C3500201EAA0508E3
:10AE58000A4608B50248034900F068FA014808BDE7
:10AE680031AA05088C3500200A4608B5024803496E
:10AE780000F05CFA014808BD3FAA05088C3500209F
:10AE880008B50A4608B9044800E00448044900F037
:10AE98004DFA034808BD00BF4AAA050857AA050885
:10AEA8008C35002008B50A4608B9044800E0044873
:10AEB800044900F03BFA034808BD00BF64AA05082E
:10AEC80085AA05088C35002010B513460C46C0F835
:10AED8003821C0F83421022280F8112100212246AD
:10AEE800FFF779F9002010BD10B50C461346002174
:10AEF8002246FFF770F9002010BD10B513460C4626
:10AF0800C0F89023C0F88C23032280F81121002177
:10AF18002246FFF745F9002010BD10B50C46134630
:10AF280000212246FFF73CF9002010BD0021042330
:10AF380010B50A46044680F811310B46FFF74BF965
:10AF48002046FEF7D7FF002010BD0021052310B5CD
:10AF58000A46044680F811310B46FFF721F92046CE
:10AF6800FEF7C8FF002010BD282303FB0100B0F83E
:10AF78008803704790F8C8350B7090F8C9354B7046
:10AF880090F8CB2590F8CA3503EB02234B8090F854
:10AF9800CD2590F8CC3503EB02238B8090F8CF2594
:10AFA80090F8CE3503EB02239BB2CB80C0F83C313E
:10AFB800012380F81131704710B591F90030002B4A
:10AFC800044601DBCB880BB9802100E00021FFF7A4
:10AFD8001BF92046BDE81040FEF78CBF38B50D467A
:10AFE80004466B780979012B10D027D3032B51D154
:10AFF80090F81231022B28D0032B47D16B889BB9CC
:10B0080091B1802910D0FFF7FFF80DE090F81231C8
:10B01800022B1AD0032B39D16B88002B3AD149B1B6
:10B02800802907D0FFF70EF9D4F8E03520469B6851
:10B03800294698472046FFF779FF2BE090F8123110
:10B04800022B02D0032B21D106E019B3802921D08D
:10B058002046FFF7D9F81DE011F0800F4FF02803C4
:10B0680006D001F07F0103FB010393F81A2103E0E6
:10B0780003FB010191F87223074B02B101221A6008
:10B08800204605490222FFF71FFF03E02046294614
:10B09800FFF792FF002038BD800D002038B590F8EA
:10B0A8001231032B04460D460CD10B79012B09D81C
:10B0B800D0F8E0359B689847EB883BB92046FFF706
:10B0C80035FF03E020462946FFF776FF002038BD0C
:10B0D80073B54B7804460D46092B00F21C81DFE856
:10B0E80013F0D10008011A01E4001A0172000A00E5
:10B0F8001A01C00092004B881A0A013A062A00F287
:10B108000A81DFE812F007001A0027000801080189
:10B1180008010801D4F8E835A0781B680DF106018C
:10B128009847EB88402B014603D094F81231012B45
:10B138003AD10823ADF8063036E0D4F8E035A078E7
:10B148009B6A0DF106019847022343700146C4F833
:10B15800EC0529E0DBB2052B00F2DD80DFE803F027
:10B1680003080D12171CD4F8E835A0785B6817E0BF
:10B17800D4F8E835A0789B6812E0D4F8E835A078D0
:10B18800DB680DE0D4F8E835A0781B6908E0D4F84E
:10B19800E835A0785B6903E0D4F8E835A0789B69C6
:10B1A8000DF1060198470146BDF80630002B00F066
:10B1B800B680EA88002A00F0B2809A4228BF1A4670
:10B1C800ADF806205CE08B88002B40F0A480CB888B
:10B1D800002B40F0A08094F812214B88032A00F03D
:10B1E8009A8003F07F05204684F813512946FFF71B
:10B1F80053F82046FFF79AFE0DB1022300E0012321
:10B2080084F812318BE08978464E0129317100F2B9
:10B21800828094F81231022B02D0032B7BD108E0F4
:10B22800002962D00121032384F8101184F8123117
:10B2380013E041B9022384F8123184F81011204632
:10B24800FFF7E4FD51E094F81011012920464DD094
:10B25800FFF7DCFD317984F810112046FFF7CAFDAD
:10B2680043E0CA88012A56D194F81231022B02D041
:10B27800032B50D102E020462B4913E004F58871D6
:10B2880020460FE094F81231023B012B43D8D4F842
:10B2980014312449002B0CBF0123032341F80C3F30
:10B2A80020460122FFF710FE39E04B88012B29D0F8
:10B2B800022B34D18B8813F0FF0F30D121691B0A80
:10B2C800013B4A68042B0FD8DFE803F003050709A0
:10B2D8000B00012306E0022304E0032302E0042319
:10B2E80000E0052363F306124A602046FFF71EFEBE
:10B2F80015E094F81231023B012B0CD84B88012B36
:10B308000DD10023C4F81431D4F8E03520469B68E9
:10B3180029469847E9E720462946FFF74DFE0020D1
:10B328007CBD00BF800D0020880D002030B5C8B15D
:10B338000023DDB20133C41814F8014C002CF8D1F5
:10B348006B1C5B0013800B7003234B70022305E01A
:10B35800CA545A1CD2B202338C54DBB210F8012BF7
:10B36800002AF5D130BD00BF70477047704770475D
:10B37800704770477047000008B5FCF785FA094B1D
:10B388005A78187002435A701AB19A7801329A7032
:10B3980030B99B78034A012B02D90023537093706C
:10B3A80008BD00BF900D00202DE9F84F394B1A78E1
:10B3B800394B2DED028B22B91A68802392FBF3F3E7
:10B3C80000E01B68354A5361354B1A8892B2002A4F
:10B3D800FBD0334B00221A80FDF79AFD10EE105A6D
:10B3E800FDF79CFD284610EE104A06F0B5FC804695
:10B3F8002046894606F0B0FC41EC100B41EC180BD6
:10B4080008F066FD57EC106BB0EE480AF0EE680ADB
:10B4180008F05EFE32463B46404649465BEC10ABC0
:10B4280006F0EEFC06F0CEFF9FED1E8A07EE100A2E
:10B43800DFED1D7A57EE087A184C52465B46C4ED8C
:10B44800007A4046494606F0DBFC06F0BBFF07EEF3
:10B45800900A27EE888A84ED018AFDF771FD84ED54
:10B46800020AFDF773FD84ED030AFCF71BF90F4B85
:10B4780062691B68D31A0E4A07EE100A1268F8EEC2
:10B48800C77A93FBF2F3C4ED047A2383BDEC028BF5
:10B49800BDE8F88FF40D0020142C0020BC370020E4
:10B4A800400D00200000F04200008C4210260020D1
:10B4B8009C25002007B50420012105F09BF84FF4D6
:10B4C8006043009301238DF8043002238DF8053082
:10B4D8000448002369468DF806308DF8073004F0DB
:10B4E800E1FC0EBD00080240084B1A684FF47A735D
:10B4F800B2FBF3F2064B013A5A60064AF02182F891
:10B50800231000229A6007221A607047D001002099
:10B5180010E000E000ED00E0034B5A6812B15A68F1
:10B52800013A5A60704700BF900D0020024B5860E6
:10B538005A68002AFCD17047900D002030B585B0BC
:10B5480004460D4601A85C490A220BF0B9F95B4B89
:10B558001B78032B10D8DFE803F00205080B01A8BD
:10B56800574907E001A8574904E001A8564901E0F6
:10B57800564901A80BF08EFA04AA131913F80C3CCB
:10B588005D19EDB22F2D01D80A3502E0392D01D908
:10B598000A3DEDB204AB1C194FF6FF7004F80C5CC1
:10B5A800FAF736FB0020FAF735FC0DF103050F24F6
:10B5B800204623345A21002315F8012FA4B2FAF7A4
:10B5C80043FCB4F5A57FF3D164205A212C22002333
:10B5D800FAF73AFC0023CD205A212C22FAF734FC42
:10B5E8000020FAF715FB354B1B78032B62D8DFE8F0
:10B5F80003F002284B5601A931480BF04BFA0A22F6
:10B6080000212F480CF06EFB314A324B127818603B
:10B61800012A06D1304A904201DC01321A602F4AD1
:10B6280006E0B0F5FA5FBCBF4FF4FA521A602C4A34
:10B638001B689342C4BF274B1A602A4B1A682A4BCF
:10B6480020E001A91F480BF025FA0A2200211D4815
:10B658000CF048FB1E4A254B12781860012A06D1C7
:10B668001D4A904201DC01321A601C4A06E0B0F51E
:10B67800FA5FBCBF4FF4FA521A60194A1B6893422A
:10B6880018DD1A4B1A6015E001A90F480BF002FAF1
:10B698000D4800210A220CF025FB154B09E001A9F1
:10B6A8000A480BF0F7F9094800210A220CF01AFBA6
:10B6B800104B186005B030BDA6AA05080F2600205B
:10B6C800E0250020042600201A2C0020CC2500208C
:10B6D800F40D0020182600201FA1070080D1F008D3
:10B6E80050DA110010260020142C0020342C0020E1
:10B6F8000C2C0020C825002010B50D4B0D4C1A68E5
:10B708000D4821460BF09EF90C4B0D481A6821464E
:10B718000BF098F90B4B0C481A6821460BF092F97C
:10B728000A4B0B481A682146BDE810400BF08AB94D
:10B7380018260020B6A00508E0250020342C00209B
:10B74800042600200C2C00201A2C0020C8250020DC
:10B75800CC2500209FED010A704700BF00000000C3
:10B768009FED010A704700BF000000009FED010A2D
:10B77800704700BF0000000018B1012801D1034B39
:10B7880000E0034B1868FDF745BD00BF0026002008
:10B798001026002010B9034B18687047024B186830
:10B7A800704700BF182600201026002010B9034B50
:10B7B80018687047024B1868704700BF342C002087
:10B7C8000026002008B54FF49570FBF77FFF40F284
:10B7D8006523C31A584240EB030008BD08B5C620CC
:10B7E800FBF774FF40F28D13C21A504240EB02007F
:10B7F80008BD4FF4957040F26521FBF759BFC6208C
:10B8080040F28D11FBF754BFDCE760EEA00AB7EEFB
:10B81800007AF0EE606A70EE077A40EE006A47EE52
:10B82800A70A36EEC77A08B5C7EE200A10EE900AC6
:10B8380006F092FA0022084B06F0E2FA0022074BC3
:10B8480006F02CF906F0BEFD07EE900AFDEEE77A49
:10B8580017EE900A9F3008BD000059400000E03FF5
:10B8680038B52DED028BF7EE008AB0EE608A70EEE7
:10B87800288A10EE900A28EE088A06F06DFA08EE7B
:10B88800A88A00220F4B06F0BBFA044618EE100AED
:10B898000D4606F061FA02460B462046294606F098
:10B8A800D9FB0022084B06F0F9F806F08BFD07EEED
:10B8B800900AFDEEE77A17EE900A7730BDEC028B1E
:10B8C80038BD00BF000069400000E03F2DE9F04F9F
:10B8D800894F2DED068B97E80F0091B00CAC10370F
:10B8E80084E80F000FCF05AE0FC697E807004FF6A4
:10B8F800FF7386E807009F2077216422F7F72DFE63
:10B90800A020772164224FF6FF73F7F726FE9E20CA
:10B91800772164224FF6FF73F7F71FFE9F207621E9
:10B9280064224FF6FF73F7F718FE4FF6FF7378217E
:10B9380064229F20F7F711FE0020F9F728FA9F20CC
:10B9480077216522FAF7A6F90C349F207721642223
:10B95800FAF7A0F90DF12C0A0394F7EE009A4FF0CC
:10B968000F0B00E04D460AF1040AF7EE008A9AED43
:10B97800009A0024B0EE68AA01E0B846354618EEF1
:10B98800900A06F0E9F95AA3D3E9002306F038FA39
:10B9980006F018FD08EE900A38EEE98AB0EE490A7A
:10B9A800F0EE480AFFF731FFB0EE490AF0EE480A18
:10B9B8000646FFF755FFB2B2074683B22CB91046C8
:10B9C80019460F22F9F7AEFA06E0A8B21FFA88F175
:10B9D800CDF800B0FAF7A8F80134B4F5967FCCD1C9
:10B9E8003D46F7EE008A002401E045464E4618EE33
:10B9F800900A06F0B1F93EA3D3E9002306F000FA55
:10BA080006F0E0FC08EE900A39EEE88AB0EE490A42
:10BA1800F0EE480AFFF7F9FEB0EE490AF0EE480AE0
:10BA28008146FFF71DFF1FFA89F2804683B22CB9C1
:10BA3800104619460F22F9F775FA05E0B0B2A9B217
:10BA4800CDF800B0FAF770F80134B4F5967FCCD190
:10BA5800039B9A4586D104AD0DF12C0B4FF0000ADB
:10BA680001E0B846B146043595ED009AF7EE008A34
:10BA7800002401E0B846B14618EE900A06F06CF9C9
:10BA88001BA3D3E9002306F0BBF906F09BFC08EEE4
:10BA9800900A38EECA8AF0EE490AB0EE480AFFF773
:10BAA800B4FEB0EE480AF0EE490A0646FFF7D8FEA3
:10BAB800B2B2074683B22CB9104619462246F9F7A6
:10BAC80031FA07E01FFA89F01FFA88F1CDF800A0D3
:10BAD800FAF72AF80134B4F5C87FCBD15D45C0D157
:10BAE80011B0BDEC068BBDE8F08F00BFAFF300804E
:10BAF800295C8FC2F528F03F84A50408121A06EEC7
:10BB0800902A081AB8EEE67A06EE900AF8EEE67A77
:10BB180008B5C7EE277A17EE900A06F01DF907A3B5
:10BB2800D3E9002306F06CF90022034B05F0B6FFB9
:10BB380006F000FC08BD00BF0000E03F0000000068
:10BB480000F073408A1A06EE902A081AB8EEE67AD0
:10BB580006EE900AF8EEE67A08B5C7EE277A17EEF1
:10BB6800900A06F0F9F807A3D3E9002306F048F98C
:10BB78000022034B05F092FF06F0DCFB08BD00BF76
:10BB88000000E03F0000000000E0684070B5064695
:10BB98000D460024610704D5A0B231462A46F9F7BC
:10BBA800C1F90134B4F5A07FF4D170BD70B5064673
:10BBB8000D460024600704D5A1B230462A46F9F79D
:10BBC800B1F90134C82CF5D170BD114B11481B785F
:10BBD8001149124A0068012B114B09D112680860FB
:10BBE8001A60104B1A68104B1A60104B1A680CE058
:10BBF8001268D2011A600B4B1A680B4BD2011A60FB
:10BC08000A4B1A68C0010860D201094B1A607047D4
:10BC1800F40D00201826002010260020342C0020C7
:10BC2800002600200C2C00209C250020EC2500205C
:10BC38002C2C0020014B1868FDF7ECBA10260020C8
:10BC480008B5FFF7C2FFBDE80840F3E770B500216B
:10BC58000A222748274D284E284C0CF043F800218B
:10BC68000A22286026480CF03DF800210A2230609C
:10BC780024480CF037F800210A22206022480CF0F2
:10BC880031F8224B326818602B682149D31A06EE26
:10BC9800903A2368B8EEE67A06EE903AF8EEE67A3D
:10BCA800C7EE277AFCEEE77A17EE903A9AB20B8045
:10BCB800531C07EE903AB8EEE77ADFED167A67EE96
:10BCC800277A154BFCEEE76A16EE901A8AB206EE52
:10BCD800902AB8EEE67A198077EEC77AF5EEC07A40
:10BCE800F1EE10FA01DD01321A80BDE87040A7E7D5
:10BCF800E025002018260020342C00200C2C0020E1
:10BD0800042600201A2C0020CC250020C82500205D
:10BD1800FC3900200000803D903A00200022F0B558
:10BD28001346202603254FF02C0C00E02646303E13
:10BD3800F6B217460132092E10F8014B0AD897FBC4
:10BD4800F5F605FB16772FB9CE1801F803C0747005
:10BD5800023301E0CC540133092AE7D12022CA5426
:10BD6800CB1848225A707A229A700022DA70F0BDF5
:10BD7800F0B51F46144B1E78012E8DB005460C46B3
:10BD880020D0A6F1030CDCF1000646EB0C06CEB978
:10BD98000E4908A80AF056FE08A86946FFF7BEFF34
:10BDA8000B496A4604A80AF04DFEBDF84800F9F7A9
:10BDB8002FFF3846F9F742FF2846214604AA3346A2
:10BDC800FAF760F80DB0F0BDA4250020B6A005086C
:10BDD800F8A7050810B501210446F9F7C9F8014B81
:10BDE8001C8110BD900D002008B50021C620FBF76E
:10BDF8005FFC4FF495700021BDE80840FBF758BC84
:10BE0800014B9F221A817047900D002000200146A7
:10BE1800C82240F23F13F9F7BFB907B50DF1070083
:10BE2800FEF775FE9DF807000EBD08B5FFF7F5FF94
:10BE38000028FBD108BD30B5044687B010EE100AC3
:10BE48000D4605F089FF02460B4601A805490AF090
:10BE5800F9FD2046294601AA0023FAF713F807B08E
:10BE680030BD00BFB0AA050808B5084803F07CFA41
:10BE78000648022103F049FB0028F9D0034803F0E3
:10BE88009FFA07EE900AB8EE670A08BD0020014045
:10BE980010B52DED028B9FED098A1924FFF7E4FFF9
:10BEA800013CE4B238EE008A002CF7D19FED040A79
:10BEB80028EE000ABDEC028B10BD00BF0000000098
:10BEC800ACC868392DE9F04F2DED068B8E4B8F4CA1
:10BED8008F495D695F68C1B00646324638A893ED60
:10BEE800038AD3ED04AAD3ED028A93ED00AA93ED59
:10BEF800069A0AF0A7FDA06805F02EFF02460B4639
:10BF080028A884490AF09EFDE06805F025FF02464E
:10BF18000B462CA880490AF095FD1AEE900A05F008
:10BF28001BFFCDE90801DDE908237C4930A80AF0A8
:10BF380089FD284605F010FFCDE90401DDE9042359
:10BF4800774934A80AF07EFD18EE900A05F004FF40
:10BF58008046894642464B46724910A80AF072FD4F
:10BF680018EE100A05F0F8FE82468B4652465B46EC
:10BF78006D4914A80AF066FD1AEE100A05F0ECFEE9
:10BF8800CDE90A01DDE90A23684918A80AF05AFD33
:10BF9800384605F0E1FE54A3D3E90023CDE90601B4
:10BFA80005F02EFF02460B461CA861490AF04AFD1F
:10BFB80049EC118B4BEC10AB08F0E6F84AA3D3E937
:10BFC800002351EC100B05F01BFF02460B4624A87A
:10BFD80058490AF037FD19EE100A05F0BDFE024671
:10BFE8000B4620A854490AF02DFDD4ED047AFDEE45
:10BFF800E77A0CA817EE902A50490AF023FDB5EE0F
:10C00800C08AF1EE10FADFED4E9A37D5304605F0CA
:10C0180091FE37A3D3E9002305F0F2FEF1EE487A4A
:10C02800044617EE900A0D4605F096FE02460B46AA
:10C038002046294605F0E4FE02460B462EA1D1E92A
:10C04800000106F007F806F0BDF99FED3E7A07EE0D
:10C05800900AF4EEC77AF1EE10FAC6BFC7EEA97AD5
:10C06800394C3A4CF4EEE97AF1EE10FA38DD9FEDEE
:10C07800347A374D374CC7EE877A76E020A3D3E978
:10C0880000235046594605F0BBFE044630460D468F
:10C0980005F050FE16A3D3E9002305F0B1FE0246D1
:10C0A8000B462046294605F0D5FF06F08BF907EE2A
:10C0B800900AB7EE007AF4EEC77AF1EE10FA46BFAE
:10C0C80067EEA97A244C254CF4EEE97AF1EE10FAE1
:10C0D8004ADD9FED1B7A224D224CC7EE877A44E059
:10C0E8001B4D42E0AFF300806666666666A64C406C
:10C0F8001F85EB51B81E1940000000A2941A6D422A
:10C108000000000080842E41AC390020BC3700209C
:10C11800D2AA0508DCAA0508E7AA0508F2AA0508B4
:10C12800FCAA050806AB050812AB05081EAB0508F6
:10C1380029AB050834AB05083FAB05084BAB050830
:10C1480000007A4400247449C1AA0508BEAA05085B
:10C1580062AA0508CAAA0508C7AA0508C4AA050844
:10C16800CDAA0508CFAA0508954D17EE900A05F047
:10C17800F3FD2A46CDE900013CA8924902940AF051
:10C1880061FC914B1A68914B1B689642CCBF002208
:10C1980001229E428E4BD8BF0022DA608D4B1B785D
:10C1A800082B40F09C800220F9F734FE4FF6FF7010
:10C1B800F9F744FD1F20F9F72BFD19210023864AC2
:10C1C8002D20F9F75FFE4FF6FF70F9F737FD0020D5
:10C1D8000024F9F71DFD0F20B42132464FF6FF73F6
:10C1E8000094FFF7C5FD0F206E2128AA2346F9F712
:10C1F80049FEB0206E210DEB00022346F9F742FEFE
:10C208000F20382118AA2346F9F73CFEB020382120
:10C218001CAA2346F9F736FE0F205C2130AA2346D4
:10C22800F9F730FEB0205C2134AA2346F9F72AFE3C
:10C238000F204A2110AA2346F9F724FEB0204A21EC
:10C2480014AA2346F9F71EFE0F209B2120AA234695
:10C25800F9F718FE0F2084213CAA2346F9F712FEAD
:10C26800B020842124AA2346F9F70CFE5B4B1B68F7
:10C27800B3F57A7FCCBF4FF4FC604FF47840F9F700
:10C28800DDFC0023A0209B210CAAF9F7FBFD544BF1
:10C298001B78012B08D14FF4FC60F9F7CFFC4FF461
:10C2A8008C7002214F4A07E04FF6E070F9F7C6FCA0
:10C2B8004D4A4FF48C7002210023F9F7E3FD00206A
:10C2C800F9F7BCFC4FF4FC60F9F7A2FCFFF7E0FDBE
:10C2D8000F20DC21FFF7AFFD1F20F9F7AFFC3D4B26
:10C2E8001B789A1FD2B2012A02D90B2B40F0258263
:10C2F8003E4B1B78023B052B00F21F82DFE813F050
:10C3080006007E00E2003B01DE015801DFED387ACD
:10C318002AEE27AA1AEE100A05F01EFD9DED060B5F
:10C328008046894607F0D4FD404653EC102B494619
:10C3380005F066FD1EA3D3E9002305F0AFFB05F069
:10C34800F9FF9DED060B044607F0C2FE404653EC8C
:10C35800102B494605F054FD02460B4616A1D1E9BB
:10C36800000105F099FB05F0E5FF4FF6E073009337
:10C37800054600230520DC213246FFF7F9FC144B63
:10C38800DB6853B11B4B18881B4B4FF4784719884F
:10C398000097A2B2ABB2F9F7C7FB164B1C60164B5D
:10C3A8004FF6E0701D60F9F733FCC6E1AFF300808B
:10C3B8000000000000E063400000000000C05D4095
:10C3C800CDAA050858AB0508342C002018260020F3
:10C3D800900D0020A425002065AB05084C1A00200C
:10C3E800F40D0020D0A90508D4A90508282C0020A0
:10C3F8000000C842F83700209C3A0020A04B18687B
:10C40800A04B9FEDA19A19683246FFF777FBF4EE2F
:10C41800498AF1EE10FAC8BFF0EE498AF5EE408A73
:10C42800DFED9A7AF1EE10FA48BFF0EE678AF4EE83
:10C43800C98AF1EE10FA04461ED8F4EEE78AF1EE46
:10C4480010FA19DBFDEEE88A002018EE902A4FF466
:10C45800FA71FFF777FB8E4BDB68054653B18D4BBE
:10C4680018888D4B4FF6FF7719880097A2B2ABB2A8
:10C47800F9F75AFB884B1D60B4EE498ADFED827AE2
:10C48800F1EE10FAC8BFB0EE678ADFED847AB4EE39
:10C49800678AF1EE10FA48BFB0EE678AB4EEC98A2F
:10C4A800F1EE10FA00F24981B4EEE78AF1EE10FAE3
:10C4B800C0F24381BDEEC88A794818EE102A4FF4BD
:10C4C800FA71AEE06E4B18686E4B32461968FFF78A
:10C4D80015FBF5EEC0AAF1EE10FA044627DDDDE9FA
:10C4E800080159A3D3E9002305F0FCFEF8B158A3CD
:10C4F800D3E90023DDE9080105F082FC0B4602467A
:10C508006849002005F0C8FA05F014FF604BDB68A5
:10C51800054653B15F4B18885F4B4FF6FF77198874
:10C528000097A2B2ABB2F9F7FFFA5B4B1D60DDE9E9
:10C53800040149A3D3E9002305F0F2FE002800F026
:10C54800FC80DDE9040140A3D3E9002305F0CAFE1D
:10C55800002800F0F28042A3D3E90023DDE90401BA
:10C5680005F04EFC02460B4600204F4905F094FAB0
:10C5780005F0E0FE57E0424B1868424B3246196816
:10C58800FFF7BCFA38A3D3E900230446DDE90A0122
:10C5980005F0C6FE50B19DED0A0B07F07DFE0022A6
:10C5A80051EC100B414B05F02BFCB1E0C825B2E073
:10C5B8002FA3D3E90023DDE9060105F021FC2EA312
:10C5C800D3E9002305F046FD05F0FCFE2C4B08EEF0
:10C5D800100A18682B4B32461968FFF78FFADFEDFF
:10C5E800347A4AEE677A2A4BFDEEE77ADB6817EE73
:10C5F800905A044625EAE57553B1264B1888264B10
:10C608004FF6FF7719880097A2B2ABB2F9F78CFA08
:10C61800BDEEC88A204B18EE102A1D606FF0B300DB
:10C62800B421FFF78FFA1A4BDB68054653B1194B53
:10C638001888204B4FF4FC6719880097A2B2ABB258
:10C64800F9F772FA1B4B75E09A9999999999B93F3C
:10C658000000000000409F409A9999999999B9BFA4
:10C668000000000000408F4089B5F81400E3693FDE
:10C6780000000000008076401F85EB51B81E19406D
:10C6880018260020342C00200000FA430000000087
:10C69800900D0020F83700209C3A00200000FAC3D3
:10C6A8000CFEFFFF0000694000005940000054C024
:10C6B80000004843E83500200000C8425FED027AD8
:10C6C800B4EE679AF1EE10FAC8BFB0EE679AB4EE0E
:10C6D800E79AF1EE10FA30D8214B1868214B324610
:10C6E8001968FFF70BFA044619EE100A05F034FB37
:10C6F80041EC100B07F0D0FD00221B4B51EC100B46
:10C7080005F07EFB02460B460020184905F0C4F9E7
:10C7180005F010FE0546164BDB6853B1154B18881B
:10C72800154B4FF6FF7719880097A2B2ABB2F9F70D
:10C73800FBF9114B1D600F4B1C60104B1B78022B33
:10C7480009D043B14FF6FF7300930520DC21324630
:10C758000023FFF70DFB41B0BDEC068BBDE8F08F61
:10C7680018260020342C00200000594000006940A1
:10C77800900D0020F83700209C3A0020282C00203B
:10C7880010B54FF4C770FAF7A1FFDB2805D14FF4B5
:10C79800C870FAF79BFF84B219E041F2E104214620
:10C7A80044F20100FAF784FF44F20100FAF78EFF21
:10C7B800A04214BF80244FF4007421B24FF4C87013
:10C7C800FAF776FF4FF4C770DB21FAF771FF2046BE
:10C7D80010BD024B00221A60704700BF04360020CB
:10C7E80070EEA10A88B030EE010A08B0704770EE0A
:10C7F800E10A88B030EE410A08B07047F0EE407A9E
:10C8080020EEA10A60EE810A47EEA10A88B017EE71
:10C81800810A08B07047D0B561EEA17A41EE017A7D
:10C828002DED048B17EE900A88B0B0EE409AF0EE2A
:10C83800609AF0EE418AB0EE618A05F08DFA002226
:10C84800002306460F4605F043FDE8B969EE887AED
:10C8580049EE287A29EE088A17EE900A05F07CFA44
:10C8680032463B4605F0F6FB19EEA88A05F0AAFD0C
:10C87800044618EE100A05F06FFA32463B4605F0FA
:10C88800E9FB05F09FFD01E00448044600EE900A2C
:10C8980000EE104A08B0BDEC048BD0BD0050C34771
:10C8A800F0B58D4B2DED068B93ED001AD3ED011AE3
:10C8B8008FB0F0EE408AB0EE608A8DED060ACDEDBD
:10C8C800070A30EE410A70EEE10A38EE811A78EE76
:10C8D800211A8DED0C1ACDED0D1A8DED0A0ACDED4C
:10C8E8000B0AFFF798FF8DED040ACDED050A04AA9F
:10C8F80092E8030008AB83E80300DDED099A9DED9B
:10C9080008AA69EEA97A4AEE0A7A17EE900A05F0A3
:10C9180023FA41EC100B07F045FD51EC100B05F024
:10C9280051FD09EE100A19EE900A05F015FA0446B1
:10C938001AEE100A0D4605F00FFA45EC104B41ECC3
:10C94800110B07F021FC51EC100B05F03BFD68EED4
:10C95800087A48EEA87AB1EE48AAC8EEA79A5F4BC3
:10C968005F4D5A691B8B6860EA612B8404468AEE26
:10C9780027AA85ED009A19EE100AC5ED028A85ED01
:10C98800038AC5ED049A85ED05AA05F0E5F94CA3DF
:10C99800D3E9002305F0C4FCDFED527A002818BF64
:10C9A800B0EE679AB7EE007A79EE077A37EE497AF1
:10C9B8004D4BC7EE877A1B78033BC5ED067A042BEF
:10C9C80071D8DFE803F0032738664F0018EE100A25
:10C9D80005F0C2F9044618EE900A0D4605F0BCF9B8
:10C9E80006460F4647EC116B45EC104B07F0CCFBA5
:10C9F80035A3D3E9002351EC100BCDE9004505F030
:10CA0800FFF93246CDE902013B46384938480AF079
:10CA180019F848E019EE900A05F09EF904461AEE56
:10CA2800100A0D4605F098F92246CDE900012B467B
:10CA38002F4830492AE019EE100A05F08DF941EC2B
:10CA4800100B07F029FC00222B4B51EC100B05F0C2
:10CA5800D7F905F0B7FC05F07FF902460B462448E4
:10CA680026491EE019EE100A05F076F9064620461A
:10CA78000F4605F071F916A3D3E9002305F0C0F9B4
:10CA8800CDE900011A481E4932463B4609F0DAFF53
:10CA980009E017EE900A05F05FF902460B461448C4
:10CAA800184909F0CFFF124C00230220CA21224660
:10CAB800F9F7E8F9002323700FB0BDEC068BF0BD41
:10CAC800AE47E17A14AEEF3F6666666666A64C40EE
:10CAD800F6285C8FC2A54C402C360020BC370020BD
:10CAE800AC390020A4707D3F282C002084AB0508B9
:10CAF800C83500209EAB0508000034C0AEAB050861
:10CB0800C0AB0508DCAB050800B560EEA07A40EEC6
:10CB1800007A2DED028B17EE900A87B0B0EE408AAE
:10CB2800F0EE608A8DED020ACDED030A05F014F9E6
:10CB380041EC100B07F036FC51EC100B05F042FCF1
:10CB4800DFED117A07EE100A78EEA78A38EE078A29
:10CB580068EEA87A48EE087AC7EE277A17EE900AA8
:10CB680005F0FAF841EC100B07F01CFC51EC100B27
:10CB780005F028FC00EE900A20EE880A60EEA80A6C
:10CB880007B0BDEC028B00BD00000000F0B52DED34
:10CB9800028BDFED3A1A3A4B8DB030EEA17AF0EE07
:10CBA800407AB7EE001A8DED020A83ED001A30EED6
:10CBB800010AC3ED011A31EE671A71EEE01ACDEDE4
:10CBC800030AF0EE470A8DED077A8DED081ACDEDD0
:10CBD800091A8DED060AFFF71EFE8DED000ACDED50
:10CBE800010A9DE8030004AB83E803009DED058A74
:10CBF800DDED048A68EE087A48EEA87A17EE900A06
:10CC080005F0AAF841EC100B07F0CCFB18EE100A5F
:10CC180057EC106B05F0A0F8044618EE900A0D4684
:10CC280005F09AF845EC104B41EC110B07F0ACFA03
:10CC38003946304655EC104B05F0C4FB05F08CF82E
:10CC480041EC100B07F0A2FA002251EC100B0D4B2F
:10CC580005F0D6F805F0B6FB29460646204605F04D
:10CC6800B1FB00EE900AF6EE007A60EEA70A00EE3D
:10CC7800106A0DB0BDEC028BF0BD00BF00000000D3
:10CC8800043A00200000E03FF0EE407A86B020EE43
:10CC9800200A67EE810A06B070472DE9F04F2DEDA6
:10CCA800028B85B0FCF734F910EE105AFCF736F910
:10CCB800284610EE104A05F04FF88046204689466F
:10CCC80005F04AF841EC100B41EC180B07F000F99D
:10CCD80057EC106BB0EE480AF0EE680A07F0F8F966
:10CCE80032463B46404649465BEC10AB05F088F8B7
:10CCF80005F068FB9FED138A07EE100ADFED127A44
:10CD080057EE087A114C5B46C4ED007A524640460D
:10CD1800494605F075F805F055FB07EE900A27EE31
:10CD2800888A04AB84ED018A94E8030003E90300D0
:10CD3800DDED030A9DED020A05B0BDEC028BBDE8EE
:10CD4800F08F00BF0000F04200008C42943A0020AF
:10CD580030B53F4B2DED088BD3ED008AD3ED019A0A
:10CD68003C4BD3ED00AAD3ED01BA3B4B93ED008ABF
:10CD780093ED019A394B93ED00AA93ED01BA38EE81
:10CD8800EA0A79EEEB0A38EE4A1A79EE4B1A93B0B2
:10CD98008DED0A0ACDED0B0A8DED0C1ACDED0D1AAD
:10CDA800FFF72CFD8DED000ACDED010A9DE803008B
:10CDB8003AEE6A0A7BEE6B0A04AB38EE681A79EE33
:10CDC800691A83E803008DED081ACDED091A8DED77
:10CDD8000E0ACDED0F0AFFF711FD8DED000ACDED1E
:10CDE800010A9DE8030006AB83E803009DED040AF1
:10CDF800DDED050A9DED061ADDED071AFFF70BFDBF
:10CE08008DED000ACDED010A9DE8030002AD85E82D
:10CE18000300134B9DED021A93ED000AD3ED010AAE
:10CE2800DDED031AFFF7EAFC8DED000ACDED010AEE
:10CE38009DE8030012AB03E903006C46DDED110A1F
:10CE480085E803009DED100A13B0BDEC088B30BDDA
:10CE5800C035002018360020883A0020183A0020F3
:10CE6800E0370020F7EE007A77EEC07A20EE022A4B
:10CE780020EE210A07EEA00AF0EE420A47EE810AE8
:10CE880088B008B070472DE9F0432DED028B924B26
:10CE98001B78012B89B08146884646D14FEAC009E4
:10CEA80001291FFA89F92BD809F58065A8B2FAF784
:10CEB80051FC8A4C0435A8B284ED000AFAF74AFC02
:10CEC80009F58645A8B284ED010AFAF743FC844CBB
:10CED800043584ED000AA8B2FAF73CFCA9F5FC4039
:10CEE80084ED010A80B2FAF735FC7E4CA9F5FA40C8
:10CEF800FC3884ED000A80B2FAF72CFC84ED010AB4
:10CF080008F1FF385FFA88F8B8F1010F00F2DF8006
:10CF1800A9F57C5080B2FAF71DFC734CA9F57A5933
:10CF280084ED000AA9F17C09CBE0022B40F0CF8008
:10CF38006E4B6F4A1B68012992ED007A00F2AC80B3
:10CF480007EE900AF8EE676A07EE903A46EE877A9F
:10CF5800BDEEE77A17EE104AA4B207EE104A04F1C4
:10CF68008005ED00B8EE478AADB2284637EEC88A8C
:10CF7800FAF7F0FB0435A8B204F50665EE008DED6E
:10CF8800020AFAF7E7FBB6B230468DED030AFAF764
:10CF9800E1FB043604F58257B0B28DED040AFE00B9
:10CFA800FAF7D8FBB6B230468DED050AFAF7D2FB90
:10CFB8000436B0B281348DED060AE400FAF7CAFBF4
:10CFC800A4B220468DED070AFAF7C4FB434E043499
:10CFD800A0B286ED000AFAF7BDFB6C1CE400A4B20F
:10CFE800204686ED010AFAF7B5FB3D4D0434A0B2A0
:10CFF80085ED000AFAF7AEFB7C1CE400A4B22046DB
:10D0080085ED010AFAF7A6FB364F0434A0B287ED86
:10D01800000AFAF79FFBD6ED001A96ED012ADDED1E
:10D02800020AF0EE408A87ED010A9DED031AB0EE80
:10D03800480AFFF717FF8DED000ACDED010A9DE8BC
:10D048000300D5ED001A95ED012AB0EE480ADDED92
:10D05800040A86E803009DED051AFFF703FF8DED2E
:10D06800000ACDED010A9DE80300D7ED001A85E816
:10D078000300B0EE480ADDED060A9DED071AB0EE92
:10D08800682AFFF7EFFE8DED000ACDED010A9DE855
:10D09800030087E803006C4608F1FF385FFA88F858
:10D0A800B8F1010F13D809F5C1594FEAC9091FFA98
:10D0B80089F94846FAF74EFB0B4C84ED000A09F152
:10D0C80004091FFA89F0FAF745FB84ED010A09B053
:10D0D800BDEC028BBDE8F083B5010020883A002042
:10D0E80018360020183A0020C0350020A02500205E
:10D0F800D82500202DE9F04F2DED048B734BC7B0D8
:10D1080005464FF476701C78FAF7E0FA06464FF4B5
:10D118007570FAF7DBFA07464FF47470FAF7FEFAFF
:10D12800012C14BF10240024C0B2032D1D9040F020
:10D13800A080674A674924A809F084FCC1B224A8E2
:10D14800FDF7E4FC33463A46634924A809F07AFC23
:10D15800C1B224A8FDF7DAFC604A5E4924A809F0A8
:10D1680071FCC1B224A8FDF7D1FC002C14BFD82053
:10D17800C820FAF7D3FA0746002C14BFDC20CC20CD
:10D18800FAF7CCFA0646002C14BFE020D020FAF7B4
:10D19800C5FA8046002C14BFE420D420FAF7BEFA62
:10D1A800F31B06EE903AB8EEE67A06EE908AF8EEB1
:10D1B800E67A3346C7EE277A3A4601904849CDF8D1
:10D1C800008024A8FDEEE77ACDED027A09F03AFC5A
:10D1D800C1B224A8FDF79AFC424A3E4924A809F0A6
:10D1E80031FCC1B224A8FDF791FCE820FAF796FAC1
:10D1F8000746EC20FAF792FA0646F020FAF78EFA7C
:10D208008046F420FAF78AFAF31B07EE903A06EE06
:10D21800908AB8EEE77AF8EEE67A3A46C7EE277AC9
:10D2280001902F49CDF80080334624A8FDEEE77A17
:10D23800CDED027A09F006FCC1B224A8FDF766FC20
:10D248001D9A022A08D124A8274909F023FC24A8FA
:10D258001421FDF75BFC29E11D9B012B40F0228185
:10D2680024A8224909F016FC24A81021FDF74EFC39
:10D2780003E01D9A012A40F01581002C14BFD82024
:10D28800C820FAF74BFA1B90002C14BFDC20CC20E6
:10D29800FAF744FA0646002C14BFE020D020FAF72B
:10D2A8003DFA1B9B1C90F61A06EE906AB8EEE67AD9
:10D2B80006EE900AF8EEE67A1026C7EE277A0024E2
:10D2C800FDEEE77ACDED1F7AE7E000BFF40D002010
:10D2D800ECAB0508E7AB0508F6AB050803AC050899
:10D2E80009AC050852AC050858AC05086DAC050832
:10D2F8001C9B1B9A2046012103FB042AFFF7C3FD50
:10D30800944B954A18681768D3ED018A92ED019AF3
:10D31800924B934AD3F80090D3ED019A1368012DEC
:10D32800209392ED018A7ED1F5EEC08AF1EE10FAD3
:10D3380054BF4FF0000C4FF0010CB5EEC09ABCF191
:10D34800000F0CBF4FF02B084FF02D08F1EE10FA2C
:10D3580054BF4FF0000E4FF0010EF5EEC09ABEF12B
:10D36800000F0CBF2B262D26F1EE10FA54BF00211A
:10D378000121B5EEC08A00290CBF4FF02B0B4FF0EE
:10D388002D0BF1EE10FA54BF00220122002A0CBF27
:10D398002B232D231E93BCF1000F01D0F1EE688AD8
:10D3A800BEF1000F01D0B1EE499A09B1F1EE699AC8
:10D3B8000AB1B1EE488A04F0CFFCCDE9000118EEBD
:10D3C800900ACDF8088004F0C7FCCDE9040138467E
:10D3D80004F0C2FCCDE9060119EE100A089604F023
:10D3E800BBFCCDE90A01484604F0B6FCCDE90C01C6
:10D3F80019EE900ACDF838B004F0AEFCCDE9100172
:10D40800209804F0A9FC1E9ACDE9120118EE100A22
:10D41800149204F0A1FC5246CDE9160124A8514902
:10D4280009F010FB2FE0022D2ED1FFF791FC8DEDB6
:10D43800220ACDED230A22AB93E8030046AB03E9A9
:10D448000300DDED457AF5EEC07AF1EE10FA449866
:10D4580005D5F1EE677A17EE906A2D2702E017EEF0
:10D46800906A2B2704F078FC02460B463046CDE93B
:10D478000023029704F070FC5246CDE9040124A869
:10D48800394909F0DFFAC6B224A83146FDF73EFB58
:10D498000120FEF74BF80134A4B21F9BA342BFF64C
:10D4A80027AF70E11D9A022A40F06D81E820FAF753
:10D4B80035F91B90EC20FAF731F90646F020FAF717
:10D4C8002DF91B9B1C9006EE900AF61AB8EEE68A18
:10D4D80006EE906AF8EEE67A002C14BFD820C82031
:10D4E800C7EE887AFDEEE77ACDED1E7AFAF716F9DF
:10D4F8000646002C14BFDC20CC20FAF70FF90746AB
:10D50800002C14BFE020D020FAF708F9BF1B07EE63
:10D51800100A06EE907AF8EEC77AB8EEE67A1B9A09
:10D528001F9087EE277A931B012D06EE903ABDEEE9
:10D53800C77A88EE278A0D4B8DED207AB8EEE67A09
:10D5480087EE277A83ED007A094B83ED008A40F055
:10D55800D0808FE0883A002018360020183A002042
:10D56800C03500207EAC0508B9AC0508A025002010
:10D57800D82500201F9A002102FB04622046219230
:10D58800FFF781FC95ED018AD8ED018AB5EEC08AD6
:10D59800F1EE10FA54BF4FF0000C4FF0010CF5EE0D
:10D5A800C08A9AED019ABCF1000F0CBF2B272D27DA
:10D5B800F1EE10FA54BF4FF0000E4FF0010EB5EE29
:10D5C800C09ABEF1000F0CBF4FF02B0B4FF02D0B84
:10D5D800F1EE10FA54BF002101212868D8F8009014
:10D5E800DAF8003000290CBF2B222D22BCF1000FE5
:10D5F80001D0B1EE488ABEF1000F01D0F1EE688A81
:10D6080009B1B1EE499A19921A9304F0A5FBCDE934
:10D61800000118EE100A029704F09EFBCDE9040100
:10D62800484604F099FBCDE9060118EE900ACDF8BA
:10D6380020B004F091FB1A9BCDE90A01184604F0CA
:10D648008BFB199ACDE90C0119EE100A0E9204F021
:10D6580083FB219ACDE910014F4924A809F0F2F97A
:10D66800C1B224A8FDF752FA01340120FDF75EFF8C
:10D67800A4B205E0494DDFF83481DFF834A1002475
:10D68800209BA342BFF676AF0024454D2DE01C9B9E
:10D698001B9A2046022103FB0426FFF7F4FB95EDB5
:10D6A800018AB5EEC08AF1EE10FA286803D5B1EE0A
:10D6B800488A2D2700E02B2704F04EFBCDE9000116
:10D6C80018EE100A029704F047FB3246CDE9040130
:10D6D800344924A809F0B6F9C1B224A8FDF716FA0E
:10D6E8000120FDF723FF0134A4B21E9BA342CEDA2A
:10D6F80049E0022D43D046E01C9B1B9A012120469D
:10D7080003FB0425FFF7BFFBFFF722FB8DED220A81
:10D71800CDED230A22AB93E8030046AB03E90300EF
:10D72800DDED457AF5EEC07AF1EE10FA449806D5AB
:10D73800F1EE677A17EE908A4FF02D0903E017EEA5
:10D74800908A4FF02B0904F007FB06460F46404627
:10D75800CDE90067CDF8089004F0FEFA2A46CDE935
:10D768000401104924A809F06DF9C1B224A8FDF7F5
:10D77800CDF901340120FDF7D9FEA4B200E0002460
:10D788001E9BA342B8DA084B1D9A1A7047B0BDEC2D
:10D79800048BBDE8F08F00BFCDAC0508883A0020A7
:10D7A800C0350020FBAC0508B50100201836002064
:10D7B800183A0020F0B52DED028B04468DB00028F4
:10D7C80000F0D480724B18890419A4B222B2002A3E
:10D7D80005DB40F23F139A42C8BF1C4600E0002414
:10D7E800F7F7B4FBA0B24EF29C71F7F7C1FB684B98
:10D7F8001C81684B186804F0AFFA5FA3D3E90023D3
:10D8080004F0FEFA04F0DEFD634B1860634B1B78EE
:10D818000A2B054624B23DD107EE104AF8EEC77A26
:10D8280017EE900A04F098FA5D4B064618680F4602
:10D8380004F080FA02460B4651A1D1E9000104F038
:10D8480009FC02460B463046394604F0D9FA06462A
:10D8580028460F4604F080FA02460B463046394601
:10D8680004F0CEFA00224F4B04F0F4FB04F0AAFDBA
:10D8780004F072FA02460B4604A84B4909F0E2F894
:10D888000020F8F7C7FA0520D72104AA0023F8F7E3
:10D89800F9FA6BE0454B1888604304F04BFA3AA359
:10D8A800D3E9002304F0D6FB04F08CFD404B08EECE
:10D8B800100A1B68FCEEC87A07EE103A17EE905A69
:10D8C800F8EEC77A3B4B68EE277A1B68FDEEE77ADD
:10D8D800ADB217EE906A28460121F618FFF7D3FA81
:10D8E800FFF736FA8DED020ACDED030A02AC94E893
:10D8F800030008AB83E80300681C80B20121FFF72E
:10D90800C2FAFFF725FA8DED020ACDED030A94E875
:10D9180003000CAB07EE105A03E90300B8EEC70A80
:10D92800DDED080A38EE400A9DED091ADDED0A1A08
:10D938009DED0B2AFFF796FA8DED020ACDED030A4D
:10D9480094E8030006AB83E803004FF6FF730093E7
:10D9580005200023DC213246FEF70AFA164B9DED1E
:10D96800060A1878DDED070AFEF79AFF0DB0BDEC40
:10D97800028BF0BDAFF300807B14AE47E17A843FA1
:10D98800000000A0D954BD410000000000F0734021
:10D99800900D0020080300207C3A0020A4250020D8
:10D9A800342C00200000F43F0EAD0508FC3900209F
:10D9B8000C2C002018260020282C00202DE9F843E4
:10D9C800461F8846B6B200250D4F12E008EB040149
:10D9D80089B23046F7F76EFA29F814000A200134A4
:10D9E800FBF722F8062CF1D116350136F22DB6B226
:10D9F80004D06FF0040407EB0509E7E7BDE8F883F6
:10DA0800383A00202DE9F04F85B00B1A0193431ED8
:10DA18009BB20293431C441F00F1060901F1FF3A2F
:10DA280001F1010B9BB20F461646A4B21FFA89F901
:10DA38001FFA8AFA1FFA8BFB039380462046514649
:10DA48003246F7F76FFA204639463246F7F76AFA50
:10DA5800204659463246F7F765FA019B0298E518C1
:10DA6800ADB229463246F7F75DFA404629463246B6
:10DA7800F7F758FA0134039829463246F7F752FA6D
:10DA8800A4B20A20FAF7D0FF4C45D7D105B0BDE8BB
:10DA9800F08F2DE9F843461F8846B6B200250E4F91
:10DAA80012E008EB040139F8142089B23046F7F780
:10DAB80039FA01340A20FAF7B7FF062CF1D11635E6
:10DAC8000136F22DB6B204D06FF0040407EB050955
:10DAD800E7E7BDE8F88300BF383A00202DE9F043B6
:10DAE8002DED068B70EE007A8DB017EE900AB0EE31
:10DAF800408A10EE904A20EE009A04F02DF906466E
:10DB080020460F4604F028F9F7EE008A41EC100B86
:10DB180041EC1A0B06F0DCF979EE287A55EC104B3B
:10DB280017EE900A04F018F92246804689462B46DB
:10DB38003046394604F064F902460B4640464946E9
:10DB480003F0AAFF04F03EFCB0EE4A0AF0EE6A0ABF
:10DB580009EE900A38EEC99ADFED377A89EE299AEC
:10DB680029EE279A06F0B4FA304653EC102B3946C2
:10DB780004F046F9044619EE900A0D4604F0ECF854
:10DB880002460B462046294604F064FA00222B4B35
:10DB980004F036F904F016FCB4EE688ADFED287A52
:10DBA800284BF1EE10FA044619EE100A08BFB0EE41
:10DBB800678A1D6804F0D0F802460B4603A822497C
:10DBC80008F040FF204604F0C7F802460B4606A8B6
:10DBD8001E4908F037FF78EE287A38EEC88A87EEB3
:10DBE800888A18EE100A04F0B7F802460B4609A80E
:10DBF800174908F027FF0520014603AA0023F8F774
:10DC080041F90520142106AA0023F8F73BF9C8209A
:10DC1800052109AA0023F8F735F94FF6E0730093B8
:10DC28000520DC212A460023FEF7A2F80DB0BDEC42
:10DC3800068BBDE8F08300BF000048420000494061
:10DC4800A4707D3FD837002017AD05081FAD050823
:10DC580027AD05082DE9F04F494B2DED048B1D78B4
:10DC6800022D85B080467BD1464E348A012120465C
:10DC7800FFF709F9FFF76CF88DED000ACDED010A01
:10DC88009DE8030004AB03E9030028469DED020A62
:10DC9800DDED030AFEF704FE3B4B1A683B4B1B689D
:10DCA80002FB04343A4B1C603A4BDFED3B7A93EDB0
:10DCB800008A68EE277A5F6817EE900A04F04CF83D
:10DCC800824638468B4604F047F841EC100B41EC8D
:10DCD800190B06F0FDF8504653EC102B594604F08A
:10DCE8008FF823A3D3E9002303F0D8FE04F04AFBFE
:10DCF800B0EE490AF0EE690A054684B206F0E8F982
:10DD0800504653EC102B594604F07AF80B4602465D
:10DD180019A1D1E9000103F0BFFE04F033FBB37C85
:10DD280081461FFA80FA1BB9B08AF18AFFF7B1FE63
:10DD3800002320465146B374FFF740FE2046514663
:10DD48001F22FFF75FFEB0EE480A00EE907AFFF759
:10DD5800C5FE338AB5829844A6F81080A6F81690B6
:10DD680005B0BDEC048BBDE8F08F00BFAFF30080B9
:10DD78000000000000E063400000000000C05D40BB
:10DD8800282C0020900D00200C2C002018260020A4
:10DD9800D8370020AC3900200000C842124B1B784D
:10DDA800022B10B50CD1114B1B78022B08D1104C4B
:10DDB8002078C0B140B2FFF74DFF0023237010BD9B
:10DDC8000C4C237E23B99F20F7F79AF8012323767A
:10DDD800064B1B78022B06D1054C94F90000FFF77F
:10DDE800E9FC0023237010BD282C002004380020F3
:10DDF800591A0020900D0020034B00201860034B97
:10DE08001870FDF7B9BC00BF0436002004380020A4
:10DE1800034B00201860034B02221A70FDF7ACBCBC
:10DE2800043600200438002037B500242546A0B267
:10DE380028213223024601340095F7F775FEB4F520
:10DE4800A07FF4D13EBD2DE9F04F2DED088B0228BF
:10DE580097B080468DED070AB34B05D0032805D04F
:10DE6800012805D10C2202E0092200E00B221A70D9
:10DE78001878F2F731FE042103914FF00009F3EE10
:10DE88000EAA9FEDAABADFEDAABA7DE1A94B1A68DE
:10DE9800A94B1B6802FB093307EE103A01211FFA50
:10DEA80089F0B8EEC78AFEF7EEFFFEF751FF8DED59
:10DEB800080ACDED090A08AD95E803000AAB83E826
:10DEC80003009E4B1A6802EBC9030EAF19689C4BFE
:10DED80019600399521812685A60FEF739FF8DEDE0
:10DEE800080ACDED090A95E803000CAB83E80300A6
:10DEF800DDED0A9A9DED0BAADDED0C8A9DED0D9ADC
:10DF0800B0EE690AF0EE4A0AB0EE681AF0EE491A65
:10DF1800FEF774FC8DED080ACDED090A95E80300BB
:10DF2800B0EE691AF0EE4A1A87E80300B0EE680A04
:10DF3800F0EE490AFEF76FFC8DED080ACDED090AEF
:10DF480095E8030010AB83E803009DED0E0ADDEDB4
:10DF58000F0AFEF7D9FD8DED080ACDED090A95E8FF
:10DF6800030016AA02E903009DED100ADDED110A6F
:10DF7800149EFEF7C9FD8DED080ACDED090A95E856
:10DF8800030087E80300DDED0F0AF5EEC00AF1EEA5
:10DF980010FA48BFF1EE600A9DED0E0ACDED0F0AAA
:10DFA800FEF7F4FD8DED080ACDED090A08AA92E8FE
:10DFB800030012AB83E803000798129D03F0CCFE20
:10DFC8005D4B139FD3F800B05E4BBDEEC87AD3F813
:10DFD80000A0CDE9040117EE102A58465146FDF776
:10DFE8008DFD07EE10AAF8EEC77A07EE10BAB4EE68
:10DFF800E78AF8EEC77AF1EE10FAB4EEE78A8CBF3A
:10E0080000220122504B0690F1EE10FAD4BF0022F4
:10E0180002F00102B8F1020FDA6012D0B8F1030F72
:10E028003ED0B8F1010F68D1304603F095FE36A313
:10E03800D3E9002303F0E4FE0022444B03F02EFD55
:10E048002AE0284603F088FEDDE9042304460D464D
:10E058002FA1D1E9000103F0FDFF02460B4620463F
:10E06800294603F0CDFE2CA3D3E9002303F0C8FE14
:10E0780004F0A8F907EE900AC7EEAA7A17EE900AFC
:10E0880003F06AFE41EC100B06F006F9002251EC91
:10E09800100B2F4B03F0B4FE04F04CF904462CE0AF
:10E0A80018EE100A03F058FE044638460D4603F0F1
:10E0B80053FE17A3D3E9002303F0A2FEDDE90423EE
:10E0C80003F0C8FF04F07EF903F046FE14A3D3E979
:10E0D800002303F095FE02460B462046294603F02E
:10E0E800B9FF04F06FF907EE900AB0EE6B7A07EE0D
:10E0F8008B7AFDEEC77A17EE904A002C2ADBC72CE4
:10E10800A8BFC72427E000BF8716D9CEF753F5BFAD
:10E118008FC2F5285CAF43400000000000907040BB
:10E1280000000080DBC48641282C00200000C8C302
:10E138000000C8430C2C002018260020F0350020D1
:10E14800C0350020342C0020900D002000006940CC
:10E15800000049C00024114BDB685BB1104B1888E4
:10E16800104B1988069B4FF6FF759AB2A3B200951B
:10E17800F7F7DAFC0B4B039A1C600699084B083238
:10E18800196009F101090392074B1B884B45BFF63B
:10E198007DAE17B0BDEC088BBDE8F08F900D002068
:10E1A800F83700209C3A0020FC3900202DE9F04384
:10E1B8002D4B85B01878F2F78FFC2C4B0B221A7078
:10E1C8002B4B1C782B4B1B78012C14BF10240024DC
:10E1D800012B0BD1002C14BFD820C820F9F79EFAC8
:10E1E8000646002C14BFE020D02004E0E820F9F710
:10E1F80095FA0646F020F9F791FA00240746DFF869
:10E2080084901D4DDFF8808020E007FB04632046E2
:10E2180001216B61A8F82040FEF735FEFEF798FD56
:10E228008DED000ACDED010A9DE8030004AB03E97A
:10E2380003000D4B9DED020A1878DDED030AFEF789
:10E248002FFB6869FDF73EFE0134A4B2B9F800302F
:10E25800A342DADA094B02221A70094B00221A7615
:10E2680005B0BDE8F08300BF282C0020A4250020BD
:10E27800F40D0020B5010020BC3700200438002030
:10E28800900D0020FC390020AC39002030B52D4D10
:10E2980095F9003085B0002B3CD0FDF785F82A4A67
:10E2A8002A4B11682A4C526819605A60608B002109
:10E2B800FEF7E9FDFEF74CFD8DED000ACDED010AF4
:10E2C8009DE8030004AB03E90300224B9DED020A1D
:10E2D800DDED030A1878FEF7E3FA1F4B628B186826
:10E2E8001E4B1B6800FB0230FDF7ECFD95F9002082
:10E2F800638BD3181A4A10681A4A12689BB200FB3B
:10E3080003206383FAF786FF174B1868FDF70EF9A9
:10E3180000232B700E4C154B628B1B889A420ED132
:10E328004FF08040002102F0C6FD0E4B1868FAF746
:10E3380071FF0F4B02221A7000236383237605B006
:10E3480030BD00BF0C3A0020BC370020C03500208B
:10E35800900D0020282C00200C2C002018260020CE
:10E368009C25002010260020C8250020FC3900200C
:10E37800043800207FB54FF08040012102F09BFD5A
:10E38800FDF712F8264A274B1168526819605A603F
:10E39800254C264B22681B68254DD31A06EE903A69
:10E3A800B8EEE67AD5ED006AF8EEE67A0021C7EE17
:10E3B800277AFCEEE77A17EE906AB0B2FEF763FDB3
:10E3C800FEF7C6FC8DED000ACDED010A9DE80300BD
:10E3D80004AB03E9030000209DED020ADDED030A0A
:10E3E800FEF75EFA134B1868134B1B6836B200FB36
:10E3F8000630124EFDF766FD1920FDF797F83078C4
:10E4080060B12A68236840B202FB0030FAF702FFC5
:10E418000B4B1868FDF78AF8002333707FBD00BFE7
:10E42800BC370020C0350020F83500201026002019
:10E438009C2500200C2C0020182600200C3A0020D7
:10E44800C825002010B500214FF0804002F033FDB0
:10E45800094B00241C702046F7F706FC074B186888
:10E46800FAF7D8FE064B074801221A70064B1C70B3
:10E47800BDE81040F3F761BA0836002010260020E6
:10E48800282C0020D4170020A425002007EE100A0D
:10E49800034BF8EE477A0022C3ED007A5A607047C2
:10E4A8002C36002007EE100A034BF8EE477A0022BC
:10E4B800C3ED007A5A607047E03700200F4B1049CF
:10E4C8001A68104B1B68D31A06EE903A0E4B1B685D
:10E4D800B8EEE67A06EE903AF8EEE67AC7EE277AD4
:10E4E800FCEEE77A17EE903A9AB20B80074B188841
:10E4F80090422CBF00200120704700BF342C002020
:10E50800FC390020182600200C2C0020142600209E
:10E5180013B502AB011D23ED010A054A89B213F8B0
:10E52800014B1454013080B28842F8D11CBD00BFA1
:10E538003A3700202DE9F8431F4F0740002F0446C3
:10E548000D4603DA013F67F00F070137BFB2DFF866
:10E5580074804FEAC7091FFA89F9484698ED000AFE
:10E5680009F10409FFF7D4FF1FFA89F098ED010AB1
:10E57800FFF7CEFF114B10261B8894FBF6F6F60129
:10E588009C42B6B20CD1701980B20D498022FAF7BC
:10E59800EBFA00B1FEE721B24FF47F70F9F788F883
:10E5A8000F2F07D17519A8B205498022FAF7DCFAAE
:10E5B80000B1FEE7BDE8F8830F000080FC390020B9
:10E5C8003A370020BC3700202DE9F043744B2DED7D
:10E5D800028B1888FF2898BF4FF4807093B0C00052
:10E5E80007F0BEFE6F4B0546186028B90520B42118
:10E5F8006D4A2B46F7F746FC0024694F6B4E4FF0E7
:10E6080000086AE0FCF7D0FE20464FF44141FFF7CE
:10E6180091FF674B1A685B6832600021736020467F
:10E62800FEF731FCFEF794FB8DED020ACDED030AEF
:10E638000DF1080999E803000AAB83E803005D4B74
:10E648009DED0A1A93ED007AD3ED017ADDED0B1AF0
:10E6580031EE470A71EEE70A31EE071A71EEA71A92
:10E668008DED0E0ACDED0F0A8DED101ACDED111AB4
:10E67800FEF7D1F88DED020ACDED030A99E8030003
:10E688000CAB83E80300FF2C4FEAC4032B4404D9E6
:10E69800C3F80080C3F8048003E00C9A1A600D9A4E
:10E6A8005A603B8840F23F10604390FBF3F080B221
:10E6B8004FF4FC630246282100933223F7F734FA1B
:10E6C8003D4B18683D4B1B68C018FAF7A3FD3C4B3F
:10E6D8001868FCF72BFF0134A4B23B88A34291DAF7
:10E6E800012213464FF4807105A804F0E5FE354E6B
:10E6F800DFF8F880294605A805F0C0F9082333702B
:10E70800314B01241C700020F6F77CFD2F48F3F7ED
:10E7180014F93078F2F7E0F92D4B9FED2E8ADFEDF2
:10E728002E8A1C700024D5ED007AB0EE687A07EEC8
:10E73800C87A2046FCEEC77A17EE906A03F0FAFA18
:10E74800264B002203F05CFB03F01CFEB6B2A3B21A
:10E75800C72E28BFC72687B253B1214BB8F800008F
:10E7680019884FF6FF7300933A463346F7F7DCF9FA
:10E778001B4BC8F8007001340835B4F5807F1E6063
:10E78800D1D1184B1868FAF745FD114B02221A70BF
:10E79800154B00221A7613B0BDEC028BBDE8F0834E
:10E7A800FC390020F03500201EA50508C0350020E2
:10E7B800BC3700202C360020F83500209C2500208E
:10E7C800C8250020282C0020510D002030170020DB
:10E7D80004380020000016430000C8420000F43F3F
:10E7E8009C3A002010260020900D0020F8370020C9
:10E7F800F0B5294B294F2A4D2A4E012285B01A70AF
:10E8080000243AE0284B1A68336802FB04336B6132
:10E81800264B1C84FCF7C8FD20464FF44141FFF706
:10E8280089FE234B2A681A606A6820465A600021CC
:10E83800FEF729FBFEF78CFA8DED000ACDED010AF3
:10E848009DE8030004AB03E903001A4B9DED020A9F
:10E858001878DDED030AFEF723F86869FDF732FB47
:10E86800154B1868154B1B68C018FAF7D3FC144BE6
:10E878001868FCF75BFE0134A4B23B88A342C1DAF6
:10E88800104B1868FAF7C6FC034B02221A700E4B9D
:10E8980000221A7605B0F0BD04380020FC390020AB
:10E8A800BC370020182600200C2C0020AC39002092
:10E8B800C0350020282C0020F83500209C25002099
:10E8C800C825002010260020900D002038B5FDF73F
:10E8D800B1F9124B124D9F221A81124B012418785C
:10E8E8002C70F2F7F9F8104B00221A600F4B1B78C6
:10E8F800072B04D00B2B0DD0062B0ED102E0BDE860
:10E90800384075E74FF0804021462C70BDE838400C
:10E9180002F0D1BABDE8384048E438BD900D002077
:10E9280004380020282C002004360020A4250020CC
:10E938002DE9F743002581462C46154E154FDFF883
:10E948005C801FE0FCF730FD49462046FFF7F2FDEA
:10E95800D8F800303868C018FAF75CFC0E4B186815
:10E96800FCF7E4FD308895FBF0F080B24FF4FC63CF
:10E978000093282102463223F7F7D6F805F59E754D
:10E98800013403353388A342DCDABDE8FE8300BFD7
:10E99800FC390020F8350020C82500209C250020DF
:10E9A80010B5104C4FF47570B4F90010F8F780FEEC
:10E9B8000D4B4FF47670B3F90010F8F779FE40F27A
:10E9C800D230F8F783FEB02804D040F2D230B0211C
:10E9D800F8F76EFE2088FFF759FD034B1888BDE84D
:10E9E80010405FE5B0010020AC01002000210A22A0
:10E9F80008B509F077F9D0F1010038BF002008BD4B
:10EA080073B5041D0E46A4B20C2200234FF6E07520
:10EA1800204601360095F7F72BF900230C22B1B2F6
:10EA280020460095F7F724F90D4B1B78012B16D1DA
:10EA38000C4E0D4D308829880024043080B20C22F9
:10EA480023460094F7F714F9308829880094043095
:10EA5800013180B289B20C222346F7F709F97CBD4F
:10EA6800E43500202A360020DC37002008B54FF6B0
:10EA7800FF70F7F7CDF80020F7F7CCF9E120232154
:10EA88002C4A0023F7F7FEF9E1204621294A002302
:10EA9800F7F7F8F9E1206921264A0023F7F7F2F998
:10EAA800E1208C21244A0023F7F7ECF92348FFF7EB
:10EAB8009DFF20B121482249012207F0C3FF4B20C6
:10EAC80023211E4A0023F7F7DDF91E48FFF78EFFC2
:10EAD80020B11C481A49012207F0B4FF4B204621F7
:10EAE800184A0023F7F7CEF91748FFF77FFF20B140
:10EAF80015481349012207F0A5FF4B206921124A46
:10EB08000023F7F7BFF91148FFF770FF20B10F484E
:10EB18000B49012207F096FF4B208C2100230B4A5A
:10EB2800F7F7B0F90A4B18880A4B1988BDE808406E
:10EB380066E700BF2EA3050833AD0508E0250020D1
:10EB4800B6A00508042600201A2C0020CC25002099
:10EB5800143A0020DC39002070B5044600200D4628
:10EB68001646F7F757F90020F7F768F84FF4FC60F6
:10EB7800F7F74EF82046294656BB1E4A3346F7F7A4
:10EB880081F91D48FFF732FF20B11B481B490122BC
:10EB980007F058FF04F17006B6B230462946164A07
:10EBA8000023F7F76FF91648FFF720FF20B1144844
:10EBB8001249012207F046FF3235ADB220462946F8
:10EBC800104A0023F7F75EF9304629460C4A07E059
:10EBD8000D4A0023F7F756F932350B4AA9B22046F9
:10EBE8000023F7F74FF9094B1888094B1988BDE836
:10EBF800704005E738AD0508803A0020C9A405082B
:10EC0800F039002040AD050869A50508143A002030
:10EC1800DC39002030B5144D9DF80C402C70134D94
:10EC28002880134D02FB04002980124D80B22880F1
:10EC3800114D2980114D2A80114A1380114B1880DB
:10EC4800114B1980114B1249E2B21A7000230B7054
:10EC580010490A709DF810200134013254430E4ABD
:10EC680014700E4A137030BD983B0020783A00208B
:10EC7800BA370020143A0020DC3900203837002049
:10EC8800A43A00202A360020DC370020DE39002094
:10EC980009360020163A0020E5350020E43500202A
:10ECA80038B5054600200C46F7F7B4F80020F6F70B
:10ECB800C5FF4FF4FC60F6F7ABFF0B48FFF796FE75
:10ECC80028B1094809490A4B002207F0BBFE28462B
:10ECD80021460023044AF7F7D5F8064B1888064B57
:10ECE8001988BDE838408BE62036002068A9050859
:10ECF8000000F03F143A0020DC390020114B1B685B
:10ED0800002B70B505460C4604DA5B420E480F49E5
:10ED18002D2202E00C480D49202207F093FE002026
:10ED2800F7F778F80020F6F789FF4FF4FC60F6F75C
:10ED38006FFF054A284621460023BDE87040F7F7D3
:10ED4800A1B800BF103A0020E837002048AD0508F8
:10ED58000F4B10B519684FF4E170F8F7C6FC40F294
:10ED68003D114FF4E070F8F7A3FC0020F7F752F8D4
:10ED78000020F6F763FF4FF4FC60F6F749FF054AF9
:10ED8800192064210023BDE81040F7F77BB800BFC5
:10ED9800103A00204FAD050808B54FF4E070F8F7B9
:10EDA80095FC40F23D13984205D14FF4E170BDE85F
:10EDB8000840F8F7B3BC002008BD38B50546002068
:10EDC8000C46F7F727F80020F6F738FF4FF4FC60F9
:10EDD800F6F71EFF0B48FFF709FE28B109480A4954
:10EDE8000A4B002207F02EFE284621460023054A3A
:10EDF800F7F748F8064B1888064B1988BDE83840DD
:10EE0800FEE500BFFC35002068A905080000F03FBA
:10EE1800143A0020DC39002038B5C501ADB2002411
:10EE2800601980B2F9F748FC0134C0B2FBF75EFE06
:10EE3800A4B24FF47A70F9F7F7FD802CF0D138BD01
:10EE480073B5104D00240E20FBF750FE002609E094
:10EE58000DF10700FBF75BFE20B19DF80730AB55BD
:10EE68000136F6B23306F3D5E00180B205498022B7
:10EE7800F9F77AFE00B1FEE70134A4B2B4F5007FD9
:10EE8800E1D17CBD3A37002007EE100AF8EE477A48
:10EE98007FB517EE900A02F05FFF02460B4601A805
:10EEA800054907F0CFFD0A20962101AA0023F6F7AD
:10EEB800E9FF07B000BD00BF56AD0508AFF30080FD
:10EEC8000EB403B070470A2810B5044602D10D20CD
:10EED800FFF7F9FF064A13681BB103F8014B1360EB
:10EEE80010BD044B1B680BB12046984710BD00BFEE
:10EEF800B00D00209C3B002010B5044601E0FFF750
:10EF0800E2FF14F8010B0028F9D110BD2DE9F04FEC
:10EF1800044685B00D464FF00A0A00E035462078D1
:10EF2800002800F0C480252801D0013467E060780B
:10EF3800302803D1A0780123033407E02D2802D01C
:10EF48000234002302E0A078022303344FF00008C3
:10EF580005E00AFB080814F8010BA8F13008A0F135
:10EF68003002D2B2092AF4D96C2801D04C2803D136
:10EF780014F8010B43F00403002800F0988060287F
:10EF880086BFA0F12002D2B202464F2A3DD006D851
:10EF9800432A2DD0442A09D0422A30D133E0552AB9
:10EFA80004D0582A29D0532A29D101E00A272DE074
:10EFB8002E1D2F68002500E001357A5D002AFBD15F
:10EFC80004E02020FFF77FFF4D4601E0980704D4B6
:10EFD800454505F10109F4D34D463846FFF78CFF46
:10EFE80003E02020FFF76FFF01354545F9D395E78A
:10EFF80028782E1DFFF767FF90E7102706E0FFF738
:10F0080062FF2E468AE7022700E008272E1D442AC1
:10F01800296804D1002902DA494243F00803002292
:10F0280000E02A46B1FBF7FE07FB1E11CDB2092D01
:10F03800714607D9782814BF4FF0070C4FF0270CFA
:10F048006544EDB230350DF80250551CBEF1000F85
:10F0580002D0102DE5D10F22190705D504A94D19A5
:10F068002D2105F8101C951C13F0010F0CBF4FF053
:10F07800200B4FF0300B9B072F4604D508E058466D
:10F08800FFF721FF4F46474507F10109F7D34F46E0
:10F09800013D1DF80500FFF716FF002DF8D103E02C
:10F0A8002020FFF710FF01374745F9D336E705B0B1
:10F0B800BDE8F08F70B5064D0C462E68286001E05B
:10F0C800FFF701FF14F8010B0028F9D12E6070BD7D
:10F0D8009C3B00200FB407B504A951F8040B01911B
:10F0E800FFF714FFBDE80E4004B070470EB417B523
:10F0F80005A9084C51F8043B206018460191FFF718
:10F1080005FF2268002313702360BDE81E4003B08A
:10F11800704700BFB00D00200EB433B505A9074CE9
:10F1280051F8043B2568206018460191FFF7EEFE70
:10F138002560BDE83C4003B0704700BF9C3B002001
:10F1480070B51E4604461C481546FFF7C3FF022E3D
:10F158001FD0042E25D0012E2AD105E0A15D174825
:10F16800FFF7B8FF013600E00026AE42F6DB2020AC
:10F17800FFF7A9FE002609E0A05DA0F12003DBB29D
:10F188005E2B88BF2E20FFF79EFE0136AE42F3DBD2
:10F198000EE034F8021B0A48FFF79CFF013DF8D146
:10F1A80006E054F8041B0748FFF794FF013DF8D127
:10F1B8000A20BDE8704086E65DAD050864AD050827
:10F1C8006AAD050870AD050808B501214FF48070D7
:10F1D80001F07CFA4FF480700021BDE8084001F08E
:10F1E80075BA43680A6823F0407323F480731343A5
:10F1F8000A7943EA02234360CA680B6930B51A43A7
:10F2080084688D68084B2A43234013434A7943EAAC
:10F21800420383600B7DC26A013B22F47002DBB2B9
:10F2280042EA0353C36230BDFDF7FFC00023036009
:10F23800037143718360C3600361012303757047E1
:10F24800074A084B516810B50B4090E8120021435B
:10F258008468C068214301430B43536010BD00BF5D
:10F2680000230140E030FCFF00230360436083601B
:10F27800C3607047836811B143F0010301E023F0D4
:10F28800010383607047436823F4400323F4007349
:10F298000B4343607047416282627047436823F0C2
:10F2A8001F030B4343607047044B5A6810B142F484
:10F2B800000201E022F400025A6070470023014076
:10F2C800044B5A6810B142F4800201E022F4800233
:10F2D8005A60704700230140092970B50CB20CD957
:10F2E80004EB44041E3CC6680725A54026EA05052C
:10F2F800A34045EA0304C4600AE0066904EB440439
:10F308000725A54026EA050513FA04F42C430461F1
:10F31800062A0CD80523013A5A43446B1F2393400D
:10F3280024EA0303914043EA0102426370BD0C2AB8
:10F3380012B20CD802EB8202233A046B1F239340CB
:10F3480024EA0303914043EA0102026370BD02EB21
:10F358008202413AC46A1F23934024EA030391407E
:10F3680043EA0102C26270BD836843F08043836050
:10F3780070478068C0F380507047836811B143F4C8
:10F38800806301E023F4806383607047836811B170
:10F3980043F0020301E023F00203836070474368EF
:10F3A800013923F4604343EA4133436070474368BB
:10F3B80011B143F4006301E023F400634360704734
:10F3C800C06C80B27047014B186870470823014031
:10F3D800836811B143F4807301E023F48073836080
:10F3E8007047836811B143F4007301E023F400739C
:10F3F80083607047044B5A6810B142F4005201E030
:10F4080022F400525A60704700230140092970B560
:10F418000CB20CD904EB44041E3CC6680725A54071
:10F4280026EA0505A34045EA0304C4600AE0066924
:10F4380004EB44040725A54026EA050513FA04F45D
:10F448002C430461836BC3F30154121B0232D2B202
:10F4580002EB82021F24944023EA040391400B43E9
:10F46800836370BD836B013923F4401343EA01536E
:10F478008363704782B0002301930190019BCB18EE
:10F488000193019B1A6002B07047836823F47023CC
:10F498000B4383607047836823F440130B438360F6
:10F4A8007047836843F48003836070478068C0F3C3
:10F4B80080507047436811B143F4806301E023F43E
:10F4C800806343607047436811B143F4805301E09F
:10F4D80023F480534360704782B000230193019066
:10F4E800019B28335B180193019B186880B202B016
:10F4F80070470123C9B213FA01F143680AB11943ED
:10F5080001E023EA010141607047036819420CBF1A
:10F51800002001207047C9430160704743680068B4
:10F5280010EA112007D00122C9B212FA01F11942DA
:10F538000CBF0020012070476FEA1121016070475D
:10F54800036823F0010303600023036043608360C2
:10F55800C3600361212343612C4B98421CD02C4B80
:10F56800984220D02B4B984225D02B4B98422AD03A
:10F578002A4B98422FD02A4B984233D0294B984295
:10F5880037D0294B984204D14FF03D5243F8AC2C68
:10F598007047264B984203D13D2243F8082C704708
:10F5A800234B984204D14FF4746243F8202C7047DF
:10F5B800204B984204D14FF4741243F8382C70470A
:10F5C8001D4B984204D14FF0746243F8502C704799
:10F5D8001A4B984203D11A4A43F8642C7047194BC6
:10F5E800984203D1184A43F87C2C7047174B98422D
:10F5F80003D1174A43F8942C7047164B984204BF1E
:10F608004FF03D5243F8AC2C704700BF10600240E9
:10F61800286002404060024058600240706002402A
:10F6280088600240A0600240B86002401064024056
:10F6380028640240406402405864024070640240FA
:10F648003D00002088640240400F0020A064024072
:10F6580000003D20B86402400268134B10B5134007
:10F66800CC680A6822434C6922438C692243CC69DE
:10F6780022430C6A22434C6A22438C6A22434C6B15
:10F6880022438C6B22431343036042690C6BCB6AA1
:10F6980022F007022343134343610B6943604B681D
:10F6A80083608B68C36010BD3F801CF0002303603B
:10F6B80043608360C360036143618361C361036224
:10F6C80043628362C362036343638363704703686F
:10F6D80011B143F0010301E023F001030360704717
:10F6E800036811B143F4004301E023F400430360CD
:10F6F8007047036811B143F0200301E023F02003B1
:10F708000360704741607047406880B27047036883
:10F7180012B143F4002301E023F4002303600161E4
:10F728007047036811B143F4802301E023F4802378
:10F73800036070470AB101617047C1607047006893
:10F74800C0F3C0407047006800F00100704740698E
:10F7580000F0380070470A4A0A4B10B50A4CA0421C
:10F7680088BF13468A004CBF5B681B6821F0F021F4
:10F7780021F0821119420CBF0020012010BD00BFEA
:10F7880000640240006002400F64024010B5084B5C
:10F79800084A094CA04288BF134611F0005F21F0C7
:10F7A800F02121F0821114BFD960996010BD00BF0B
:10F7B80000600240006402400F6402400B0607D557
:10F7C800436912B143F0800301E023F080034361F1
:10F7D800802909D001F01E01036812B119430160A4
:10F7E800704723EA010101607047124B124A10B5B5
:10F7F800124CA0428CBF14461C4621F0F02323F083
:10F80800C3132BB1026802F01E0202EAD12202E001
:10F81800426902F0800288004CBF6368236821F0C7
:10F82800F02121F08210184002D0101C18BF0120CE
:10F8380010BD00BF00600240006402400F64024037
:10F8480010B5084B084A094CA04288BF134611F06E
:10F85800005F21F0F02121F0821114BFD960996076
:10F8680010BD00BF00600240006402400F64024007
:10F87800044B00221A605A609A60DA60024A5A61A0
:10F88800704700BF003C0140FFFF7F00837910B53F
:10F89800002B29D01A4B01681C68CA4314401C600D
:10F8A8005C6822405A60027902F1804202F59E3279
:10F8B80014682143116002689C68D1430C409C6025
:10F8C800DC682140D9604179102906D19968114333
:10F8D8009960D9680A43DA6010BD01F1804303F5E5
:10F8E8009E3319680A4308E00379016803F18043ED
:10F8F80003F59E331A6822EA01021A6010BD00BFA0
:10F90800003C014000230C220360037142718371A3
:10F918007047024B1A6902431A617047003C014064
:10F92800034B5B6918420CBF00200120704700BFE1
:10F93800003C0140014B5861704700BF003C01404A
:10F94800054B1A685B69034004D010420CBF0020C5
:10F958000120704718467047003C0140014B586130
:10F96800704700BF003C01404FF0204318B943F2F4
:10F97800DB021A6003E043F2D20243F820204FF082
:10F988002042411C6FF0704342F8213002F5827228
:10F9980042F82030704770B584684568C368C16A0A
:10F9A800026825431D4303691D4343691D43836959
:10F9B8001D43C3691D43036A1D43436A1D43836A8C
:10F9C8001D43036B0D431D434FF02043082C43F8A0
:10F9D800225005D153F8224044F0400443F8224015
:10F9E800436B9E691D6835435E6845EA06159E6847
:10F9F80045EA0625DE6845EA06451E695B6945EA6B
:10FA08000655541C45EA03654FF02043B1F5804F75
:10FA180043F8245010D1836B9869196801435868DA
:10FA280041EA0011986841EA002118695B6941EAD6
:10FA3800005141EA036101E06FF07041014B43F866
:10FA4800221070BD040100A0022242604FF48052CF
:10FA58004262416B4FF4005210B5826200230F22BC
:10FA6800FF2403608360C360036143618361C361F2
:10FA78000362C36203630A604A608C60CA600A61F9
:10FA88004A618B61816B0A604A608C60CA600A6156
:10FA98004A618B6110BD4FF0204321B153F82020FB
:10FAA80042F0010203E053F82010024A0A4043F8EA
:10FAB80020207047FEFF0F0010280CBF064B074B95
:10FAC8004FF040024FF0180119605A604FF0FC32B5
:10FAD8009A60DA60704700BF600000A0800000A054
:10FAE80030B5836844681C43C36844F008041C4369
:10FAF80003691C43436944EA4324836944EA433461
:10FB0800C36999685A68090441EA02211A68DB68DE
:10FB1800114341EA0361036A9A685D68120442EA84
:10FB280005221D68DB682A4342EA03620368102B3A
:10FB38000CBF034B034B1C609960DA6030BD00BFFB
:10FB4800600000A0800000A010230360C2690023A9
:10FB580043608360C360036143618361FC23136076
:10FB680053609360D360026A136053609360D360FC
:10FB7800704741B110280CBF074B084B1A6842F078
:10FB880004021A60704710280CBF034A034A044B4A
:10FB980011680B4013607047600000A0800000A04F
:10FBA800FBFF0F0041B110280CBF084B084B1A6827
:10FBB80042F040021A60704710280CBF034A044AFA
:10FBC800044B11680B401360704700BF600000A031
:10FBD800800000A0BFFF0F00102802D1024B586917
:10FBE8007047024B58697047600000A0800000A071
:10FBF800054B18221A6000225A604FF0FC329A60B6
:10FC0800DA601A61704700BFA00000A0026843686C
:10FC180042F0100242EA4322836842EA4332144B1C
:10FC280010B51A60C26891685468090441EA042151
:10FC38001468D268214341EA02629A6002699168B5
:10FC48005468090441EA04211468D268214341EA4E
:10FC58000262DA60426991685068090441EA002149
:10FC68001068D268014341EA02621A6110BD00BF00
:10FC7800A00000A0C2680023036043608360FC23E7
:10FC8800136053609360D36002691360536093609C
:10FC9800D3604269136053609360D3607047054B2B
:10FCA80018B11A6842F0040202E01968024A0A40D0
:10FCB8001A607047A00000A0FBFF0F0062B1102877
:10FCC80001D10E4B03E0B0F5807F03D10C4B5A688D
:10FCD800114311E00B4BFAE7102804D1074B5A687F
:10FCE80022EA010108E0B0F5807F0CBF044B054B08
:10FCF8005A686FEA0101114059607047600000A01E
:10FD0800800000A0A00000A0102801D1064B04E04C
:10FD1800B0F5807F0CBF054B054B5B680B420CBFF1
:10FD280000200120704700BF600000A0800000A0F4
:10FD3800A00000A0102804D1074B5A6822EA01014C
:10FD480008E0B0F5807F0CBF044B054B5A686FEA9A
:10FD58000101114059607047600000A0800000A0B8
:10FD6800A00000A0102801D1084B04E0B0F5807F66
:10FD78000CBF074B074B5B6813EA010004D013EA7A
:10FD8800D1010CBF00200120704700BF600000A017
:10FD9800800000A0A00000A0102804D1084B5A68D9
:10FDA80022EAD10109E0B0F5807F0CBF054B064B74
:10FDB8005A684FEAD10122EA01015960704700BF31
:10FDC800600000A0800000A0A00000A008B52C4B97
:10FDD800984205D10120014600F048FC012048E086
:10FDE800284B984205D10220012100F03FFC022057
:10FDF8003FE0254B984205D10420012100F036FC54
:10FE0800042036E0214B984205D10820012100F05A
:10FE18002DFC08202DE01E4B984205D11020012111
:10FE280000F024FC102024E01A4B984205D1202031
:10FE3800012100F01BFC20201BE0174B984205D144
:10FE48004020012100F012FC402012E0134B9842A0
:10FE580005D18020012100F009FC802009E0104B29
:10FE680098420BD14FF48070012100F0FFFB4FF452
:10FE780080700021BDE8084000F0F8BB08BD00BF55
:10FE8800000002400004024000080240000C02404A
:10FE9800001002400014024000180240001C0240FA
:10FEA800002002402DE9F0470023D1F800801A46CF
:10FEB8004FF0010C03270CFA02F404EA0805A542E6
:10FEC8002ED1066817FA03F4E443264006600E793B
:10FED800D0F8009006FA03FA013E4AEA0909012E11
:10FEE800C0F8009014D8866891F80590264086607E
:10FEF800866809FA03F949EA06068660466826EA2A
:10FF0800050545608D7946689540ADB23543456035
:10FF1800C5682C40C460CC79C5689C402C43C4603B
:10FF280001320233102AC6D1BDE8F0874FF6FF73BD
:10FF380003600023037143718371C371704782B0FA
:10FF48004FF480330193019B0B430193019BC361E1
:10FF5800C161019BC361C3690193C369019302B085
:10FF68007047036919420CBF0020012070470069DF
:10FF780080B27047436919420CBF002001207047C6
:10FF8800406980B2704701837047418370470AB166
:10FF980001837047418370474161704743694B4013
:10FFA8004361704701F00703C908083130B59B0069
:10FFB80050F821500F249C4025EA040440F82140C1
:10FFC80050F8214012FA03F31C4340F8214030BD99
:10FFD80008B5134B984207D14FF40010012100F0E7
:10FFE80069FB4FF4001014E00E4B984207D14FF410
:08FFF8008000012100F05EFB16
:020000040801F1
:100000004FF4800009E00A4B98420BD14FF40000F6
:10001000012100F053FB4FF400000021BDE808402F
:1000200000F04CBB08BD00BF005400400058004029
:10003000005C00407FB50446868868460D4600F0A7
:100040006DFA02992C482B6826F03F063604B1FB66
:10005000F0F0360C80B20643A680228822F001021E
:100060001204120C2280254A93420AD85B00B1FB8D
:10007000F3F301309BB280B22084032B98BF04239A
:1000800021E0EE884BF6FF72964205D103225343DE
:10009000B1FBF3F39BB206E019225343B1FBF3F338
:1000A0009BB243F480431A054FF4967208BF43F0A5
:1000B000010350434FF47A7290FBF2F0013080B2AA
:1000C00043F400432084A38323886989AA889BB2D0
:1000D00043F001032380238823F4816323F0020388
:1000E0001B040A431B0C13439BB223802A89AB8950
:1000F00013439BB223817FBD40420F00A0860100C5
:1001000041F288330360002383804BF6FF72038142
:1001100043814FF48043C28083817047038819B1C3
:100120009BB243F0010303E023F001031B041B0C0B
:1001300003807047038819B19BB243F4807303E0D6
:1001400023F480731B041B0C03807047038819B1D0
:100150009BB243F4007303E023F400731B041B0CF5
:100160000380704712B141F0010101E001F0FE018E
:1001700001827047038819B19BB243F4806303E0A6
:1001800023F480631B041B0C0380704783899BB29C
:1001900001F0FE0123F0FE030B4383817047838946
:1001A00019B19BB243F0010303E023F001031B04E8
:1001B0001B0C83817047038819B19BB243F0400345
:1001C00003E023F040031B041B0C038070470388EB
:1001D00029B16FEA43436FEA53439BB201E05B04EA
:1001E0005B0C03807047038819B99BB243F080030E
:1001F00003E023F080031B041B0C03807047B1F560
:10020000804F838B04D023F480431B041B0C02E03B
:100210009BB243F4804383837047B1F5006F03883A
:1002200003D19BB243F4006303E023F400631B0497
:100230001B0C03807047B1F5005F038803D19BB2AC
:1002400043F4005303E023F400531B041B0C03800E
:100250007047038819B19BB243F0100303E023F009
:1002600010031B041B0C0380704701827047008A37
:10027000C0B27047038819B19BB243F4805303E0C6
:1002800023F480531B041B0C03807047B1F5006FEF
:10029000038803D19BB243F4006303E023F40063BB
:1002A0001B041B0C03807047038819B19BB243F0F9
:1002B000200303E023F020031B041B0C0380704782
:1002C000008BC0F307207047838819B19BB243F4B9
:1002D000006303E023F400631B041B0C838070475E
:1002E000838819B19BB243F4805303E023F4805315
:1002F0001B041B0C8380704782B000230193019084
:10030000019BCB180193019B188880B202B0704703
:1003100083889BB20AB1194301E023EA010181807D
:100320007047838A008B9BB243EA0040084020F06C
:100330007F40431A584240EB03007047838A008B8A
:100340009BB243EA004020F07F40704782B0002318
:10035000009301930B0F01900093009B21F07F41CC
:1003600013B1019B143302E0019B090C1833019374
:10037000019B1B6819420CBF0020012002B070478E
:10038000C94389B2818270478388808A80B20840DD
:100390009BB206D001F0E06113EA11410CBF0020CE
:1003A00001207047C94389B2818270470A4B1A689D
:1003B00042F001021A6000229A60196821F08471EB
:1003C00021F48031196005495960196821F48021B0
:1003D0001960DA60704700BF003802401030002416
:1003E000024B00221A701870704700BF023802409A
:1003F000034B1A6822F0F80242EAC0021A60704702
:1004000000380240014B1860704700BF00004742AF
:10041000064B002201281A701A7002D0042804D159
:1004200001E01870704705221A707047703802405A
:10043000014B1860704700BF800E4742014341EAFC
:10044000821200995B08013B42EA016141EA0341E3
:10045000014B5960704700BF00380240014B1860E3
:10046000704700BF600047428001034B40EA0171C2
:10047000C3F88410704700BF00380240014B186079
:10048000704700BF68004742014B1860704700BFCB
:100490004C004742034B9A6822F0EC6202430A4345
:1004A0009A60704700380240034B9A6822F0784205
:1004B00002430A439A60704700380240034B9A682F
:1004C00022F0030202439A60704700BF00380240E6
:1004D000024B986800F00C00704700BF00380240E3
:1004E000034B9A6822F0F00202439A60704700BF03
:1004F00000380240034B9A6822F4E05202439A60AB
:10050000704700BF00380240034B9A6822F46042F3
:1005100042EAC0029A607047003802401E4B9A6857
:1005200002F00C02042A10B503D0082A03D01B4B9A
:1005300018E01B4B16E059685A6811F4800F59688F
:1005400014BF174B154B02F03F02B3FBF2F3124AF4
:100550005268C2F30142C1F3881101324B43520089
:10056000B3FBF2F30C4903608B680E4A0468C3F3D3
:100570000313D35C34FA03F343608C68C4F382241E
:10058000145D33FA04F484608968C1F34231525C2B
:10059000D340C36010BD00BF003802400024F40007
:1005A00000127A001003002000F44073B3F5407F7E
:1005B000084B08D1996820F0704221F4F81122F418
:1005C00040720A439A601A6F000542EA1050186799
:1005D000704700BF00380240014B1860704700BFF1
:1005E0003C0E4742014B1860704700BF400E474227
:1005F000014B1860704700BF5C014742044B1A6B07
:1006000009B1104301E022EA00001863704700BFFF
:1006100000380240044B5A6B09B1104301E022EA52
:1006200000005863704700BF00380240044B9A6BCB
:1006300009B1104301E022EA00009863704700BF4F
:1006400000380240044B1A6C09B1104301E022EA61
:1006500000001864704700BF00380240044B5A6C19
:1006600009B1104301E022EA00005864704700BF5E
:1006700000380240044B1A6909B1104301E022EA34
:1006800000001861704700BF00380240044B5A69EF
:1006900009B1104301E022EA00005861704700BF31
:1006A00000380240044B9A6909B1104301E022EA84
:1006B00000009861704700BF00380240044B1A6A7E
:1006C00009B1104301E022EA00001862704700BF40
:1006D00000380240044B5A6A09B1104301E022EA93
:1006E00000005862704700BF00380240044B1A6D8A
:1006F00009B1104301E022EA00001865704700BF0D
:1007000000380240044B5A6D09B1104301E022EA5F
:1007100000005865704700BF00380240044B9A6DD6
:1007200009B1104301E022EA00009865704700BF5C
:1007300000380240044B1A6E09B1104301E022EA6E
:1007400000001866704700BF00380240044B5A6E24
:1007500009B1104301E022EA00005866704700BF6B
:1007600000380240044B1A7809B1104301E022EA34
:1007700000001870704700BF0D3802404309012B7C
:10078000074A01D1136803E0022B0CBF136F536FAC
:1007900000F01F0033FA00F000F00100704700BFC6
:1007A0000038024007B5002301933120FFF7E6FF30
:1007B000019B01330193019BB3F5A06F01D0002889
:1007C000F3D03120FFF7DAFF003018BF01200EBD53
:1007D000024B5A6F42F080725A67704700380240ED
:1007E000034BDB6818420CBF00200120704700BF9C
:1007F00000380240014B1870704700BF0E380240AD
:1008000008B5154B98420BD101214FF48050FFF7EA
:1008100061FF4FF480500021BDE80840FFF75ABF48
:100820000E4B984207D14FF480400121FFF746FF5D
:100830004FF4804009E00A4B98420BD14FF400403E
:100840000121FFF73BFF4FF400400021BDE80840C5
:10085000FFF734BF08BD00BF003001400038004042
:10086000003C00400B88028810B54C8823438C88DC
:100870002343CC8823430C8923434C8923438C890D
:100880002343CC8902F44152234313439BB2038098
:10089000838B23F400631B041B0C83830B8A03826A
:1008A00010BD838B23F47B6323F00F031B041B0C0D
:1008B0008383022303848B68F0B5858B022BADB252
:1008C00038D0294A8E889468002E14BF022601264B
:1008D000240203D5946824F400049460D2F8844080
:1008E000D2F884705268DFF884C002F03F02BCFB8B
:1008F000F2F2C4F388145443C7F30272B4FBF2F467
:10090000CA88B2F5007F4FF00A0201D1240A02E042
:100910007601B4FBF6F46243B2FBF3F305330A222B
:100920009BB2B3FBF2F303F001021202C3F34F03D5
:1009300092B200E000229C1EA4B2FE2C28BF00222E
:10094000CC8828BF0223134323439BB203840B8824
:100950004A882B4343F4006313438A8813438A89EC
:1009600013439BB28383F0BD0038024000127A002B
:100970000023038043808380C3800381438183817C
:10098000C381072303827047002302220380438030
:100990008380C380826083817047038819B19BB2D2
:1009A00043F0400303E023F040031B041B0C0380CF
:1009B0007047838B19B19BB243F4806303E023F447
:1009C00080631B041B0C83837047038823F400633C
:1009D0001B041B0C038003889BB20B4303807047EE
:1009E000B1F5804F038803D19BB243F4804303E009
:1009F00023F480431B041B0C038070474FF6FF63F6
:100A00009942038803D09BB243F4807303E023F43C
:100A100080731B041B0C03807047838819B19BB241
:100A200043F0040303E023F004031B041B0C838046
:100A30007047838819B19BB243F0100303E023F0A1
:100A400010031B041B0C83807047838B23F47B6390
:100A500023F00F031B041B0C8383022303840B88E6
:100A6000828BB3F5007F10B592B205D0002B0CBF7E
:100A70004FF48073002301E04FF480734C882243CD
:100A80008C88898942F4006222430A4392B213435C
:100A9000838310BD808980B270478181704703884D
:100AA00019B19BB243F4005303E023F400531B0439
:100AB0001B0C0380704703889BB243F48053038070
:100AC0007047012902D0008B80B27047808A80B2C3
:100AD0007047008A80B2704783889BB20AB119437D
:100AE00001E023EA010181807047090901238B405D
:100AF0009BB21AB1828892B2134303E0828892B209
:100B000022EA030383807047038919420CBF002047
:100B100001207047C94389B20181704710B58488AC
:100B20000089012301F00F0280B213FA02F2104093
:100B3000A4B205D009098B401C420CBF0020012043
:100B400010BD01F00F0101238B40DB439BB20381F9
:100B5000704700BF08B501214FF48040FFF7BAFD90
:100B60004FF480400021BDE80840FFF7B3BD014BC2
:100B7000186070470038014001F0030289080A4BF1
:100B8000023130B5920053F821500F24944025EAE9
:100B9000040443F8214053F8214010FA02F21443B0
:100BA00043F8214030BD00BF00380140014B1860C0
:100BB000704700BFDC002742014B1860704700BF40
:100BC00000042742024B186AC0F30020704700BFA0
:100BD0000038014030B5048C24F001042404240CB6
:100BE0000484058B048CADB2A4B225F0F305154343
:100BF00024F00A0445EA031544F00104ADB20C43A5
:100C00000583048430BD30B5048C24F01004240422
:100C1000240C0484048B058C24F44074ADB22405A8
:100C2000240D25F0A00544EA022445F0100544EA0D
:100C3000033445EA0115A4B2ADB20483058430BD86
:100C400008B5474B984205D101200146FFF742FD08
:100C500001203DE0B0F1804F05D101200146FFF7B2
:100C60002DFD012076E03F4B984205D10220012165
:100C7000FFF724FD02206DE03B4B984205D1042094
:100C80000121FFF71BFD042064E0384B984205D199
:100C900008200121FFF712FD08205BE0344B984249
:100CA00005D110200121FFF709FD102052E0314B42
:100CB000984205D120200121FFF700FD202049E0C6
:100CC0002D4B984209D102200121FFF703FD02209C
:100CD0000021BDE80840FFF7FDBC284B984207D132
:100CE0004FF480300121FFF7F5FC4FF48030EFE73F
:100CF000234B984207D14FF400300121FFF7EAFC63
:100D00004FF40030E4E71F4B984207D14FF48020A6
:100D10000121FFF7DFFC4FF48020D9E71A4B9842FE
:100D200005D140200121FFF7C9FC402012E0174BFC
:100D3000984205D180200121FFF7C0FC802009E006
:100D4000134B98420BD14FF480700121FFF7B6FC92
:100D50004FF480700021BDE80840FFF7AFBC08BD2C
:100D6000000001400004004000080040000C00406A
:100D70000010004000140040000401400040014009
:100D8000004401400048014000180040001C0040A1
:100D9000002000401C4A038890429BB212D002F50A
:100DA000806290420ED0B0F1804F0BD0A2F580321D
:100DB000904207D002F58062904203D002F5806233
:100DC000904203D14A8823F0700313430F4A9042A4
:100DD00008D002F58062904204D023F440730A895F
:100DE0009BB2134303804B68C3620B880385064B99
:100DF000984203D003F58063984201D18B7A038631
:100E000001238382704700BF0000014000100040B2
:100E10004FF0FF33436000230380038143808372DC
:100E20007047018582827047038823F070031B049A
:100E30001B0C0B430380704741627047C1627047CF
:100E4000406A7047008D80B27047038819B19BB229
:100E500043F0020303E023F002031B041B0C038096
:100E60007047038819B19BB243F0040303E023F0F9
:100E700004031B041B0C03807047038819B19BB249
:100E800043F0800303E023F080031B041B0C03806A
:100E90007047038823F008031B041B0C038003889E
:100EA0009BB20B4303807047038823F440731B04F9
:100EB0001B0C038003889BB20B430380704703889D
:100EC00019B19BB243F0010303E023F001031B04BB
:100ED0001B0C03807047038C23F001031B041B0CC5
:100EE000038470B5038C8488028B0D884E8822F0B1
:100EF00073021204120C2A438D8923F002031B048F
:100F000035431B0CADB22B430E4DA842A4B203D007
:100F100005F58065A8420ED1CD894E8A23F00803DD
:100F20002B438D8823F004032B430D8A354324F48F
:100F30004074ADB22C43848002838A684263038488
:100F400070BD00BF00000140038C23F010031B04A0
:100F50001B0C0384038C828830B5048B0D8824F429
:100F6000E6442404240C23F0200344EA05241B0453
:100F70008D891B0C43EA05134D8843EA0513134D75
:100F8000A84292B2A4B29BB203D005F58065A842F4
:100F900015D1CD8923F080039BB243EA05134FF6A8
:100FA000BF751D408B8845EA03130D8A22F4406209
:100FB00042EA85024D8A42EA85029BB292B2828061
:100FC0008A6804838263038430BD00BF000001404F
:100FD000038C23F480731B041B0C0384038C828812
:100FE00030B5848B0D8824F073042404240C23F47E
:100FF00000731B042C438D891B0C43EA05234D8889
:1010000043EA0523124DA84292B29BB203D005F5E4
:101010008065A84215D1CD8923F400639BB243EAD1
:1010200005234FF6FF351D408B8845EA03230D8AC3
:1010300022F4405242EA05124D8A42EA05129BB25E
:1010400092B282808A688483C263038430BD00BF09
:1010500000000140038C23F480531B041B0C038409
:10106000038C30B58488828B0D8822F4E64212040A
:10107000120C23F4005342EA05221B048D891B0C39
:1010800043EA05334D8843EA05330B4DA842A4B229
:1010900092B29BB203D005F58065A84205D10D8AB6
:1010A00024F4804444EA8514A4B2848082838A684C
:1010B0000264038430BD00BF0000014000230380B0
:1010C0004380838083608381C3810382438270472E
:1010D00030B5058C0124ADB28C4025EA040400F142
:1010E0001803048409B1082907D149084FF68F7005
:1010F000CC582040C850C8580AE00439C1F34E010A
:1011000048F6FF70CC582040C8501202C85892B21E
:101110000243CA5030BD4163704781637047C16369
:10112000704701647047038B23F070031B041B0C92
:101130000B4303837047038B23F4E0431B041B0C16
:1011400043EA01239BB203837047838B23F0700330
:101150001B041B0C0B4383837047838B23F4E043F6
:101160001B041B0C43EA01239BB283837047038B50
:1011700023F008031B041B0C0B4303837047038BF2
:1011800023F400631B041B0C43EA01239BB203837B
:101190007047838B23F008031B041B0C0B438383D2
:1011A0007047838B23F400631B041B0C43EA012369
:1011B0009BB283837047038B23F004031B041B0C37
:1011C0000B4303837047038B23F480631B041B0CC6
:1011D00043EA01239BB203837047838B23F004030C
:1011E0001B041B0C0B4383837047838B23F48063A6
:1011F0001B041B0C43EA01239BB283837047038BC0
:1012000023F080031B041B0C0B4303837047038BE9
:1012100009025B0441EA53439BB203837047838B0B
:1012200023F080031B041B0C0B4383837047838BC9
:1012300009025B0441EA53439BB283837047038CEA
:1012400023F002031B041B0C0B4303847047038C25
:1012500023F008031B041B0C0B4303847047038C0F
:1012600023F020031B041B0C43EA01139BB20384ED
:101270007047038C23F080031B041B0C43EA01130B
:101280009BB203847047038C23F400731B041B0C74
:1012900043EA01239BB203847047038C23F4006369
:1012A0001B041B0C43EA01239BB203847047038C8D
:1012B00023F400531B041B0C43EA01339BB2038449
:1012C000704710B5048C01238B40A4B224EA0303B9
:1012D0000384038C12FA01F10B439BB2038410BD0B
:1012E00010B5048C04238B40A4B224EA03030384C6
:1012F000038C12FA01F10B439BB2038410BD00234F
:101300000122038043808280C38003817047406B49
:101310007047806B7047C06B7047006C7047038BE1
:1013200023F00C031B041B0C0383038B9BB20B43A6
:1013300003837047038B23F440631B041B0C03835C
:10134000038B9BB243EA01239BB203837047F8B53A
:101350000C464988A288B4F800E023890546002994
:101360000CBF02270027012A14BF01260226BEF166
:10137000000F10D1FFF72EFC2846E188FFF7CFFFC2
:101380002846394632462389FFF73DFCE188284646
:10139000BDE8F840CEE7FFF736FC2846E188FFF7C6
:1013A000C9FF2846394632462389FFF713FCE188F6
:1013B0002846BDE8F840B2E7838B23F00C031B04FA
:1013C0001B0C8383838B9BB20B4383837047838B7C
:1013D00023F440631B041B0C8383838B9BB243EA7F
:1013E00001239BB283837047F8B50D460B88AA880A
:1013F000498804463BB92B89FFF7ECFBE988204676
:10140000BDE8F8408BE7042B07D12B89FFF7FBFBE6
:10141000E9882046BDE8F8408CE7082BB5F808C0FD
:10142000078C1DD127F480773F043F0C0784868BFF
:10143000038CB6B29BB226F0F30623F4206346EA8F
:101440000C1C43EA01211FFA8CFC89B24CEA02020F
:1014500041F4807182830184E988BDE8F840ABE7FC
:1014600027F480573F043F0C0784868B038C26F4B7
:10147000407623F4005336055B04360D5B0C46EAD8
:10148000022243EA013342EA0C329BB2E98892B26B
:1014900043F4805382830384BDE8F84097E74A8889
:1014A0000B8813438A881343CA8813430A8913435A
:1014B0004A8913438A8913439BB2A0F8443070478A
:1014C0000023038043808380C38003814381838121
:1014D0007047B0F8443029B16FEA43436FEA534391
:1014E0009BB201E05B045B0CA0F84430704783883A
:1014F00019B19BB243F0040303E023F004031B047F
:101500001B0C83807047838819B19BB243F00103A1
:1015100003E023F001031B041B0C838070478389C5
:101520009BB20AB1194301E023EA010181817047AE
:1015300081827047038A19420CBF00200120704746
:10154000C94389B201827047038A828911EA030084
:1015500092B203D011420CBF002001207047C94352
:1015600089B2018270470A43A0F8482070478389F6
:101570009BB20AB1194301E023EA0101818170475E
:10158000838819B19BB243F0080303E023F00803FA
:101590001B041B0C83807047038923F007031B0483
:1015A0001B0C03817047038923F070031B041B0C81
:1015B0000B43038103899BB243F007030381704708
:1015C00038B50D4611460122602D044602D1FFF7C1
:1015D0001AFB01E0FFF7FEFA238923F070031B04D6
:1015E0001B0C1D43258123899BB243F007032381F4
:1015F00038BD038923F070031B041B0C0B430381CC
:101600007047838823F070031B041B0C838083883E
:101610009BB20B4383807047038923F007031B04AD
:101620001B0C038103899BB20B4303817047038921
:1016300023F080031B041B0C038103899BB20B4323
:101640000381704710B50489E4B20C43144344EAA3
:101650000324A4B2048110BD10B50446FFF7F2FFC5
:1016600023899BB243F48043238110BD10B5044607
:10167000FFF7E8FF238923F077031B041B0C43F0DB
:101680007703238110BD70B50489068B058C26F481
:101690004076ADB226F0030624F00704360425F0A8
:1016A00022052404360C1543240C46F4807645EAC2
:1016B0000315214346F00106ADB20181068305847E
:1016C00070BD838819B19BB243F0800303E023F01F
:1016D00080031B041B0C83807047A0F850107047D8
:1016E00008B5234B984205D110200121FEF7F2FFE7
:1016F000102037E01F4B984207D14FF400300121F2
:10170000FEF7DCFF4FF4003009E01B4B98420BD191
:101710004FF480200121FEF7D1FF4FF480200021FB
:10172000BDE80840FEF7CABF144B984207D14FF4FA
:1017300000200121FEF7C2FF4FF40020EFE7104B1D
:10174000984207D14FF480100121FEF7B7FF4FF404
:101750008010E4E70B4B984209D120200121FEF7CD
:10176000B9FF20200021BDE80840FEF7B3BF08BD47
:10177000001001400044004000480040004C004080
:101780000050004000140140038ACA889BB223F431
:10179000405330B513430D46038283890989AA88D3
:1017A00023F4B0530A43698923F00C031B040A4352
:1017B0001B0C92B213438381838AAA899BB223F4C0
:1017C0004073134385B0838204466846FEF7A6FE45
:1017D0001A4B9C4203D003F580639C4201D1039BCA
:1017E00000E0029BA28912B2002A4FF019012A6878
:1017F00001FB03F101DA520000E092006423B1FB27
:10180000F2F1B1FBF3F21201100903FB1011A089F0
:1018100000B2002806DAC9003231B1FBF3F303F05D
:10182000070305E009013231B1FBF3F303F00F03C5
:101830001A4392B2228105B030BD00BF00100140B2
:101840004FF4165303600C2200238380C38003816E
:101850004281838170470B88028A10B54C882343EC
:101860008C88C988234392B20B4322F470629BB2E6
:101870001343038210BD0023038043808380C38011
:101880007047838919B19BB243F4005303E023F4FA
:1018900000531B041B0C83817047038B03F47F43AD
:1018A0000383038B9BB20B4303837047838929B166
:1018B0006FEA43436FEA53439BB201E05B045B0C66
:1018C00083817047838A19B19BB243F4006303E0BC
:1018D00023F400631B041B0C83827047C905C90DE8
:1018E000818070478088C005C00D7047038A23F04F
:1018F0000F031B041B0C0382038A9BB20B4303825E
:101900007047838919B19BB243F0020303E023F0CF
:1019100002031B041B0C83817047838923F400633B
:101920001B041B0C838183899BB20B43838170470B
:10193000038A23F020031B041B0C0382038A9BB23F
:101940000B4303827047038A19B19BB243F480436F
:1019500003E023F480431B041B0C0382704783893C
:101960009BB243F0010383817047838A19B19BB214
:1019700043F0080303E023F008031B041B0C8382DD
:101980007047038BDBB20383038B9BB243EA0123D3
:1019900003837047838A19B19BB243F0200303E0AD
:1019A00023F020031B041B0C83827047838A19B128
:1019B0009BB243F0100303E023F010031B041B0C45
:1019C00083827047838A23F004031B041B0C8382E9
:1019D000838A9BB20B4383827047838A19B19BB27F
:1019E00043F0020303E023F002031B041B0C838279
:1019F0007047838A9BB20AB1194301E023EA0101CF
:101A000081827047C1F3421310B501F01F01012418
:101A100014FA01F1A34201D10C3004E0022B01D1F0
:101A2000103000E0143003680AB1194301E023EAE2
:101A30000101016010BD038819420CBF0020012084
:101A40007047C94389B201807047012210B501F087
:101A50001F03C1F342149A40012C01D1838903E092
:101A6000022C0CBF038A838A9BB21340028892B275
:101A700043B1090A012313FA01F111420CBF0020FE
:101A8000012010BD184610BD090A01238B40DB431D
:101A90009BB20380704700BF81F0004102E000BFAD
:101AA00083F0004330B54FEA41044FEA430594EA1E
:101AB000050F08BF90EA020F1FBF54EA000C55EA59
:101AC000020C7FEA645C7FEA655C00F0E2804FEA2A
:101AD0005454D4EB5555B8BF6D420CDD2C4480EA0C
:101AE000020281EA030382EA000083EA010180EA3C
:101AF000020281EA0303362D88BF30BD11F0004F8A
:101B00004FEA01314FF4801C4CEA113102D04042BF
:101B100061EB410113F0004F4FEA03334CEA1333FA
:101B200002D0524263EB430394EA050F00F0A78012
:101B3000A4F10104D5F1200E0DDB02FA0EFC22FA0D
:101B400005F2801841F1000103FA0EF2801843FA01
:101B500005F359410EE0A5F120050EF1200E012AF2
:101B600003FA0EFC28BF4CF0020C43FA05F3C01830
:101B700051EBE37101F0004507D54FF0000EDCF1A9
:101B8000000C7EEB00006EEB0101B1F5801F1BD352
:101B9000B1F5001F0CD349085FEA30004FEA3C0C56
:101BA00004F101044FEA445212F5800F80F09A804C
:101BB000BCF1004F08BF5FEA500C50F1000041EB50
:101BC000045141EA050130BD5FEA4C0C404141EB54
:101BD000010111F4801FA4F10104E9D191F0000F7B
:101BE00004BF01460020B1FA81F308BF2033A3F1FE
:101BF0000B03B3F120020CDA0C3208DD02F1140CF5
